:020000040800F2
:1000000000060020E1010008E3010008E301000808
:10001000E3010008E3010008E3010008E301000830
:10002000E3010008E3010008E3010008B92F00081C
:10003000E3010008E3010008E3010008E301000810
:10004000E3010008E3010008E3010008E301000800
:10005000E3010008E301000861320008893200086A
:10006000B1320008D932000801330008E30100086A
:10007000E3010008E3010008E3010008E3010008D0
:10008000E3010008E3010008E3010008E3010008C0
:10009000E3010008E3010008E30100082933000838
:1000A000E3010008E3010008E3010008E3010008A0
:1000B000FD330008E3010008E3010008E301000844
:1000C000E3010008E3010008E3010008E301000880
:1000D000E3010008E3010008E3010008E301000870
:1000E0008D330008E3010008E3010008E301000884
:1000F000E3010008E3010008E3010008E301000850
:10010000E3010008E3010008E3010008E30100083F
:10011000E3010008E3010008E3010008E30100082F
:10012000E3010008E3010008E3010008E30100081F
:10013000E3010008E3010008E3010008E30100080F
:10014000E3010008E3010008E30100086D2700084F
:10015000E3010008E3010008E3010008E3010008EF
:10016000E3010008E3010008E3010008E3010008DF
:10017000E3010008E3010008E3010008E3010008CF
:10018000E3010008E3010008E3010008E3010008BF
:10019000E3010008E3010008E3010008E3010008AF
:1001A000E3010008E3010008E3010008E30100089F
:1001B000E3010008E3010008E3010008E30100088F
:1001C000E3010008E3010008E3010008E30100087F
:1001D000E3010008E3010008E3010008E30100086F
:1001E00002E000F000F8FEE772B6374880F30888B6
:1001F000364880F3098836483649086040F20000E6
:10020000CCF200004EF63471CEF200010860BFF36C
:100210004F8FBFF36F8F40F20000C0F2F0004EF638
:100220008851CEF200010860BFF34F8FBFF36F8F8C
:100230004FF00000E1EE100A4EF63C71CEF20001E4
:100240000860062080F31488BFF36F8F01F056FF1B
:1002500002F050FE4FF055301F491B4A91423CBFFF
:1002600041F8040BFAE71D49184A91423CBF41F896
:10027000040BFAE71A491B4A1B4B9A423EBF51F83E
:10028000040B42F8040BF8E700201849184A914281
:100290003CBF41F8040BFAE701F034FF02F07EFEA8
:1002A000144C154DAC4203DA54F8041B8847F9E7A7
:1002B00000F042F8114C124DAC4203DA54F8041B22
:1002C0008847F9E701F01CBF00060020002200204B
:1002D0000000000808ED00E00000002000060020FB
:1002E000C8370008002200204022002040220020C1
:1002F000602E0020E0010008E0010008E001000895
:10030000E00100082DE9F04F2DED108AC1F80CD066
:10031000C3689D46BDEC108ABDE8F08F002383F3CF
:1003200011882846A047002001F084FAFEE701F07A
:10033000EDF900DFFEE7000038B500F061FB01F0E9
:10034000ADFE054601F0D0FE0446D8B90F4B9D42E4
:100350001AD001339D4218BF044641F2883504BFCC
:1003600001240025002001F0A3FE0CB100F076F876
:1003700000F0ECFC00F09AFB284600F0B7F800F023
:100380006DF8F9E70025EDE70546EBE7010007B05A
:1003900008B500F05DFBA0F120035842584108BDAC
:1003A00007B541F21203022101A8ADF8043000F0B4
:1003B0006DFB03B05DF804FB38B5302383F311887F
:1003C000174803680BB101F001FB164A14480023DB
:1003D0004FF47A7101F0F0FA002383F31188124C84
:1003E000236813B12368013B2360636813B163681A
:1003F000013B63600D4D2B7833B963687BB90220F4
:1004000000F01EFC322363602B78032B07D1636856
:100410002BB9022000F014FC4FF47A73636038BDEE
:1004200040220020B9030008602300205822002049
:10043000084B187003280CD8DFE800F00805020804
:10044000022000F0F3BB022000F0E6BB024B0022CA
:100450005A60704758220020602300201F4B204A1A
:1004600010B51C461968013136D004339342F9D1D6
:100470006268A24230D31B4B9B6803F1006303F513
:1004800040439A4228D2002000F02AFB0220FFF7C6
:10049000CFFF154B1A6C00221A64196E1A66196E7A
:1004A000596C5A64596E5A665A6E1A6942F0005273
:1004B0001A611A6922F000521A611B6972B64FF074
:1004C000E0233021C3F8084DD4E9003281F31188CC
:1004D0009D4683F30888104710BD00BF00C0000888
:1004E00020C0000800220020003802402DE9F04F13
:1004F00093B0AA4B00902022FF210AA89D6800F02B
:10050000CFFBA74A1378A3B9A64801210360117055
:10051000302383F3118803680BB101F057FAA24A24
:10052000A04800234FF47A7101F046FA002383F3C8
:100530001188009B13B19D4B009A1A609C4A009C45
:100540001378032B1EBF00231370984A4FF0000A44
:1005500018BF5360D3465646D146012000F066FBD3
:1005600024B1924B1B68002B00F01182002000F098
:100570006FFA0390039B002BF2DB012000F04CFB91
:10058000039B213B162BE8D801A252F823F000BFB1
:10059000ED05000815060008A90600085B0500081F
:1005A0005B0500085B050008330700080309000825
:1005B0001D0800087F080008A7080008CD080008EB
:1005C0005B050008DF0800085B050008510900080A
:1005D0008D0600085B05000895090008F90500086C
:1005E0008D0600085B0500087F0800080220FFF761
:1005F000CFFE002840F0F581009B0221BAF1000FE8
:1006000008BF1C4605A841F21233ADF8143000F0C3
:100610003DFAA2E74FF47A7000F01AFA071EEBDBFE
:100620000220FFF7B5FE0028E6D0013F052F00F2BB
:10063000DA81DFE807F0030A0D101336052305936E
:10064000042105A800F022FA17E054480421F9E734
:1006500058480421F6E758480421F3E74FF01C08F6
:10066000404600F03FFA08F104080590042105A86F
:1006700000F00CFAB8F12C0FF2D1012000FA07F7C4
:1006800047EA0B0B5FFA8BFB4FF0000900F054FBBD
:1006900026B10BF00B030B2B08BF0024FFF780FEE5
:1006A0005BE746480421CDE7002EA5D00BF00B03F5
:1006B0000B2BA1D10220FFF76BFE074600289BD031
:1006C000012000F00DFA0220FFF7B2FE00261FFA0B
:1006D00086F8404600F014FA044690B100214046E6
:1006E00000F01EFA01360028F1D1BA46044641F264
:1006F0001213022105A8ADF814303E4600F0C6F9E9
:100700002BE70120FFF794FE2546244B9B68AB4264
:1007100007D9284600F0E6F9013040F0678104353A
:10072000F3E7234B00251D70204BBA465D603E4623
:10073000ACE7002E3FF460AF0BF00B030B2B7FF404
:100740005BAF0220FFF774FE322000F081F9B0F1B8
:100750000008FFF651AF18F003077FF44DAF0F4AC2
:10076000926808EB050393423FF646AFB8F5807FE9
:100770003FF742AF124B0193B84523DD4FF47A7037
:1007800000F066F90390039A002AFFF635AF019B4B
:10079000039A03F8012B0137EDE700BF0022002088
:1007A0005C23002040220020B903000860230020C1
:1007B0005822002004220020082200200C220020C1
:1007C0005C220020C820FFF7E3FD074600283FF425
:1007D00013AF1F2D11D8C5F1200242450AAB25F0F9
:1007E000030028BF424683490192184400F032FAC0
:1007F000019A8048FF2100F053FA4FEAA8037D498F
:100800000193C8F38702284600F052FA06460028F2
:100810003FF46DAF019B05EB830537E70220FFF73F
:10082000B7FD00283FF4E8AE00F0A6F900283FF439
:10083000E3AE0027B846704B9B68BB4218D91F2F08
:1008400011D80A9B01330ED027F0030312AA1344D8
:1008500053F8203C05934046042205A900F0A0FA75
:1008600004378046E7E7384600F03CF90590F2E7A8
:10087000CDF81480042105A800F008F906E700234C
:10088000642104A8049300F0F7F800287FF4B4AEC4
:100890000220FFF77DFD00283FF4AEAE049800F083
:1008A00053F90590E6E70023642104A8049300F0BF
:1008B000E3F800287FF4A0AE0220FFF769FD0028CE
:1008C0003FF49AAE049800F04FF9EAE70220FFF7F0
:1008D0005FFD00283FF490AE00F05EF9E1E70220F2
:1008E000FFF756FD00283FF487AE05A9142000F05D
:1008F00059F904210746049004A800F0C7F83946C6
:10090000B9E7322000F0A4F8071EFFF675AEBB076A
:100910007FF472AE384A926807EB090393423FF6C0
:100920006BAE0220FFF734FD00283FF465AE27F0E0
:1009300003074F44B9453FF4A9AE484600F0D2F84A
:100940000421059005A800F0A1F809F10409F1E7D8
:100950004FF47A70FFF71CFD00283FF44DAE00F015
:100960000BF9002844D00A9B01330BD008220AA9B6
:10097000002000F09DF900283AD02022FF210AA88B
:1009800000F08EF9FFF70CFD1C4800F059FF13B082
:10099000BDE8F08F002E3FF42FAE0BF00B030B2BB6
:1009A0007FF42AAE0023642105A8059300F064F8C3
:1009B000074600287FF420AE0220FFF7E9FC8046BE
:1009C00000283FF419AEFFF7EBFC41F2883000F04D
:1009D00037FF059800F0E2F9464600F0ADF93C46D5
:1009E000BBE5064652E64FF0000905E6BA467EE64C
:1009F00037467CE65C22002000220020A086010011
:100A00007047000070B50F4B1B780133DBB2012B30
:100A10000C4611D80C4D29684FF47A730E6AA2FB6C
:100A20000332014622462846B047844204D1074B90
:100A300000221A70012070BD4FF4FA7000F000FF20
:100A40000020F8E710220020082600209423002030
:100A500007B50023024601210DF107008DF807308C
:100A6000FFF7D0FF20B19DF8070003B05DF804FB4D
:100A70004FF0FF30F9E700000A4608B50421FFF700
:100A8000C1FF80F00100C0B2404208BD30B4054C47
:100A90002368DD69044B0A46AC460146204630BC5B
:100AA000604700BF08260020A086010070B501F055
:100AB000E7F9094E094D30800024286833888342C5
:100AC00008D901F0D7F92B6804440133B4F5404F3D
:100AD0002B60F2D370BD00BF962300206823002056
:100AE00001F090BA00F1006000F5404000687047E6
:100AF00000F10060920000F5404001F00FBA0000E4
:100B0000054B1A68054B1B889B1A834202D9104477
:100B100001F0B0B900207047682300209623002020
:100B200038B5084D044629B128682044BDE838404E
:100B300001F0C0B92868204401F0A4F90028F3D0DE
:100B400038BD00BF6823002010F003030AD1B0F5C0
:100B5000047F05D200F10050A0F51040D0F8003815
:100B6000184670470023FBE700F10050A0F5104045
:100B7000D0F8100A70470000064991F8243033B1CC
:100B80000023086A81F824300822FFF7B1BF012052
:100B9000704700BF6C230020014B1868704700BFEE
:100BA000002004E070B5194B1D68194B0138C5F3DE
:100BB0000B0408442D0C04221E88A6420BD15C684D
:100BC0000A46013C824213460FD214F9016F4EB11E
:100BD00002F8016BF6E7013A03F10803ECD1814218
:100BE0000B4602D22C2203F8012B0A4A0524168850
:100BF000AE4204D1984284BF967803F8016B013C61
:100C000002F10402F3D1581A70BD00BF002004E0C5
:100C1000E0340008CC340008022802BF024B4FF039
:100C200080729A61704700BF00000240022802BF34
:100C3000024B4FF480729A61704700BF000002407F
:100C4000022801BF024A536983F4807353617047DD
:100C50000000024010B50023934203D0CC5CC45482
:100C60000133F9E710BD000010B5013810F9013F5C
:100C70003BB191F900409C4203D11AB10131013AD4
:100C8000F4E71AB191F90020981A10BD1046FCE75C
:100C900003460246D01A12F9011B0029FAD1704707
:100CA00002440346934202D003F8011BFAE770475F
:100CB0002DE9F8431F4D144695F824200746884631
:100CC00052BBDFF870909CB395F824302BB92022EA
:100CD000FF2148462F62FFF7E3FF95F82400C0F19B
:100CE0000802A24228BF2246D6B24146920005EB36
:100CF0008000FFF7AFFF95F82430A41B1E44F6B226
:100D0000082E17449044E4B285F82460DBD1FFF745
:100D100033FF0028D7D108E02B6A03EB820383421C
:100D2000CFD0FFF729FF0028CBD10020BDE8F88302
:100D30000120FBE76C230020024B1A78024B1A704B
:100D4000704700BF942300201022002010B50F4CE4
:100D50000F4800F0B5F821460D4800F0DDF8246892
:100D60000C48626DD2F8043843F00203C2F804382C
:100D700000F066FD0849204600F0D4F9626DD2F813
:100D8000043823F00203C2F8043810BDAC35000863
:100D90000826002040420F00B435000870470000CC
:100DA00030B5094D0A4491420DD011F8013B58402D
:100DB000082340F30004013B2C4013F0FF0384EAB6
:100DC0005000F6D1EFE730BD2083B8ED02684368EC
:100DD0001143016003B118477047000013B5446B1D
:100DE000D4F894341A681178042915D1217C022989
:100DF00012D11979128901238B4013420CD101A918
:100E000004F14C0001F032FFD4F89444019B2179A5
:100E10000246206800F0D0F902B010BD143001F095
:100E2000B5BE00004FF0FF33143001F0AFBE00003C
:100E30004C3001F087BF00004FF0FF334C3001F021
:100E400081BF0000143001F083BE00004FF0FF317D
:100E5000143001F07DBE00004C3001F053BF0000A3
:100E60004FF0FF324C3001F04DBF000000207047C2
:100E700010B5D0F894341A6811780429044617D1B3
:100E8000017C022914D15979528901238B401342E4
:100E90000ED1143001F016FE024648B1D4F8944445
:100EA0004FF4807361792068BDE8104000F072B99A
:100EB00010BD0000406BFFF7DBBF00007047000073
:100EC0007FB5124B036000234360C0E90233012564
:100ED00002260F4B057404460290019300F1840230
:100EE000294600964FF48073143001F0C7FD094B7A
:100EF0000294CDE9006304F523724FF48073294610
:100F000004F14C0001F08EFE04B070BD0035000805
:100F1000B50E0008DD0D00080B68302282F3118841
:100F20000A7903EB820290614A79093243F8220080
:100F30008A7912B103EB820398610223C0F89414FA
:100F40000374002080F311887047000038B5037FD8
:100F5000044613B190F85430ABB9201D012502218D
:100F6000FFF734FF04F1140025776FF0010100F062
:100F70008FFC84F8545004F14C006FF00101BDE87F
:100F8000384000F085BC38BD10B50121044604305E
:100F9000FFF71CFF0023237784F8543010BD0000B6
:100FA00038B504460025143001F080FD04F14C00F2
:100FB000257701F04FFE201D84F854500121FFF7E2
:100FC00005FF2046BDE83840FFF752BF90F8443097
:100FD00003F06003202B07D190F84520212A4FF021
:100FE000000303D81F2A06D800207047222AFBD10D
:100FF000C0E90E3303E0034A82630722C26303643D
:10100000012070471122002037B5D0F894341A68B7
:101010001178042904461AD1017C022917D11979C3
:10102000128901238B40134211D100F14C0528464F
:1010300001F0D0FE58B101A9284601F017FED4F8FE
:101040009444019B21790246206800F0B5F803B072
:1010500030BD0000F0B500EB810385B09E69044609
:101060000D46FEB1302383F3118804EB8507301D54
:101070000821FFF7ABFEFB685B691B6806F14C00BB
:101080001BB1019001F000FE019803A901F0EEFDF3
:10109000024648B1039B2946204600F08DF8002304
:1010A00083F3118805B0F0BDFB685A691268002A05
:1010B000F5D01B8A013B1340F1D104F14402EAE769
:1010C000093138B550F82140DCB1302383F3118861
:1010D000D4F894241368527903EB8203DB689B698C
:1010E0005D6845B104216018FFF770FE294604F1E0
:1010F000140001F0F1FC2046FFF7BAFE002383F351
:10110000118838BD7047000001F050B8012303700A
:101110000023C0E90133C36183620362C362436297
:101120000363704738B50446302383F311880025E4
:10113000C0E90355C0E90555416001F047F80223B5
:10114000237085F31188284638BD000070B500EB88
:10115000810305465069DA600E46144618B1102224
:101160000021FFF79DFDA06918B110220021FFF7B3
:1011700097FD31462846BDE8704001F0F1B8000007
:10118000826802F0011282600022C0E904228261BA
:1011900001F072B9F0B400EB81044789E4680125DD
:1011A000A4698D403D43458123600023A2606360B4
:1011B000F0BC01F08DB90000F0B400EB81040789A8
:1011C000E468012564698D403D4305812360002367
:1011D000A2606360F0BC01F007BA000070B50223A2
:1011E000002504460370C0E90255C0E90455C564F2
:1011F000856180F8345001F04FF863681B6823B1B3
:1012000029462046BDE87040184770BD0378052B7D
:1012100010B504460AD080F85030052303704368A7
:101220001B680BB1042198470023A36010BD000088
:101230000178052906D190F85020436802701B6898
:1012400003B118477047000070B590F83430044679
:1012500013B1002380F8343004F14402204601F039
:101260002DF963689B68B3B994F8443013F06005B6
:1012700035D00021204601F0CDFB0021204601F0B1
:10128000BFFB63681B6813B10621204698470623FD
:1012900084F8343070BD204698470028E4D0B4F874
:1012A0004A30E26B9A4288BFE36394F94430E56BBD
:1012B000002B4FF0300380F20381002D00F0F2800C
:1012C000092284F8342083F311880021D4E90E2305
:1012D0002046FFF771FF002383F31188DAE794F8C3
:1012E000452003F07F0343EA022340F20232934297
:1012F00000F0C58021D8B3F5807F48D00DD8012BF0
:101300003FD0022B00F09380002BB2D104F14C02AD
:10131000A2630222E2632364C1E7B3F5817F00F098
:101320009B80B3F5407FA4D194F84630012BA0D127
:10133000B4F84C3043F0020332E0B3F5006F4DD007
:1013400017D8B3F5A06F31D0A3F5C063012B90D8A7
:10135000636894F846205E6894F84710B4F8483003
:101360002046B047002884D04368A3630368E36342
:101370001AE0B3F5106F36D040F6024293427FF484
:1013800078AF5C4BA3630223E3630023C3E794F8C5
:101390004630012B7FF46DAFB4F84C3023F00203DC
:1013A000C4E90E55A4F84C30256478E7B4F844300D
:1013B000B3F5A06F0ED194F8463084F84E30204635
:1013C00000F0C2FF63681B6813B1012120469847F3
:1013D000032323700023C4E90E339CE704F14F0379
:1013E000A3630123C3E72378042B10D1302383F3B5
:1013F00011882046FFF7C4FE85F311880321636836
:1014000084F84F5021701B680BB12046984794F820
:101410004630002BDED084F84F30042323706368FD
:101420001B68002BD6D0022120469847D2E794F8BB
:1014300048301D0603F00F0120460AD501F030F8B0
:10144000012804D002287FF414AF2B4B9AE72B4BD2
:1014500098E701F017F8F3E794F84630002B7FF493
:1014600008AF94F8483013F00F01B3D01A062046A5
:1014700002D501F0E3FAADE701F0D6FAAAE794F855
:101480004630002B7FF4F5AE94F8483013F00F018E
:10149000A0D01B06204602D501F0BCFA9AE701F065
:1014A000AFFA97E7142284F8342083F311882B468F
:1014B0002A4629462046FFF76DFE85F31188E9E6A6
:1014C0005DB1152284F8342083F311880021D4E91A
:1014D0000E232046FFF75EFEFDE60B2284F8342043
:1014E00083F311882B462A4629462046FFF764FEDF
:1014F000E3E700BF30350008283500082C35000828
:1015000038B590F834300446002B3ED0063BDAB2B2
:101510000F2A34D80F2B32D8DFE803F037313108E7
:10152000223231313131313131313737C56BB0F899
:101530004A309D4214D2C3681B8AB5FBF3F203FB09
:1015400012556DB9302383F311882B462A4629465C
:10155000FFF732FE85F311880A2384F834300EE059
:10156000142384F83430302383F3118800231A467F
:1015700019462046FFF70EFE002383F3118838BD7D
:10158000036C03B198470023E7E70021204601F0F0
:1015900041FA0021204601F033FA63681B6813B159
:1015A0000621204698470623D7E7000010B590F89B
:1015B0003430142B044629D017D8062B05D001D877
:1015C0001BB110BD093B022BFBD80021204601F0C6
:1015D00021FA0021204601F013FA63681B6813B159
:1015E000062120469847062319E0152BE9D10B2345
:1015F00080F83430302383F3118800231A461946CB
:10160000FFF7DAFD002383F31188DAE7C3689B69EB
:101610005B68002BD5D1036C03B19847002384F895
:101620003430CEE700230375826803691B6899682C
:101630009142FBD25A680360426010605860704764
:1016400000230375826803691B6899689142FBD87F
:101650005A680360426010605860704708B50846D9
:10166000302383F311880B7D032B05D0042B0DD081
:101670002BB983F3118808BD8B6900221A604FF0E3
:10168000FF338361FFF7CEFF0023F2E7D1E9003299
:1016900013605A60F3E70000FFF7C4BF054BD96839
:1016A0000875186802681A60536001220275D860D4
:1016B000FEF728BE9823002030B50C4BDD684B1C8C
:1016C00087B004460FD02B46094A684600F074F9EB
:1016D0002046FFF7E3FF009B13B1684600F076F960
:1016E000A86907B030BDFFF7D9FFF9E798230020BC
:1016F0005D160008044B1A68DB6890689B68984286
:1017000094BF00200120704798230020084B10B59B
:101710001C68D86822681A60536001222275DC6058
:10172000FFF78EFF01462046BDE81040FEF7EABDF8
:1017300098230020044B1A68DB6892689B689A42E1
:1017400001D9FFF7E3BF70479823002038B5074C55
:1017500007490848012300252370656001F072FBEA
:101760000223237085F3118838BD00BF00260020B6
:10177000383500089823002000F05EB9EFF311809F
:1017800020B9EFF30583302282F3118870470000FF
:1017900010B530B9EFF30584C4F3080414B180F335
:1017A000118810BDFFF7C6FF84F31188F9E7000028
:1017B000034A516853685B1A9842FBD8704700BFD0
:1017C000001000E08B60022308618B82084670479E
:1017D0008368A3F1840243F8142C026943F8442C73
:1017E000426943F8402C094A43F8242CC26843F864
:1017F000182C022203F80C2C002203F80B2C044AAC
:1018000043F8102CA3F12000704700BF1D0300080F
:101810009823002008B5FFF7DBFFBDE80840FFF77D
:101820003BBF0000024BDB6898610F20FFF736BF1B
:1018300098230020302383F31188FFF7F3BF0000C3
:1018400008B50146302383F311880820FFF734FFE1
:10185000002383F3118808BD064BDB6839B1426869
:1018600018605A60136043600420FFF725BF4FF0F3
:10187000FF307047982300200368984206D01A680A
:101880000260506099611846FFF706BF704700007C
:1018900038B504460D462068844200D138BD03683F
:1018A00023605C608561FFF7F7FEF4E710B503681D
:1018B0009C68A2420CD85C688A600B604C60216016
:1018C000596099688A1A9A604FF0FF33836010BD9F
:1018D0001B68121BECE700000A2938BF0A2170B50B
:1018E00004460D460A26601901F0A6FA01F092FAA4
:1018F000041BA54203D8751C2E460446F3E70A2EA6
:1019000004D9BDE87040012001F0DCBA70BD0000D0
:10191000F8B5144B0D46D96103F1100141600A2A54
:101920001969826038BF0A22016048601861A818EE
:10193000144601F073FA0A2701F06CFA431BA34224
:10194000064606D37C1C281901F076FA2746354650
:10195000F2E70A2F04D9BDE8F840012001F0B2BA3D
:10196000F8BD00BF98230020F8B506460D4601F0EB
:1019700051FA0F4A134653F8107F9F4206D12A4668
:1019800001463046BDE8F840FFF7C2BFD169BB68E9
:10199000441A2C1928BF2C46A34202D92946FFF726
:1019A0009BFF224631460348BDE8F840FFF77EBF63
:1019B00098230020A823002010B4C0E903230023AB
:1019C0005DF8044B4361FFF7CFBF000010B5194C21
:1019D000236998420DD0D0E90032816813605A60C3
:1019E0009A680A449A60002303604FF0FF33A361B2
:1019F00010BD2346026843F8102F53600022026096
:101A000022699A4203D1BDE8104001F00FBA9368F1
:101A100081680B44936001F0FDF92269E1699268E5
:101A2000441AA242E4D91144BDE81040091AFFF754
:101A300053BF00BF982300202DE9F047DFF8BC809A
:101A400008F110072C4ED8F8105001F0E3F9D8F83F
:101A50001C40AA68031B9A423ED81444D5E90032C0
:101A60004FF00009C8F81C4013605A60C5F8009098
:101A7000D8F81030B34201D101F0D8F989F31188B8
:101A8000D5E9033128469847302383F311886B69E1
:101A9000002BD8D001F0BEF96A69A0EB04094A45D1
:101AA00082460DD2022001F00DFA0022D8F8103043
:101AB000B34208D151462846BDE8F047FFF728BF9A
:101AC000121A2244F2E712EB090938BF4A462946A6
:101AD0003846FFF7EBFEB5E7D8F81030B34208D030
:101AE0001444211AC8F81C00A960BDE8F047FFF7AC
:101AF000F3BEBDE8F08700BFA82300209823002094
:101B000000207047FEE70000704700004FF0FF30F4
:101B10007047000002290CD0032904D0012907488E
:101B200018BF00207047032A05D8054800EBC20003
:101B30007047044870470020704700BF1036000807
:101B400020220020C435000870B59AB0054608462A
:101B500001A9144600F0C2F801A8FFF799F8431C48
:101B60005B00C5E900340022237003236370C6B212
:101B700001AB02341046D1B28E4204F1020401D806
:101B80001AB070BD13F8011B04F8021C04F8010C14
:101B90000132F0E708B5302383F311880348FFF7DB
:101BA00033FA002383F3118808BD00BF0826002004
:101BB00090F8443003F01F02012A07D190F8452025
:101BC0000B2A03D10023C0E90E3315E003F06003B4
:101BD000202B08D1B0F848302BB990F84520212AA5
:101BE00003D81F2A04D8FFF7F1B9222AEBD0FAE76D
:101BF000034A82630722C26303640120704700BF67
:101C00001822002007B5052917D8DFE801F01916BA
:101C100003191920302383F31188104A0190012100
:101C2000FFF794FA01980E4A0221FFF78FFA0D4848
:101C3000FFF7B6F9002383F3118803B05DF804FBC6
:101C4000302383F311880748FFF780F9F2E7302348
:101C500083F311880348FFF797F9EBE76435000831
:101C6000883500080826002038B50C4D0C4C0D496D
:101C70002A4604F10800FFF767FF05F1CA0204F1E4
:101C800010000949FFF760FF05F5CA7204F118005A
:101C90000649BDE83840FFF757BF00BFD02A0020F3
:101CA00020220020443500084E3500085935000830
:101CB00070B5044608460D46FEF7EAFFC6B2204658
:101CC000013403780BB9184670BD32462946FEF739
:101CD000CBFF0028F3D10120F6E700002DE9F04703
:101CE00005460C46FEF7D4FF2B49C6B22846FFF73F
:101CF000DFFF08B10A36F6B228492846FFF7D8FFB9
:101D000008B11036F6B2632E0BD8DFF88C80DFF8FE
:101D10008C90234FDFF894A02E7846B92670BDE84A
:101D2000F08729462046BDE8F04701F0B1BB252EDB
:101D30002ED1072241462846FEF796FF70B9194B6F
:101D4000224603F1100153F8040B42F8040B8B42B6
:101D5000F9D11B78137007351134DDE708224946A5
:101D60002846FEF781FF98B90F4BA21C1978090984
:101D70000232C95D02F8041C13F8011B01F00F01C7
:101D80005345C95D02F8031CF0D118340835C3E788
:101D900004F8016B0135BFE73036000859350008FB
:101DA0004A36000838360008107AFF1F1C7AFF1FD9
:101DB000BFF34F8F024AD368DB03FCD4704700BFE8
:101DC000003C024008B5094B1B7873B9FFF7F0FFE0
:101DD000074B1A69002ABFBF064A5A6002F18832CF
:101DE0005A601A6822F480621A6008BD2E2D002005
:101DF000003C02402301674508B50B4B1B7893B9A3
:101E0000FFF7D6FF094B1A6942F000421A611A68BF
:101E100042F480521A601A6822F480521A601A68DA
:101E200042F480621A6008BD2E2D0020003C024062
:101E30000B28F0B516D80C4C0C4923787BB90C4D07
:101E40000E460C234FF0006255F8047B46F8042B35
:101E5000013B13F0FF033A44F6D10123237051F8FC
:101E60002000F0BD0020FCE7602D0020302D002078
:101E70005C360008014B53F8200070475C360008C0
:101E80000C2070470B2810B5044601D9002010BD66
:101E9000FFF7CEFF064B53F824301844C21A0BB993
:101EA0000120F4E712680132F0D1043BF6E700BFED
:101EB0005C3600080B2838B5044628D8FFF75EFCCE
:101EC000FFF776FFFFF77EFF124AF323D360E300AC
:101ED000DBB243F4007343F002031361136943F46C
:101EE0008033136105462046FFF762FFFFF7A0FF2E
:101EF000094B53F8241000F0E9F82846FFF77CFF5F
:101F0000FFF746FC2046BDE83840FFF7BBBF002086
:101F100038BD00BF003C02405C36000812F00103EF
:101F20002DE9F04105460E4614464BD18218B2F118
:101F3000016F61D8314B1B6813F001035CD0304F47
:101F4000FFF71CFCFFF73EFFF323FB60FFF730FFBA
:101F5000314640F20128032C18D824F00104284E01
:101F60000C446D1A40F20118A142336905EB0107D8
:101F70002AD123F001033361FFF73EFFFFF708FC8E
:101F80000120BDE8F081043C0435E4E7AB07E4D16F
:101F90003B6923F440733B613B6943EA08033B61BF
:101FA00051F8046B2E60BFF34F8FFFF701FF2B68D2
:101FB0009E42E8D03B6923F001033B61FFF71CFF21
:101FC000FFF7E6FB0020DCE723F44073336133695D
:101FD00043EA080333610B883B80BFF34F8FFFF761
:101FE000E7FE3F8831F8023BBFB2BB42BCD0336949
:101FF00023F001033361E1E71846C2E700380240ED
:10200000003C0240084908B50B7828B11BB9FFF71E
:10201000D9FE01230B7008BD002BFCD0BDE80840A1
:102020000870FFF7E9BE00BF2E2D002010B5024456
:10203000064BD2B2904200D110BD441C00B253F8FE
:10204000200041F8040BE0B2F4E700BF5028004044
:102050000F4B30B51C6F240407D41C6F44F400747C
:102060001C671C6F44F400441C670A4C236843F44B
:10207000807323600244084BD2B2904200D130BD3D
:10208000441C00B251F8045B43F82050E0B2F4E77E
:1020900000380240007000405028004007B501227F
:1020A00001A90020FFF7C2FF019803B05DF804FB0F
:1020B00013B50446FFF7F2FFA04205D0012201A9A3
:1020C00000200194FFF7C4FF02B010BD704700006C
:1020D000034B1A681AB9034AD2F874281A60704779
:1020E000642D00200030024008B5FFF7F1FF024BDD
:1020F0001868C0F3407008BD642D002070470000D0
:10210000FEE700000A4B0B480B4A90420BD30B4BE7
:10211000DA1C121AC11E22F003028B4238BF0022C1
:102120000021FEF7BDBD53F8041B40F8041BECE78B
:1021300008380008602E0020602E0020602E00204D
:1021400070B5D0E915439E6800224FF0FF3504EBCF
:1021500042135101D3F800090028BEBFD3F800098B
:1021600040F08040C3F80009D3F8000B0028BEBF40
:10217000D3F8000B40F08040C3F8000B0132631825
:102180009642C3F80859C3F8085BE0D24FF0011338
:10219000C4F81C3870BD0000890141F020010161C4
:1021A00003699B06FCD41220FFF702BB10B5054C57
:1021B0002046FEF7ABFF4FF0A0436365024BA365DB
:1021C00010BD00BF682D0020B036000870B5037840
:1021D000012B054650D12A4B446D98421BD1294B07
:1021E0005A6B42F080025A635A6D42F080025A657F
:1021F0005A6D5A6942F080025A615A6922F080028F
:102200005A610E2143205B6900F022FC1E4BE36003
:102210001E4BC4F800380023C4F8003EC0232360DE
:102220006E6D4FF40413A3633369002BFCDA0123B2
:1022300033610C20FFF7BCFA3369DB07FCD41220B2
:10224000FFF7B6FA3369002BFCDA0026A6602846B1
:10225000FFF776FF6B68C4F81068DB68C4F8146891
:10226000C4F81C684BB90A4BA3614FF0FF3363619C
:10227000A36843F00103A36070BD064BF4E700BF01
:10228000682D002000380240401400400300200266
:10229000003C30C0083C30C0F8B5446D0546002114
:1022A0002046FFF779FFA96D00234FF001128F68D8
:1022B000C4F834384FF00066C4F81C284FF0FF30E3
:1022C00004EB431201339F42C2F80069C2F8006B6D
:1022D000C2F80809C2F8080BF2D20B686A6DEB6508
:1022E000636210231361166916F01006FBD11220E9
:1022F000FFF75EFAD4F8003823F4FE63C4F8003820
:10230000A36943F4402343F01003A3610923C4F8F5
:102310001038C4F814380A4BEB604FF0C043C4F8CF
:10232000103B084BC4F8003BC4F81069C4F80039EE
:10233000EB6D03F1100243F48013EA65A362F8BD6C
:102340008C36000840800010426D90F84E10D2F894
:10235000003823F4FE6343EA0113C2F800387047E3
:102360002DE9F84300EB8103456DDA68166806F045
:102370000306731E022B05EB41130C4680460FFA31
:1023800081F94FEA41104FF00001C3F8101B4FF0E4
:10239000010104F1100398BFB60401FA03F3916937
:1023A0008EBF334E06F1805606F5004600293AD01E
:1023B000578A04F15801490137436F50D5F81C186A
:1023C0000B43C5F81C382B180021C3F810195369AA
:1023D0000127611EA7409BB3138A928B9B08012A99
:1023E00088BF5343D8F85C20981842EA034301F1B0
:1023F000400205EB8202C8F85C0021465360284683
:10240000FFF7CAFE08EB8900C3681B8A43EA8453BE
:10241000483464011E432E51D5F81C381F43C5F8BB
:102420001C78BDE8F88305EB4917D7F8001B21F4A9
:102430000041C7F8001BD5F81C1821EA0303C0E7C8
:1024400004F13F0305EB83030A4A5A6028462146FC
:10245000FFF7A2FE05EB4910D0F8003923F4004342
:10246000C0F80039D5F81C3823EA0707D7E700BFC2
:102470000080001000040002826D1268C265FFF740
:102480005FBE00005831436D49015B5813F40040B2
:1024900004D013F4001F0CBF02200120704700007D
:1024A0004831436D49015B5813F4004004D013F4E4
:1024B000001F0CBF022001207047000000EB8101CB
:1024C000CB68196A0B6813604B6853607047000053
:1024D00000EB810330B5DD68AA691368D36019B9D0
:1024E000402B84BF402313606B8A1468426D1C44E8
:1024F000013CB4FBF3F46343033323F0030302EB27
:10250000411043EAC44343F0C043C0F8103B2B687A
:1025100003F00303012B09B20ED1D2F8083802EB05
:10252000411013F4807FD0F8003B14BF43F0805378
:1025300043F00053C0F8003B02EB4112D2F8003BDD
:1025400043F00443C2F8003B30BD00002DE9F041E8
:10255000244D6E6D06EB40130446D3F8087BC3F898
:10256000087B38070AD5D6F81438190706D505EBC5
:1025700084032146DB6828465B689847FA071FD525
:10258000D6F81438DB071BD505EB8403D968CCB922
:102590008B69488A5A68B2FBF0F600FB16228AB9AA
:1025A0001868DA6890420DD2121AC3E90024302369
:1025B00083F311880B482146FFF78AFF84F31188C3
:1025C000BDE8F081012303FA04F26B8923EA0203D8
:1025D0006B81CB68002BF3D021460248BDE8F04167
:1025E000184700BF682D002000EB810370B5DD683F
:1025F000436D6C692668E6604A0156BB1A444FF485
:102600000020C2F810092A6802F00302012A0AB267
:102610000ED1D3F8080803EB421410F4807FD4F8ED
:10262000000914BF40F0805040F00050C4F8000989
:1026300003EB4212D2F8000940F00440C2F800094E
:10264000D3F83408012202FA01F10143C3F8341827
:1026500070BD19B9402E84BF4020206020682E8AAA
:102660008419013CB4FBF6F440EAC44040F0005049
:102670001A44C6E72DE9F8433B4D6E6D06EB401357
:102680000446D3F80889C3F8088918F0010F4FEA07
:1026900040171AD0D6F81038DB0716D505EB8003A3
:1026A000D9684B691868DA68904230D2121A4FF034
:1026B00000091A60C3F80490302383F3118821467F
:1026C0002846FFF791FF89F3118818F0800F1CD07E
:1026D000D6F834380126A640334216D005EB8403E1
:1026E0006D6DD3F80CC0DCF814200134E4B2D2F8DC
:1026F00000E005EB04342F445168714515D3D5F83B
:10270000343823EA0606C5F83468BDE8F8830123A7
:1027100003FA04F22B8923EA02032B818B68002B36
:10272000D3D0214628469847CFE7BCF81000AEEB3F
:102730000103834228BF0346D7F8180980B2B3EBE0
:10274000800FE2D89068A0F1040959F8048FC4F80A
:102750000080A0EB09089844B8F1040FF5D818449C
:102760000B4490605360C7E7682D00202DE9F74FB8
:10277000A24C656D6E69AB691E4016F480586E619F
:1027800007D02046FEF72AFD03B0BDE8F04F00F069
:1027900047BC002E12DAD5F8003E98489B071EBFB2
:1027A000D5F8003E23F00303C5F8003ED5F8043801
:1027B00023F00103C5F80438FEF73AFD370505D5C7
:1027C0008E48FFF7BDFC8D48FEF720FDB0040CD508
:1027D000D5F8083813F0060FEB6823F470530CBFDC
:1027E00043F4105343F4A053EB6031071BD56368E7
:1027F000DB681BB9AB6923F00803AB612378052BB9
:102800000CD1D5F8003E7D489A071EBFD5F8003E92
:1028100023F00303C5F8003EFEF70AFD6368DB689A
:102820000BB176489847F30274D4B70227D5D4F891
:102830005490DFF8C8B100274FF0010A09EB4712A6
:10284000D2F8003B03F44023B3F5802F11D1D2F826
:10285000003B002B0DDA62890AFA07F322EA030330
:10286000638104EB8703DB68DB6813B139465846A4
:102870009847A36D01379B68FFB29F42DED9F006EF
:1028800017D5676D3A6AC2F30A1002F00F0302F41B
:10289000F012B2F5802F00F08580B2F5402F08D1FC
:1028A00004EB83030022DB681B6A07F58057904224
:1028B0006AD13003D5F8184813D5E10302D50020BA
:1028C000FFF744FEA20302D50120FFF73FFE63039A
:1028D00002D50220FFF73AFE270302D50320FFF7B7
:1028E00035FE75037FF550AFE00702D50020FFF7F6
:1028F000C1FEA10702D50120FFF7BCFE620702D589
:102900000220FFF7B7FE23077FF53EAF0320FFF756
:10291000B1FE39E7636DDFF8E4A0019300274FF0C3
:102920000109A36D9B685FFA87FB9B453FF67DAF6E
:10293000019B03EB4B13D3F8001901F44021B1F5CF
:10294000802F1FD1D3F8001900291BDAD3F8001902
:1029500041F09041C3F80019D3F800190029FBDBBE
:102960005946606DFFF718FC218909FA0BF321EA3B
:102970000303238104EB8B03DB689B6813B1594687
:10298000504698470137CCE7910708BFD7F8008039
:10299000072A98BF03F8018B02F1010298BF4FEAA2
:1029A000182884E7023304EB830207F58057526846
:1029B000D2F818C0DCF80820DCE9001CA1EB0C0CF4
:1029C000002188420AD104EB830463689B699A68FA
:1029D00002449A605A6802445A606AE711F0030F91
:1029E00008BFD7F800808C4588BF02F8018B01F141
:1029F000010188BF4FEA1828E3E700BF682D0020D7
:102A0000436D03EB4111D1F8003B43F40013C1F8CF
:102A1000003B7047436D03EB4111D1F8003943F49B
:102A20000013C1F800397047436D03EB4111D1F831
:102A3000003B23F40013C1F8003B7047436D03EBE8
:102A40004111D1F8003923F40013C1F8003970475F
:102A500000F1604303F561430901C9B283F8001333
:102A6000012200F01F039A4043099B0003F16043D9
:102A700003F56143C3F880211A60704730B5039CA9
:102A80000172043304FB0325C0E90653049B03636E
:102A90000021059BC160C0E90000C0E90422C0E933
:102AA0000842C0E90A11436330BD0000416A0022B8
:102AB000C0E90411C0E90A22C2606FF00101FEF70B
:102AC000E7BE0000D0E90432934201D1C2680AB9DE
:102AD000181D70470020704703691960C2680132F1
:102AE000C260C269134482690361934224BF436A8E
:102AF00003610021FEF7C0BE38B504460D46E36809
:102B00003BB16269131D1268A3621344E3620020A3
:102B100007E0237A33B929462046FEF79DFE0028B8
:102B2000EDDA38BD6FF00100FBE70000C368C26951
:102B3000013BC3604369134482694361934224BFEC
:102B4000436A436100238362036B03B118477047F4
:102B500070B53023044683F31188866A3EB9FFF7C7
:102B6000CBFF054618B186F31188284670BDA36ACD
:102B7000E26A13F8015BA362934202D32046FFF797
:102B8000D5FF002383F31188EFE700002DE9F84F0C
:102B900004460E46174698464FF0300989F31188CF
:102BA0000025AA46D4F828B0BBF1000F09D1414650
:102BB0002046FFF7A1FF20B18BF311882846BDE81E
:102BC000F88FD4E90A12A7EB050B521A934528BFD8
:102BD0009346BBF1400F1BD9334601F1400251F837
:102BE000040B43F8040B9142F9D1A36A40334036F9
:102BF000A3624035D4E90A239A4202D32046FFF764
:102C000095FF8AF31188BD42D8D289F31188C9E7AC
:102C100030465A46FEF71EF8A36A5B445E44A36240
:102C20005D44E7E710B5029C0172043303FB042105
:102C3000C0E906130023C0E90A33039B0363049B26
:102C4000C460C0E90000C0E90422C0E9084243634F
:102C500010BD0000026AC260426AC0E9042200227C
:102C6000C0E90A226FF00101FEF712BED0E9042389
:102C70009A4201D1C26822B9184650F8043B0B6051
:102C8000704700231846FAE7C368C2690133C3607E
:102C90004369134482694361934224BF436A436199
:102CA0000021FEF7E9BD000038B504460D46E36893
:102CB0003BB123691A1DA262E2691344E36200205A
:102CC00007E0237A33B929462046FEF7C5FD0028E0
:102CD000EDDA38BD6FF00100FBE700000369196011
:102CE000C268013AC260C2691344826903619342B7
:102CF00024BF436A036100238362036B03B1184757
:102D00007047000070B530230D460446114683F32A
:102D10001188866A2EB9FFF7C7FF10B186F31188B4
:102D200070BDA36A1D70A36AE26A01339342A36275
:102D300004D3E16920460439FFF7D0FF002080F377
:102D40001188EDE72DE9F84F04460D469046994667
:102D50004FF0300A8AF311880026B346A76A4FB9AC
:102D600049462046FFF7A0FF20B187F3118830467F
:102D7000BDE8F88FD4E90A073A1AA8EB060797428C
:102D800028BF1746402F1BD905F1400355F8042BE7
:102D900040F8042B9D42F9D1A36A4033A362403628
:102DA000D4E90A239A4204D3E16920460439FFF7A3
:102DB00095FF8BF311884645D9D28AF31188CDE768
:102DC00029463A46FDF746FFA36A3B443D44A362C9
:102DD0003E44E5E7D0E904239A4217D1C3689BB18A
:102DE000836A8BB1043B9B1A0ED01360C368013B0E
:102DF000C360C3691A44836902619A4224BF436A6B
:102E00000361002383620123184670470023FBE718
:102E100000F030B94FF08043586A70474FF080435C
:102E2000002258631A610222DA6070474FF0804333
:102E30000022DA60704700004FF08043586370470B
:102E4000FEE7000070B51B4B01630025044686B009
:102E5000586085620E4600F0BFF804F11003C4E923
:102E600004334FF0FF33C4E90635C4E90044A560DC
:102E7000E562FFF7CFFF2B460246C4E9082304F1C1
:102E800034010D4A256580232046FEF79BFC012373
:102E9000E0600A4A0375009272680192B268CDE957
:102EA0000223074B6846CDE90435FEF7B3FC06B0B4
:102EB00070BD00BF00260020BC360008C1360008E7
:102EC000412E0008024AD36A1843D062704700BFFF
:102ED000982300204B6843608B688360CB68C36095
:102EE0000B6943614B6903628B6943620B68036042
:102EF0007047000008B5264B26481A6940F2FF11BA
:102F00000A431A611A6922F4FF7222F001021A615F
:102F10001A691A6B0A431A631A6D0A431A651E4A24
:102F20001B6D1146FFF7D6FF02F11C0100F5806012
:102F3000FFF7D0FF02F1380100F58060FFF7CAFF0C
:102F400002F1540100F58060FFF7C4FF02F1700147
:102F500000F58060FFF7BEFF02F18C0100F5806094
:102F6000FFF7B8FF02F1A80100F58060FFF7B2FF9C
:102F700002F1C40100F58060FFF7ACFF02F1E0014F
:102F800000F58060FFF7A6FFBDE8084000F0EEB84E
:102F90000038024000000240C836000808B500F0C2
:102FA00059FAFEF7D3FBFFF793F8BDE80840FEF7A8
:102FB0005BBE000070470000EFF3098305494A6BD0
:102FC00022F001024A63683383F30988002383F304
:102FD0001188704700EF00E0302080F3118862B65E
:102FE0000C4B0D4AD96821F4E0610904090C0A432D
:102FF000DA60D3F8FC20094942F08072C3F8FC2063
:103000000A6842F001020A602022DA7783F822007F
:10301000704700BF00ED00E00003FA05001000E07B
:1030200010B5302383F311880E4B5B6813F40063F3
:1030300014D0F1EE103AEFF30984683C4FF080733E
:10304000E361094BDB6B236684F30988FEF752FBCF
:1030500010B1064BA36110BD054BFBE783F311884C
:10306000F9E700BF00ED00E000EF00E02F030008EB
:10307000320300080F4B1A6C42F001021A641A6EF8
:1030800042F001021A660C4A1B6E936843F001037A
:1030900093604FF0804353229A624FF0FF32DA621E
:1030A00000229A615A63DA605A6001225A611A60FA
:1030B000704700BF00380240002004E04FF080421B
:1030C00008B51169D3680B40D9B2C9439B07116198
:1030D00007D5302383F31188FEF74EFB002383F3DB
:1030E000118808BD1F4B1A696FEAC2526FEAD252AB
:1030F0001A611A69C2F308021A614FF0FF301A69A7
:103100005A69586100215A6959615A691A6A62F00C
:1031100080521A621A6A02F080521A621A6A5A6A55
:1031200058625A6A59625A6A1A6C42F080521A649A
:103130001A6E42F080521A661A6E0B4A106840F4FA
:1031400080701060186F00F44070B0F5007F1EBFF3
:103150004FF4803018671967536823F40073536085
:1031600000F054B90038024000700040334B4FF07B
:1031700080521A64324A4FF4404111601A6842F09A
:1031800001021A601A689107FCD59A6822F00302BE
:103190009A602A4B9A6812F00C02FBD1196801F070
:1031A000F90119609A601A6842F480321A601A684C
:1031B0009203FCD55A6F42F001025A671F4B5A6FB7
:1031C0009007FCD51F4A5A601A6842F080721A6054
:1031D0001B4A53685904FCD5184B1A689201FCD558
:1031E000194A9A60194B1A68194B9A42194B21D106
:1031F000194A1168194A91421CD140F205121A600D
:10320000144A136803F00F03052BFAD10B4B9A688D
:1032100042F002029A609A6802F00C02082AFAD17F
:103220005A6C42F480425A645A6E42F480425A66A2
:103230005B6E704740F20572E1E700BF0038024064
:10324000007000400854400700948838002004E0D3
:1032500011640020003C024000ED00E041C20F413B
:10326000074A08B5536903F00103536123B1054AC6
:1032700013680BB150689847BDE80840FFF7D0BE0F
:10328000003C0140E02D0020074A08B5536903F0D7
:103290000203536123B1054A93680BB1D068984784
:1032A000BDE80840FFF7BCBE003C0140E02D002017
:1032B000074A08B5536903F00403536123B1054A73
:1032C00013690BB150699847BDE80840FFF7A8BEE5
:1032D000003C0140E02D0020074A08B5536903F087
:1032E0000803536123B1054A93690BB1D06998472C
:1032F000BDE80840FFF794BE003C0140E02D0020EF
:10330000074A08B5536903F01003536123B1054A16
:10331000136A0BB1506A9847BDE80840FFF780BEBA
:10332000003C0140E02D0020164B10B55C6904F410
:1033300078725A61A30604D5134A936A0BB1D06A16
:103340009847600604D5104A136B0BB1506B984731
:10335000210604D50C4A936B0BB1D06B9847E2055C
:1033600004D5094A136C0BB1506C9847A30504D5DA
:10337000054A936C0BB1D06C9847BDE81040FFF73D
:103380004FBE00BF003C0140E02D0020194B10B59E
:103390005C6904F47C425A61620504D5164A136DD7
:1033A0000BB1506D9847230504D5134A936D0BB1AB
:1033B000D06D9847E00404D50F4A136E0BB1506EE0
:1033C0009847A10404D50C4A936E0BB1D06E984770
:1033D000620404D5084A136F0BB1506F9847230459
:1033E00004D5054A936F0BB1D06F9847BDE81040E4
:1033F000FFF716BE003C0140E02D002008B5FFF7A6
:103400005DFEBDE80840FFF70BBE0000062108B5D1
:103410000846FFF71DFB06210720FFF719FB0621D1
:103420000820FFF715FB06210920FFF711FB0621F5
:103430000A20FFF70DFB06211720FFF709FB0621E5
:103440002820FFF705FBBDE8084007211C20FFF7F7
:10345000FFBA000008B5FFF745FE00F00BF8FDF7D6
:1034600053FEFDF72BFDFFF7A5FDBDE80840FFF774
:10347000CFBC00000023054A19460133102BC2E9D6
:10348000001102F10802F8D1704700BFE02D0020C2
:10349000034611F8012B03F8012B002AF9D17047DC
:1034A00053544D3332463F3F3F0053544D33324621
:1034B0003430780053544D3332463432780053540C
:1034C0004D33324634343658580000000120330062
:1034D0000010410001105A0003105900071031007C
:1034E00000000000A034000813040000AA34000803
:1034F00019040000B434000821040000BE340008A0
:1035000000000000390E0008250E0008610E0008BA
:103510004D0E0008590E0008450E0008310E000837
:103520001D0E00086D0E00080000000001000000E4
:10353000000000006330000034350008F023002054
:10354000002600204172647550696C6F740025423A
:103550004F415244252D424C002553455249414C80
:1035600025000000020000000000000055100008C7
:10357000C110000840004000A02A0020B02A00200E
:103580000200000000000000030000000000000036
:10359000051100080000000010000000C02A0020F3
:1035A000000000000100000000000000682D002065
:1035B00001010200051C0008151B0008B11B0008D2
:1035C000951B000843000000CC35000809024300A9
:1035D000020100C0320904000001020201000524BA
:1035E0000010010524010001042402020524060044
:1035F00001070582030800FF09040100020A000018
:10360000000705010240000007058102400000009C
:1036100012000000183600081201100102000040DC
:1036200009124157000201020301000004030904CA
:1036300025424F41524425005370656564794265C7
:1036400065463430354D696E69003031323334357A
:1036500036373839414243444546000000400000B7
:103660000040000000400000004000000000010099
:103670000000020000000200000002000000020042
:103680000000020000000200000002000000000034
:103690004912000801150008AD150008400040005F
:1036A000C82D0020C82D002001000000D82D0020CA
:1036B0008000000040010000030000006D61696EA1
:1036C0000069646C650000000001812A00000000B0
:1036D000AAAAAAAA00010024FFFE00000000000020
:1036E00000A00A000000000100000000AAAAAAAA87
:1036F00000000001FFFF00000000000000000000CB
:103700000000001000000000AAAAAAAA00000010F1
:10371000FFFF0000000000000000000000000000AB
:1037200000000000AAAAAAAA00000000FFFF0000F3
:103730000000000000000000000000000000000089
:10374000AAAAAAAA00000000FFFF000000000000D3
:10375000000000000000000000000000AAAAAAAAC1
:1037600000000000FFFF000000000000000000005B
:103770000000000000000000AAAAAAAA00000000A1
:10378000FFFF00000000000000000000000000003B
:10379000000000000A00000000000000030000001C
:1037A0000000000000000000000000000000000019
:1037B0000000000000000000000000000000000009
:1037C00000000000000000006F0400000000000086
:1037D00000400F0000000000FF00960000000008FD
:1037E0000096000000000800040000002C360008CD
:1037F00000000000000000000000000000000000C9
:103800000000000000000000FFFFFFFFFFFFFFFFC0
:10381000FFFFFFFFFFFFFFFFFFFFFFFFFFFFFFFFB8
:10382000FFFFFFFFFFFFFFFFFFFFFFFFFFFFFFFFA8
:10383000FFFFFFFFFFFFFFFFFFFFFFFFFFFFFFFF98
:10384000FFFFFFFFFFFFFFFFFFFFFFFFFFFFFFFF88
:10C000000006002089D20008B5440608114406083D
:10C010007D44060811440608494406088BD20008EE
:10C020008BD200088BD200088BD200089523080819
:10C030008BD200088BD200088BD200088BD200086C
:10C040008BD200088BD200088BD200088BD200085C
:10C050008BD200088BD20008A1350808C935080822
:10C06000F13508081936080841360808A9E207081A
:10C07000D1E20708FDE2070829E3070855E30708AE
:10C080007DE30708A9E307082DE207088BD2000823
:10C090008BD200088BD200088BD2000869360808C2
:10C0A000B5370808B9370808CD370808D137080868
:10C0B000D5370808E5370808F937080835E90708CB
:10C0C000DDEA07088BD200088BD200088BD200086B
:10C0D0008BD200083D370808513708086537080833
:10C0E000CD3608088BD200088BD200088BD200080E
:10C0F0008BD200088BD200088BD20008D5E307084A
:10C100008BD200088BD200088BD200088BD200089B
:10C11000793708088D3708088BD200088BD20008C1
:10C1200001E4070829E4070855E4070881E4070843
:10C13000ADE407088BD200088BD200088BD2000830
:10C140008BD200088BD200088BD20008C12A0808C5
:10C15000D5E4070801E507082DE50708A137080819
:10C160008BD200088BD200088BD200088BD200083B
:10C170008BD200088BD200088BD200088BD200082B
:10C180008BD200088BD200088BD200088BD200081B
:10C190008BD200088BD200088BD200088BD200080B
:10C1A0008BD200088BD200088BD200088BD20008FB
:10C1B0008BD200088BD200088BD200088BD20008EB
:10C1C0008BD200088BD200088BD200088BD20008DB
:10C1D0008BD200088BD200088BD200088BD20008CB
:10C1E00021E700080DF70008BD5B010885AD0208D6
:10C1F000392B0408A54504083D9104080199040859
:10C20000399C0408CDFB0408491705086589050811
:10C210006D3D0608F9CE0608610007084555070878
:10C220001D7C0708D191070875BF07083DC50708A1
:10C2300081F0004102E000BF83F0004330B54FEAD7
:10C2400041044FEA430594EA050F08BF90EA020F44
:10C250001FBF54EA000C55EA020C7FEA645C7FEAD7
:10C26000655C00F0E2804FEA5454D4EB5555B8BFFA
:10C270006D420CDD2C4480EA020281EA030382EA6B
:10C28000000083EA010180EA020281EA0303362DFD
:10C2900088BF30BD11F0004F4FEA01314FF4801CD0
:10C2A0004CEA113102D0404261EB410113F0004FE2
:10C2B0004FEA03334CEA133302D0524263EB430399
:10C2C00094EA050F00F0A780A4F10104D5F1200E37
:10C2D0000DDB02FA0EFC22FA05F2801841F1000192
:10C2E00003FA0EF2801843FA05F359410EE0A5F166
:10C2F00020050EF1200E012A03FA0EFC28BF4CF097
:10C30000020C43FA05F3C01851EBE37101F000454C
:10C3100007D54FF0000EDCF1000C7EEB00006EEB59
:10C320000101B1F5801F1BD3B1F5001F0CD34908E3
:10C330005FEA30004FEA3C0C04F101044FEA44523A
:10C3400012F5800F80F09A80BCF1004F08BF5FEAC1
:10C35000500C50F1000041EB045141EA050130BDA1
:10C360005FEA4C0C404141EB0101013C28BFB1F5B3
:10C37000801FE9D291F0000F04BF01460020B1FAFE
:10C3800081F308BF2033A3F10B03B3F120020CDAD1
:10C390000C3208DD02F1140CC2F10C0201FA0CF0AF
:10C3A00021FA02F10CE002F11402D8BFC2F1200C14
:10C3B00001FA02F120FA0CFCDCBF41EA0C019040CA
:10C3C000E41AA2BF01EB0451294330BD6FEA040413
:10C3D0001F3C1CDA0C340EDC04F11404C4F12002FE
:10C3E00020FA04F001FA02F340EA030021FA04F310
:10C3F00045EA030130BDC4F10C04C4F1200220FA67
:10C4000002F001FA04F340EA0300294630BD21FAA4
:10C4100004F0294630BD94F0000F83F4801306BF6A
:10C4200081F480110134013D4EE77FEA645C18BF5E
:10C430007FEA655C29D094EA050F08BF90EA020FF5
:10C4400005D054EA000C04BF1946104630BD91EAED
:10C45000030F1EBF0021002030BD5FEA545C05D1F0
:10C460004000494128BF41F0004130BD14F580042F
:10C470003CBF01F5801130BD01F0004545F0FE41A3
:10C4800041F470014FF0000030BD7FEA645C1ABFD8
:10C49000194610467FEA655C1CBF0B46024650EA0F
:10C4A000013406BF52EA033591EA030F41F400213B
:10C4B00030BD00BF90F0000F04BF0021704730B5C1
:10C4C0004FF4806404F132044FF000054FF0000196
:10C4D00050E700BF90F0000F04BF0021704730B557
:10C4E0004FF4806404F1320410F0004548BF40422C
:10C4F0004FF000013EE700BF42004FEAE2014FEA81
:10C5000031014FEA02701FBF12F07F4393F07F4F5B
:10C5100081F06051704732F07F4208BF704793F05E
:10C520007F4F04BF41F40021704730B54FF4607471
:10C5300001F0004521F000411CE700BF50EA010274
:10C5400008BF704730B54FF000050AE050EA01021D
:10C5500008BF704730B511F0004502D5404261EB8D
:10C5600041014FF4806404F132045FEA915C3FF4CE
:10C57000D8AE4FF003025FEADC0C18BF03325FEA6B
:10C58000DC0C18BF033202EBDC02C2F1200300FA1C
:10C5900003FC20FA02F001FA03FE40EA0E0021FA41
:10C5A00002F11444BDE600BF70B54FF0FF0C4CF42F
:10C5B000E06C1CEA11541DBF1CEA135594EA0C0FE1
:10C5C00095EA0C0F00F0DEF82C4481EA030621EA1C
:10C5D0004C5123EA4C5350EA013518BF52EA033557
:10C5E00041F4801143F4801338D0A0FB02CE4FF009
:10C5F0000005E1FB02E506F00042E0FB03E54FF039
:10C600000006E1FB03569CF0000F18BF4EF0010E30
:10C61000A4F1FF04B6F5007F64F5407404D25FEA2C
:10C620004E0E6D4146EB060642EAC62141EA5551DF
:10C630004FEAC52040EA5E504FEACE2EB4F1FD0C21
:10C6400088BFBCF5E06F1ED8BEF1004F08BF5FEA9F
:10C65000500E50F1000041EB045170BD06F0004651
:10C6600046EA010140EA020081EA0301B4EB5C04FE
:10C67000C2BFD4EB0C0541EA045170BD41F48011F6
:10C680004FF0000E013C00F3AB8014F1360FDEBF1B
:10C69000002001F0004170BDC4F10004203C35DAF7
:10C6A0000C341BDC04F11404C4F1200500FA05F37A
:10C6B00020FA04F001FA05F240EA020001F000421B
:10C6C00021F0004110EBD37021FA04F642EB060191
:10C6D0005EEA430E08BF20EAD37070BDC4F10C04BB
:10C6E000C4F1200500FA04F320FA05F001FA04F27F
:10C6F00040EA020001F0004110EBD37041F100016B
:10C700005EEA430E08BF20EAD37070BDC4F1200575
:10C7100000FA05F24EEA020E20FA04F301FA05F2DD
:10C7200043EA020321FA04F001F0004121FA04F285
:10C7300020EA020000EBD3705EEA430E08BF20EA55
:10C74000D37070BD94F0000F0FD101F0004640008F
:10C7500041EB010111F4801F08BF013CF7D041EA11
:10C76000060195F0000F18BF704703F00046520015
:10C7700043EB030313F4801F08BF013DF7D043EAE6
:10C780000603704794EA0C0F0CEA135518BF95EA9C
:10C790000C0F0CD050EA410618BF52EA4306D1D123
:10C7A00081EA030101F000414FF0000070BD50EA42
:10C7B000410606BF1046194652EA430619D094EACC
:10C7C0000C0F02D150EA013613D195EA0C0F05D1B6
:10C7D00052EA03361CBF104619460AD181EA03010A
:10C7E00001F0004141F0FE4141F470014FF00000C2
:10C7F00070BD41F0FE4141F4780170BD70B54FF05D
:10C80000FF0C4CF4E06C1CEA11541DBF1CEA1355DC
:10C8100094EA0C0F95EA0C0F00F0A7F8A4EB0504BE
:10C8200081EA030E52EA03354FEA013100F08880B5
:10C830004FEA03334FF0805545EA131343EA12637E
:10C840004FEA022245EA111545EA10654FEA002633
:10C850000EF000419D4208BF964244F1FD0404F5EC
:10C86000407402D25B084FEA3202B61A65EB030548
:10C870005B084FEA32024FF480104FF4002CB6EB05
:10C88000020E75EB030E22BFB61A754640EA0C0085
:10C890005B084FEA3202B6EB020E75EB030E22BFC5
:10C8A000B61A754640EA5C005B084FEA3202B6EB06
:10C8B000020E75EB030E22BFB61A754640EA9C00C5
:10C8C0005B084FEA3202B6EB020E75EB030E22BF95
:10C8D000B61A754640EADC0055EA060E18D04FEA53
:10C8E000051545EA16754FEA06164FEAC30343EAF3
:10C8F00052734FEAC2025FEA1C1CC0D111F4801FC0
:10C900000BD141EA00014FF000004FF0004CB6E7B8
:10C9100011F4801F04BF01430020B4F1FD0C88BF57
:10C92000BCF5E06F3FF6AFAEB5EB030C04BFB6EB62
:10C93000020C5FEA500C50F1000041EB045170BD55
:10C940000EF0004E4EEA113114EB5C04C2BFD4EB82
:10C950000C0541EA045170BD41F480114FF0000E06
:10C96000013C90E645EA060E8DE60CEA135594EA82
:10C970000C0F08BF95EA0C0F3FF43BAF94EA0C0F85
:10C980000AD150EA01347FF434AF95EA0C0F7FF4FA
:10C9900025AF104619462CE795EA0C0F06D152EA4E
:10C9A00003353FF4FDAE1046194622E750EA410632
:10C9B00018BF52EA43067FF4C5AE50EA41047FF443
:10C9C0000DAF52EA43057FF4EBAE12E74FF0FF3CA8
:10C9D00006E000BF4FF0010C02E000BF4FF0010C79
:10C9E0004DF804CD4FEA410C7FEA6C5C4FEA430CF2
:10C9F00018BF7FEA6C5C1BD001B050EA410C0CBF41
:10CA000052EA430C91EA030F02BF90EA020F0020A2
:10CA1000704710F1000F91EA030F58BF994208BF09
:10CA200090422CBFD8176FEAE37040F001007047C6
:10CA30004FEA410C7FEA6C5C02D150EA013C07D11D
:10CA40004FEA430C7FEA6C5CD6D152EA033CD3D068
:10CA50005DF8040B704700BF8446104662468C4662
:10CA60001946634600E000BF01B5FFF7B7FF002895
:10CA700048BF10F1000F01BD4DF808EDFFF7F4FFBE
:10CA80000CBF012000205DF808FB00BF4DF808ED49
:10CA9000FFF7EAFF34BF012000205DF808FB00BF6C
:10CAA0004DF808EDFFF7E0FF94BF012000205DF88E
:10CAB00008FB00BF4DF808EDFFF7CEFF94BF012043
:10CAC00000205DF808FB00BF4DF808EDFFF7C4FF3C
:10CAD00034BF012000205DF808FB00BF4FEA410C85
:10CAE0007FEA6C5C02D150EA013C0AD14FEA430C68
:10CAF0007FEA6C5C02D152EA033C02D14FF00000A5
:10CB000070474FF0010070474FEA410212F50012E2
:10CB100015D211D56FF47873B3EB625212D94FEA84
:10CB2000C12343F0004343EA505311F0004F23FA6E
:10CB300002F018BF404270474FF00000704750EAC3
:10CB4000013005D111F0004008BF6FF00040704780
:10CB50004FF00000704700BF4A0011D212F50012DA
:10CB600011D20DD56FF47873B3EB62520ED44FEA45
:10CB7000C12343F0004343EA505323FA02F07047C5
:10CB80004FF00000704750EA013002D14FF0FF3003
:10CB900070474FF0000070474FEA4102B2F1E043A6
:10CBA00024BFB3F5001CDCF1FE5C0DD901F0004C94
:10CBB0004FEAC0024CEA5070B2F1004F40EB8300E4
:10CBC00008BF20F00100704711F0804F21D113F110
:10CBD0003872BCBF01F00040704741F480114FEA49
:10CBE0005252C2F11802C2F1200C10FA0CF320FAD2
:10CBF00002F018BF40F001004FEAC1234FEAD323EF
:10CC000003FA0CFC40EA0C0023FA02F34FEA430358
:10CC1000CCE77FEA625307D150EA01331EBF4FF0E1
:10CC2000FE4040F44000704701F0004040F0FE40FC
:10CC300040F40000704700BF80F0004002E000BFF9
:10CC400081F0004142001FBF5FEA410392EA030FF7
:10CC50007FEA226C7FEA236C6AD04FEA1262D2EB41
:10CC60001363C1BFD218414048404140B8BF5B4246
:10CC7000192B88BF704710F0004F40F4000020F0DF
:10CC80007F4018BF404211F0004F41F4000121F0F5
:10CC90007F4118BF494292EA030F3FD0A2F101023F
:10CCA00041FA03FC10EB0C00C3F1200301FA03F17D
:10CCB00000F0004302D5494260EB4000B0F5000FA0
:10CCC00013D3B0F1807F06D340084FEA310102F15F
:10CCD0000102FE2A51D2B1F1004F40EBC25008BF11
:10CCE00020F0010040EA03007047490040EB0000DB
:10CCF000013A28BFB0F5000FEDD2B0FA80FCACF1DC
:10CD0000080CB2EB0C0200FA0CF0AABF00EBC25008
:10CD100052421843BCBFD0401843704792F0000FF6
:10CD200081F4000106BF80F400000132013BB5E749
:10CD30004FEA41037FEA226C18BF7FEA236C21D0BF
:10CD400092EA030F04D092F0000F08BF0846704724
:10CD500090EA010F1CBF0020704712F07F4F04D1F2
:10CD6000400028BF40F00040704712F100723CBF05
:10CD700000F50000704700F0004343F0FE4040F42F
:10CD8000000070477FEA226216BF08467FEA2363ED
:10CD90000146420206BF5FEA412390EA010F40F4D8
:10CDA000800070474FF0000304E000BF10F0004324
:10CDB00048BF40425FEA000C08BF704743F096430B
:10CDC00001464FF000001CE050EA010208BF704726
:10CDD0004FF000030AE000BF50EA010208BF7047AD
:10CDE00011F0004302D5404261EB41015FEA010CC2
:10CDF00002BF84460146002043F0B64308BFA3F1BA
:10CE00008053A3F50003BCFA8CF2083AA3EBC2539B
:10CE100010DB01FA02FC634400FA02FCC2F12002BA
:10CE2000BCF1004F20FA02F243EB020008BF20F0F1
:10CE30000100704702F1200201FA02FCC2F1200257
:10CE400050EA4C0021FA02F243EB020008BF20EA4C
:10CE5000DC7070477BB972B90029BEBF00204FF06B
:10CE6000004106E008BF00281CBF6FF000414FF0F2
:10CE7000FF3000F007BAADF1080C6DE904CE0029CF
:10CE800009DB002B1ADB00F095F8DDF804E0DDE9A2
:10CE9000022304B07047404261EB4101002B1BDBD1
:10CEA00000F088F8DDF804E0DDE9022304B0404238
:10CEB00061EB4101524263EB43037047524263EB23
:10CEC000430300F077F8DDF804E0DDE9022304B065
:10CED000404261EB41017047524263EB430300F073
:10CEE00069F8DDF804E0DDE9022304B0524263EBA7
:10CEF0004303704753B94AB9002908BF00281CBF33
:10CF00004FF0FF314FF0FF3000F0BCB9ADF1080C2D
:10CF10006DE904CE00F04EF8DDF804E0DDE902230F
:10CF200004B07047430803F05533C01A830803F078
:10CF3000333300F03330184400EB101000F00F30A2
:10CF400000EB002000EB0040000E704707EE900A57
:10CF5000F5EEC07AF1EE10FA01D400F00BB8F1EE64
:10CF6000677A08B517EE900A00F004F8404261EBCA
:10CF7000410108BDD0B5FFF7BFFA0C4B00220646B1
:10CF80000F46FFF711FBFFF7E7FD0446FFF792FAA4
:10CF9000074B0022FFF708FB02460B463046394696
:10CFA000FFF74AF9FFF7D8FD2146D0BD0000F03D5C
:10CFB0000000F0412DE9F047089D04468E46002B05
:10CFC0004DD18A42944669D9B2FA82F252B101FA3D
:10CFD00002F3C2F1200120FA01F10CFA02FC41EA4D
:10CFE000030E94404FEA1C48210CBEFBF8F61FFAD2
:10CFF0008CF708FB16E341EA034306FB07F199426D
:10D000000AD91CEB030306F1FF3080F01F8199421F
:10D0100040F21C81023E63445B1AA4B2B3FBF8F0F9
:10D0200008FB103344EA034400FB07F7A7420AD980
:10D030001CEB040400F1FF3380F00A81A74240F2A8
:10D0400007816444023840EA0640E41B00261DB113
:10D05000D4400023C5E900433146BDE8F0878B4248
:10D0600009D9002D00F0EF800026C5E90001304607
:10D070003146BDE8F087B3FA83F6002E4AD18B42E1
:10D0800002D3824200F2F980841A61EB030301208B
:10D090009E46002DE0D0C5E9004EDDE702B9FFDE77
:10D0A000B2FA82F2002A40F09280A1EB0C014FEA22
:10D0B0001C471FFA8CFE0126200CB1FBF7F307FB7F
:10D0C000131140EA01410EFB03F0884208D91CEB22
:10D0D000010103F1FF3802D2884200F2CB804346BF
:10D0E000091AA4B2B1FBF7F007FB101144EA01449E
:10D0F0000EFB00FEA64508D91CEB040400F1FF312D
:10D1000002D2A64500F2BB800846A4EB0E0440EA1A
:10D1100003409CE7C6F12007B34022FA07FC4CEA23
:10D12000030C20FA07F401FA06F31C43F9404FEA16
:10D130001C4900FA06F3B1FBF9F8200C1FFA8CFE2B
:10D1400009FB181140EA014108FB0EF0884202FA7F
:10D1500006F20BD91CEB010108F1FF3A80F0888040
:10D16000884240F28580A8F102086144091AA4B2FD
:10D17000B1FBF9F009FB101144EA014100FB0EFE7E
:10D180008E4508D91CEB010100F1FF346CD28E45AD
:10D190006AD90238614440EA0840A0FB0294A1EB3E
:10D1A0000E01A142C846A64656D353D05DB1B3EB9B
:10D1B000080261EB0E0101FA07F722FA06F3F140CB
:10D1C0001F43C5E9007100263146BDE8F087C2F172
:10D1D0002003D8400CFA02FC21FA03F391400143EA
:10D1E0004FEA1C471FFA8CFEB3FBF7F007FB103623
:10D1F0000B0C43EA064300FB0EF69E4204FA02F4CF
:10D2000008D91CEB030300F1FF382FD29E422DD921
:10D21000023863449B1B89B2B3FBF7F607FB163356
:10D2200041EA034106FB0EF38B4208D91CEB0101D6
:10D2300006F1FF3816D28B4214D9023E6144C91A56
:10D2400046EA004638E72E46284605E70646E3E666
:10D250001846F8E64B45A9D2B9EB020864EB0C0E70
:10D260000138A3E74646EAE7204694E74046D1E77F
:10D27000D0467BE7023B614432E7304609E764442D
:10D28000023842E7704700BF02E000F000F8FEE716
:10D2900072B6374880F30888364880F309883648E4
:10D2A0003649086040F20000CCF200004EF63471BE
:10D2B000CEF200010860BFF34F8FBFF36F8F40F2D3
:10D2C0000000C0F2F0004EF68851CEF20001086076
:10D2D000BFF34F8FBFF36F8F4FF00000E1EE100AE6
:10D2E0004EF63C71CEF200010860062080F31488EF
:10D2F000BFF36F8F75F0ACF875F0F0FF4FF055305D
:10D300001F491B4A91423CBF41F8040BFAE71D49F3
:10D31000184A91423CBF41F8040BFAE71A491B4AEC
:10D320001B4B9A423EBF51F8040B42F8040BF8E73E
:10D3300000201849184A91423CBF41F8040BFAE713
:10D3400075F08AF876F01EF8144C154DAC4203DAED
:10D3500054F8041B8847F9E701F0D2F9114C124D3B
:10D36000AC4203DA54F8041B8847F9E775F072B849
:10D37000000600200022002000C0000808ED00E0A8
:10D380000000002000060020D8420A0800220020E9
:10D39000C8250020C8250020C02A0120E0C10008BF
:10D3A00030C2000830C2000830C200082DE9F04F3A
:10D3B0002DED108AC1F80CD0C3689D46BDEC108AD3
:10D3C000BDE8F08F002383F311882846A047002092
:10D3D00074F032F8FEE773F09FFE00DFFEE7000016
:10D3E00001F0FF01102A2BDB10F0070F08D010F816
:10D3F000013B013A8B422DD010F0070F42B3F6D11A
:10D40000F0B441EA012141EA014122F007047FF032
:10D4100000070023F0E80256083C85EA010586EA89
:10D42000010685FA47F5A3FA87F586FA47F6A5FAC5
:10D4300087F68EB9EED1F0BC01F0FF0102F00702D1
:10D4400032B110F8013B013A83EA010313B1F8D17C
:10D450000020704701387047002D06BF354603385D
:10D46000073815F0010F07D1013015F4807F02BF96
:10D47000013015F4C03F0130F0BC0138704700BFE7
:10D4800010F8012B11F8013B012A28BF9A42F7D06E
:10D49000D01A7047034613F8012B002AFBD1181A43
:10D4A0000138704738B50022002304460D46FFF7C7
:10D4B000EDFA28B920462946BDE8384000F00AB800
:10D4C000204605F1004100F005F8404261EB4101C2
:10D4D00038BD00BFD0B50C4B002206460F46FFF703
:10D4E00063F8FFF739FB0446FEF7E4FF074B002221
:10D4F000FFF75AF802460B4630463946FEF79CFEC7
:10D50000FFF72AFB2146D0BD0000F03D0000F041AE
:10D51000002070477047000070470000704700000F
:10D52000002070470020704700207047012070479E
:10D5300000207047704700000020704700207047AF
:10D5400070470000704700000020704700207047BF
:10D5500070B5154ED6F8780203681B689847042802
:10D560001ADC01281DDC002814BF012441240F4BC4
:10D570001D68E86A0368DB69984701280AD0D6F875
:10D5800078220B4B9A4205D0EB6A93F89C300BB192
:10D5900044F08004204670BD0A2814BF01241924D9
:10D5A000E5E71924E3E700BFD0550020CC25002093
:10D5B00050580020044BD3F8780203F520729042B3
:10D5C00014BF042002207047D0550020014B93F86F
:10D5D00088017047D04500207047000038B5C578F5
:10D5E0000B461C2D044628BF1C251C220021184672
:10D5F00078F0A8FE2A4604F10C01BDE8384078F026
:10D6000057BE000038B5C5780B46102D044628BF1C
:10D61000102510220021184678F094FE2A4604F1C5
:10D620000C01BDE8384078F043BE000008B53EF07C
:10D63000C5F930B9034A92F80C3343F0040382F879
:10D640000C3308BDD055002038B591ED000AF7EE37
:10D65000000A0D4618F088FB20B10B4801F0DCFEF3
:10D66000002038BDD5ED007A9FED087AF0EEE77A1C
:10D67000F4EEC77AF1EE10FA03D5034801F0DEFEAE
:10D68000EEE70320EDE700BFD025002000000034C6
:10D6900010B5044608F0A0FA204610BD13B58B8BD8
:10D6A000B72B0C4607D0B3F5967F21D002B0BDE86A
:10D6B000104041F021BE124912481E2201F0E6FE40
:10D6C000D4ED017A94ED007A0D48FCEEE77ABCEED9
:10D6D000C77A17EE903A8DED017A9DF804109AB250
:10D6E00001F074FB002814BF0020042002B010BD1C
:10D6F00004480549022201F0C9FE0020F6E700BFF8
:10D7000078580020D02500204C58002000B51F4A32
:10D71000DFED1F6AD2EDC17A92EDC07AD2F8F41231
:10D72000007CA2F580538BB093F9AA310491002BB1
:10D7300018BFB0EE677AD2EDBB7A8DED057AFDEEBB
:10D74000E77A3E2117EE903AD2EDBC7AF4EEE67A13
:10D75000F1EE10FA58BFF0EE667AFCEEE77A1BB2F3
:10D76000ADF82030ADF8223017EE903A0022039247
:10D7700006920792ADF82430B7221A23CDE9003281
:10D7800003AA3BF09FFB0BB05DF804FBD0550020D3
:10D7900000FF7F4770B5154C94F812238AB022B968
:10D7A0000AB0BDE870403CF059BE057C56F0B6FEAC
:10D7B000D4E99C61D4F86C32A4F50054CDE905138A
:10D7C000B4F86824ADF826200023CDE90733ADF87E
:10D7D000243068221C23CDE90306CDE90032212143
:10D7E00003AA28463BF06EFB0AB070BDD05500205E
:10D7F000F0B53B4CB4F8CC31DE078DB0054637D5DB
:10D80000D4F88032089302238DF82430D4F8903273
:10D81000D4F88402CDF82530D4F88C32D4F87812BC
:10D82000D4F87C220590CDF8293062202123D4F849
:10D830007062D4F86C720691CDE90030C2211923D0
:10D84000287C079203AA049603973BF03BFB287CB5
:10D850003BF0CEFA0646287C3CF0CEF900F12103DD
:10D860009E4205D2287C0DB0BDE8F0403AF03CBDA8
:10D87000B4F8CC31990731D5D4F868330893032331
:10D880008DF82430D4F87833D4F86423CDF82530DB
:10D89000D4F87433D4F86C03D4F860130792CDF83D
:10D8A000293062222123D4F85863D4F854730590A8
:10D8B000CDE90032287C0691192303AAC2210397DF
:10D8C00004963BF0FFFA287C3BF092FA0446287C51
:10D8D0003CF092F900F121039C42C3D30DB0F0BD9E
:10D8E000D045002005207047024BD3F8780203682A
:10D8F0001B681847D055002030B5CD788BB0272D48
:10D9000028BF27250C4627220021684678F01AFDFB
:10D910002A4604F10C01684678F0CAFC1A4BD3F889
:10D92000781203F5227291422BD1DDED057A9FED3D
:10D93000177AF0EEE77AF4EEC77AF1EE10FA20D516
:10D940009DF8262002F0410141291AD1110618D470
:10D9500002F01801182914D00199C3F88C1282F032
:10D9600004020299C3F89012C2F380020399C3F82B
:10D97000941283F89C220499079AC3F89812C3F86A
:10D98000A0220BB030BD00BFD055002000000034F5
:10D9900030B5194D95F8113385B00C464BBBCA789C
:10D9A0008DF80C30092A28BF09220C3101A8CDE9D5
:10D9B000013378F07DFC9DF808305A1F012A18D9F0
:10D9C00003F0F703122B14D0A5F58053B3F98A2185
:10D9D00012B9E279A3F88A21227AE179074800F0A6
:10D9E000B1F9227AE179054800F0E4F9012385F8DC
:10D9F000113305B030BD00BFD0550020F0500020DD
:10DA0000F0B51B4BB3F98A3189B005460E46144672
:10DA10003BB1D779BB4204D009B0BDE8F0403FF03C
:10DA2000F5BFA27A637A43EA0223E27A43EA024329
:10DA30001D2B13D0212B08D01BB921462846FFF7F8
:10DA4000A7FF224631462846E6E701A92046FFF710
:10DA5000C5FD084801A901F09FFFF2E701A9204692
:10DA6000FFF7D0FD034801A901F0ECFFE9E700BF93
:10DA7000D0450020D025002013B5CA78072A4FF0E2
:10DA80000003044628BF07220C3168460093CDF8F6
:10DA9000033078F00DFCBDF900304BB901231C2197
:10DAA000204684F80F3302B0BDE8104041F0DCBBE3
:10DAB00002B010BD30B5CD7889B01E2D28BF1E250F
:10DAC0000C461E220021684678F03CFC2A4604F1F0
:10DAD0000C01684678F0ECFB0248694601F0FEFF55
:10DAE00009B030BDD025002000B589B0084601A995
:10DAF000FFF774FD034801A901F04EFF09B05DF87E
:10DB000004FB00BFD02500201FB508466946FFF77B
:10DB100079FD0348694601F095FF05B05DF804FB07
:10DB2000D02500202DE9F041CC7894B0262C28BFD8
:10DB3000262488462622002107460AA878F002FCFF
:10DB400002AD224608F10C010AA878F0B1FB284684
:10DB500007F09EFD9DF84A30022B06AC03D0032B44
:10DB600044D0002B66D1DFED357ADDED106A9FEDF4
:10DB7000346A9DED0F7A66EEA76ADDED0E7A27EE28
:10DB8000067A67EE867A0023FDEEE66ABDEEC77A76
:10DB9000FDEEE77A17EE102A17EE901A0093204652
:10DBA00016EE903A07F094FD94E80F0085E80F0018
:10DBB00097F80F3363BB012698F8083098F80720D0
:10DBC0008DF8193000238DF818208DF81B3099221C
:10DBD0000423CDE90032387C8DF81A6003232246F5
:10DBE0002F213BF06FF914B0BDE8F081DFED137A1F
:10DBF000DDED106A9FED126A9DED0F7A66EEA76A61
:10DC0000DDED0E7A27EE067A67EE867A0123BBE712
:10DC1000BDF8446086B90B483246294601F0D4FB72
:10DC20000028C8D0084A062138463DF05BFB87F83B
:10DC30000F63C1E70226BFE70026BDE70000C84228
:10DC40008096184BD0250020B4A5080838B58A7AEC
:10DC50004B7A43EA0223CA7A43EA0243272B05465A
:10DC60000C460CD81C2B10D91D3B0A2B0DD8DFE815
:10DC700003F01E0C0C0C1B0C0C0C0C121500452B8D
:10DC80000FD0522B01D1FFF737FE21462846BDE8C1
:10DC9000384040F0C9B9FFF7EFFEF6E7FFF742FF63
:10DCA000F3E7FFF707FFF0E7FFF71EFFEDE7FFF7EA
:10DCB0002BFFEAE700207047C8207047012070471B
:10DCC00000207047002070470120704790F8903086
:10DCD0008B4286BF00EB8100D0F894000020704793
:10DCE00090F890308B4286BF00EB8100D0F8940012
:10DCF00000207047014B93F886017047D045002003
:10DD0000036A43F4E0530362436A43F4E05343621B
:10DD1000836A43F4E05383627047000013B54FF405
:10DD20004470CDE9002107F04FFF044628B1DDE93A
:10DD3000002140F0DDFE024B2360204602B010BD02
:10DD400050A708082DE9F04FDFF8649085B006462B
:10DD50000F46904600254FF4837A96F89030ECB247
:10DD6000A34222D920463BF043F8834620463BF0AD
:10DD700043FF031D9B4514D399F9AB31ADF808302F
:10DD800094220623CDE90032422102AA20468DF8D2
:10DD90000A708DF80B80ADF80CA03BF093F80135BC
:10DDA000DBE720463AF0A0FAF9E705B0BDE8F08FCE
:10DDB000D04500202DE9F04FDFF8649085B006468D
:10DDC0000F469046002540F2011A96F89030ECB2CA
:10DDD000A34222D920463BF00BF8834620463BF075
:10DDE0000BFF031D9B4514D399F9AB31ADF80830F7
:10DDF00094220623CDE90032422102AA20468DF862
:10DE00000A708DF80B80ADF80CA03BF05BF8013583
:10DE1000DBE720463AF068FAF9E705B0BDE8F08F95
:10DE2000D04500201FB500F54053002100F5935068
:10DE3000D3F8F4220191D3F8EC32029201A9083010
:10DE4000039301F0ABFF03F077FB03F041F905B05A
:10DE50005DF804FB70B586B006461322002101A8C8
:10DE600010EE105A10EE904A78F06CFAA3238DF859
:10DE7000043095238DF8053056F058FB1322CDF869
:10DE80000700CDF80B1006F57C6001A9CDF80F5006
:10DE9000CDF8134037F080FA06B070BD2DE9F0419F
:10DEA0008AB00446884617460021232201A8109D07
:10DEB0001E4678F047FAA3238DF8043095238DF899
:10DEC000053001238DF8063056F030FB2B68CDF875
:10DED0001B306B68CDF80700CDF80B10CDF81F3064
:10DEE0002322AB68CDF80F8001A904F57C60CDF842
:10DEF0001370CDF81760CDF8233037F04DFA0AB023
:10DF0000BDE8F0819720704710B500F540530446F6
:10DF1000D3F8780203681B6898471A22C1B204F547
:10DF20007C6037F0F9FB04F59070BDE810400FF00D
:10DF3000FDBF000037B500F506510446012204314B
:10DF400036F006F8012504F50051104A009500232B
:10DF50003031DA2033F01AFE0D4A0095002304F523
:10DF60007C61FD2033F012FE0A4B1A68D20705D4FB
:10DF7000094A1D6004F58C540C34146006480121D4
:10DF800003B0BDE8304033F053BE00BF08010A08BB
:10DF9000645D0908C8250020002200200020704789
:10DFA000002070470069C0F3401070470F299DBFE3
:10DFB000302303FB010050300020704700207047E1
:10DFC0000120704770470000036800221B68184753
:10DFD00000207047002070470020704700207047E5
:10DFE00000207047002070470020704700207047D5
:10DFF00000207047002070477047000010207047D5
:10E0000000207047704700000320704701207047D0
:10E0100070470000012070470020704770470000E3
:10E0200000F50750143070470048704784CB08084B
:10E0300008B500F54050D0F8780203681B6898478F
:10E04000C0B208BD034808600F2111704FF0FF32C5
:10E050001A60704714E308080020704700207047DA
:10E060007047000015F024BF37F0FCBA41F036BC11
:10E070003FF01EBE05F0CCBB06F0ACBA00F0D4BE3B
:10E0800000F0CEBE00F0ECBE01F024BC00F0BABE41
:10E0900000F0C0BE00F02ABF70B51F4B036000F552
:10E0A00000530446D3F8D00C1C4AC3F8202B08B107
:10E0B00007F096FD1A4B236004F5805393F86C2EFD
:10E0C00042B9D3F8685E2DB1284614F013FE2846F5
:10E0D00007F082FD04F58B50103053F0F9FC04F585
:10E0E0008350183043F0CCFC04F6C44504F6644673
:10E0F000B54204D0183D284614F06CFAF8E7094BF5
:10E10000C4F8983804F6941039F0DEF804F510607D
:10E1100039F0DAF8204670BD48E40808807509082F
:10E12000C8560908F82C090838B5484B044640F889
:10E13000043B43F01DFE04F1100006F071FB04F1F6
:10E14000680035F077F904F590700FF0D1FA04F516
:10E15000866005F0CDF904F2545007F043FD04F653
:10E16000980015F049FD04F5446043F089FD04F57D
:10E17000516034F081FE04F57C6037F055F804F509
:10E180008350183043F064FC04F58550143006F0D9
:10E1900033FC04F58B50103053F086FC04F58C50A2
:10E1A0000C3035F053FC04F58F5044F08BFF04F530
:10E1B00080530025264A83F8045204F5905004F554
:10E1C000905304331430136030F08CFF04F59350F7
:10E1D0002946083001F0D8FE04F5C55018304CF03F
:10E1E0000BFB04F5E7501C3050F0BCFC04F5F0507C
:10E1F000143052F0B3FD04F5F350183053F0E8F941
:10E2000004F5F650103001F01FFD04F500503030D9
:10E210004CF0BEFF04F50250083049F041FE04F511
:10E22000005304F5055083F844510A4D1C3053F057
:10E230008BFF2B6813B1084856F040F92046074978
:10E2400033F01CFF2C60204638BD00BFC8560908BB
:10E250000C640020885B002014E1080800560908BF
:10E2600010B59FED225A9FED224A9FED222ADFED45
:10E27000221A9FED221A9FED220A86B00446F0EE84
:10E28000453AB0EE453AF0EE452AF0EE450AF7EE93
:10E29000004A54308DED054A8DED042ACDED031A68
:10E2A0008DED021A8DED015A8DED000A4CF044F807
:10E2B0009DED015A9DED054A9DED042ADDED031A01
:10E2C0009DED021A9DED000AF7EE004AF0EE453A88
:10E2D000B0EE453AF0EE452AF0EE450A04F59E70A0
:10E2E0004CF02AF8204606B010BD00BF0000000028
:10E2F000CDCCCC3D00007A450AD7A33CCDCC4C3DDB
:10E30000CDCC4C3EF0B500F50055224BB5F886213A
:10E310001A7087B0044643F011FA42F0C7FF204656
:10E3200001F00CFC04F5805393F8E42412F0010290
:10E3300010D102A8019207F0ABF904F5935002A99D
:10E34000083002F0DBFE28B12368019ADB6C02A9D9
:10E3500020469847104E3368DB6A93F89C7037B1BB
:10E3600095F846311BB956F0D9F8C5F8480133681D
:10E3700085F84671DB6A93F89C20084B5A7135F09A
:10E38000CBFA35F01DF804F50B5007B0BDE8F040AE
:10E390004CF022B805230020CC250020B55A0020DF
:10E3A000FFF7B0BF10B50821044601F0ABF918B172
:10E3B00017F0DEF815F024FB0121204601F0A2F948
:10E3C00010B12046FFF72EFD0421204601F09AF9F6
:10E3D00018B104F57C6036F09DFB1021204601F059
:10E3E00091F928B104F57C60BDE8104036F02CBCF2
:10E3F00010BD0000FFF7D6BF102925D8DFE801F0D7
:10E40000090D11191524242424241D242424242432
:10E41000210000F54A500430704700F54A502C3076
:10E42000704700F54A502430704700F54A500830D4
:10E43000704700F54A502830704700F549503C308D
:10E44000704700F54A5070470020704708B54CF0FF
:10E45000A3FF044B1B68DB6A93F89C10BDE80840DF
:10E460004CF076BFCC250020FFF7F0BF2DE9FF412F
:10E470000446FFF759FE884B236004F5065004F567
:10E4800000550430FFF7ECFE002304F50E50C5F8EC
:10E49000A8332C3041F040FCDFF860827F4BC5F898
:10E4A000AC3342F2FC3642F2FC67A01941F0C2FDE7
:10E4B00044F806803036BE42F7D1A01943F01EF86A
:10E4C00004F52C50043039F041F904F52C5010308B
:10E4D00039F03CF904F52C570023A5F81C3B2037F4
:10E4E0006F4BC5F8203B07F1080055F075F904F5AE
:10E4F0002D5604F52E580C3608F1300830461436E7
:10E500003DF0E8FD4645F9D10723C5F8D43C00238A
:10E51000A5F8D83C4FF4CB7007F05CFBC5F8D00CE5
:10E5200004F533501C3055F057F904F534502030C1
:10E5300055F052F95B4B1A6802B91F605A4BC5F887
:10E54000203B0026594B03930294009604AB04F53C
:10E55000345013E90C0040213C3005F0B9FC04F5BF
:10E56000495004F54055283007F092F804F54A5315
:10E57000C5F878324E4BC5F87C324E4BC5F8803228
:10E580004D4BC5F884324D4BC5F888324FF07E5361
:10E59000C5F88C324A4BC5F8A43204F54A58494BA9
:10E5A000C5F8A8320027484BC5F8AC3208F130084E
:10E5B000C5F89872C5F89472C5F8907208F1040015
:10E5C00007F066F808F1140007F062F83F4B404886
:10E5D000C5F8DC7204F54C52C5F8E072C5F8E47277
:10E5E0001860103233464FF6FF774FF0140C9EB28E
:10E5F0000CFB06010133097C0029F8D1354B364963
:10E600001E800B6813B1354855F058FF85F811335B
:10E6100004F54C50012385F8123314300A6053F08E
:10E6200041FE2F4BC5F814332E4BC5F86843C5E99E
:10E63000DB342D4B04F54E50C5E9DD342B4BC5F8CA
:10E640007C33103007F024F804F54E502C3007F0DE
:10E650001FF804F54F50083007F01AF804F54D562E
:10E66000234BC5F8DC33A5F8E07306F1A40007F0EE
:10E670000FF84FF0FF330C36C5F840341D4B1E49E0
:10E680001E60304633F0FAFC2046A5F88873A5F8E2
:10E69000A47304B0BDE8F08148E40808F8E0080875
:10E6A00080750908A45E002024A8080895E00008E9
:10E6B000BCE40808A0E1080804E50808F0E408083C
:10E6C00018E50808B4E10808C8E10808505B002014
:10E6D00030DB08084C5B00200C5B002028E10808B8
:10E6E00060E1080859E000085DE0000861E000080A
:10E6F0000000FFFF845A00202C3909084CE108086B
:10E7000038B5054B1C6823680A461D68034B014653
:10E710002046A847002038BDCC250020D025002069
:10E7200010B555F01FFB064C064B18602046FFF74E
:10E730009DFE2046044A0549BDE8104075F0D4B856
:10E74000D0250020CC25002004BD002099E0000841
:10E7500038B52DED028B0D46F0EE608AB0EE408AA2
:10E76000144602F0E9FE90ED937AD0ED957A67EECB
:10E77000877A90ED927A67EEA87AE7EE087AC5ED8F
:10E78000007AD0ED920AD0ED937A90ED957A67EE0B
:10E79000A07A67EEA80AE7EE480ABDEC028BC4ED4A
:10E7A000000A38BD30B52DED068B83B0F0EE409AEF
:10E7B000B0EE60AA0D46044602F0BEFED0ED7F7AB0
:10E7C000D0F80002B8EEE79A17F09AFB07EE900A2D
:10E7D000F8EEE78A79EEC9AA3AEE688AFDEEEAAA6F
:10E7E000B0EE480A17F06EFBBDEEC00A5DB110EE48
:10E7F000103ADFED190A002BCCBF38EE608A38EEF4
:10E80000208ABDEEC80AF8EEC00A01AAB8EEEA0AEC
:10E8100069462046FFF79CFFDFED107A104B009A07
:10E82000C3F8F82269EEA79A019AC3F8FC2229EEF0
:10E83000279A2AEE27AA68EEA78AA3F58053C3ED8C
:10E840009B9A83ED9C9A83EDD5AAC3EDD68A03B03B
:10E85000BDEC068B30BD00BF00A00C470AD7233C9F
:10E86000D055002038B52DED028B0D46B0EE408A14
:10E87000F0EE608A144602F05FFED0ED937A9FEDD1
:10E88000147AF0EEE77AF4EEC77AF1EE10FA1DD4BE
:10E89000D0ED957A90ED927A67EEE87AE8EE077A15
:10E8A000C5ED007A90ED937AD0ED957A90ED926A6D
:10E8B000C7EE876A0120C6EE077A67EEA80AE6EE81
:10E8C000880AC4ED000ABDEC028B38BD0020FAE7CF
:10E8D0000000003430B55F4C2DED068BB4F9C43127
:10E8E000DFED5D8A5B4285B008EE103A054604F61E
:10E8F000043038F02FFFB8EEC88A90ED00AAB4F9C2
:10E90000C43128EE288AF6EE009A98EE29AA04F679
:10E91000043008EE103A38F01DFFB8EEC88A90EDCA
:10E92000009AB4F9C83128EE288A04F5316098EECF
:10E93000299A08EE103A38F00DFFB4F9CA31D0ED3B
:10E94000009A04F531600AEE903A38F003FFB8EE11
:10E95000C88AF8EEEAAAD8EE289A6A4602A990ED8B
:10E96000008A8DED00AA9AEEA88A2846F0EE4A0A9F
:10E97000B0EE690A8DED038A8DED019ACDED029A14
:10E98000FFF770FF01AA03A9F0EE490AB0EE480AAA
:10E990002846FFF767FF02F0CFFDD0F8000217F01E
:10E9A000AFFA04F58053D4ED6F7A93EDBB0A30EEE5
:10E9B000270A08EE100A20EE280A17F083FAB8EEAC
:10E9C000C88A30EE480A17F07DFADFED247A9DED13
:10E9D000007AB5EEC00AF1EE10FAACBF70EE676ACD
:10E9E000F0EE406AB4EEE67AB4BF70EE277AF0EE4D
:10E9F000407AF1EE10FA2ADD9DED016AB4EEE76A85
:10EA0000F1EE10FA23D5B5EEC00AF1EE10FA08DDEA
:10EA100077EE665A37EEC65AF4EEC55AF1EE10FAA2
:10EA200013D4B5EEC00AF1EE10FA10D537EE667ABF
:10EA300077EEC67AB4EEE77AF1EE10FACCBF012099
:10EA4000002005B0BDEC068B30BD0120F9E70020A9
:10EA5000F7E700BFD04500200000C84200A00C47E7
:10EA600070B5314C2DED028BA4F58055D5ED6F7A44
:10EA700094EDBB0ADFED2D8A30EE270A84B020EE3C
:10EA8000280A064617F01EFAB5F9CA31D5ED707A94
:10EA900001EE103AB5F9C831B0EE408A00EE903A76
:10EAA00094EDBD0AB8EEC11A30EE270AF8EEE00A7E
:10EAB0000C2017F05BFA20EE280A30468DED010A93
:10EAC000FFF708FF9DED010A0146F0EE480A3046C7
:10EAD000FFF768FE9DED010A03AA02A9F0EE480ABD
:10EAE0003046FFF735FEB5F9C631002B0DDD07EED8
:10EAF000903A94EDBC7AF8EEE77AB4EEE77AF1EE6C
:10EB000010FA02DA94F8B0324BB99DED020A0848C7
:10EB100000F00CFB9DED030A054800F0E3FB04B098
:10EB2000BDEC028B70BD00BFD05500200000C84274
:10EB3000D025002038B5484C94F80C3313F001016F
:10EB4000054643D1A4F580529FED447AB2F998214D
:10EB500094EDBB0A07EE902AF8EEE77A13F0100F57
:10EB600067EE877AF7EE006ABFEE007A08BFB0EE74
:10EB7000667AA7EE270AC3F30012DFED397A84ED37
:10EB8000BB0AB5EEC00AF1EE10FA0AD51AB161F36C
:10EB9000041384F80C33B4EEE70AF1EE10FA06DC45
:10EBA0000BE0B4EEE70AF1EE10FA06DD2AB994F8AC
:10EBB0000C3343F0100384F80C339FED291ADFED7A
:10EBC000290A2C2017F0D2F984EDBB0A94F80C33F3
:10EBD0009807C3F340012ED4234A9FED207AB2F95F
:10EBE0009A0107EE900AB2F9C801B2F9CA21F8EE0B
:10EBF000E77A01EE102A00EE900A1A0767EE877A8C
:10EC0000F8EEE00A94EDBD7AB8EEC11A18D577EEA9
:10EC1000677AF4EEE07AF1EE10FAC4EDBD7A03D52E
:10EC200061F3C30384F80C3394EDBD0A3C2017F064
:10EC30009DF984EDBD0A2846BDE83840FFF710BFB6
:10EC400077EE877AF4EEC17AF1EE10FAC4EDBD7A70
:10EC5000EADD43F00803E5E7D05500200AD7A33CDE
:10EC60000000B44300000000D04500200A20704797
:10EC700001207047094B93F8B012024609B1FFF723
:10EC8000EFBE93F8111329B9A3F5805393F8D0314F
:10EC9000DB0702D51046FFF74DBF7047D055002067
:10ECA000042070470120704730B52DED028B8BB0EA
:10ECB000044655F033FC07AB054606AA05A9201DFE
:10ECC00018F072FE274A9FED288A136841F28831B6
:10ECD000EB1A8B421CD915603FF0ECFEDDED067A95
:10ECE00067EE887A054617EE900AFDF705FCDDED24
:10ECF000077A67EE887ACDE9020117EE900AFDF7F0
:10ED0000FBFB1A4ACDE900010621284639F0E2F85A
:10ED1000DDED067ADDED070A9FED150A60EE880A43
:10ED200027EE888A60EE800A204628EE000A00213D
:10ED3000FFF738FDDDED070A9DED060A09AA08A9CF
:10ED40002046FFF705FD9DED080A0A4800F0EEF9A0
:10ED50009DED090A074800F0C5FA0BB0BDEC028B27
:10ED600030BD00BF185A0020E02E6542C8E40808F4
:10ED70000000C842D02500200020704701207047C5
:10ED8000024B01461868026812681047AC5E00200A
:10ED900008B50020FFF7F4FFC188472042F03AFB96
:10EDA000472042F003FA0120FFF7EAFFC18848201C
:10EDB00042F030FBBDE80840482042F0F7B90000BF
:10EDC0000220704701207047FFF7B4BE08B50B461C
:10EDD000013BDBB2012B114611D85BB9472042F051
:10EDE00019FB472042F0E2F942F0D8FB42F0BEF8AE
:10EDF000012008BD482042F00DFB4820F2E700202A
:10EE0000F7E7000008B541F0E1F8BDE8084040F040
:10EE1000BDBF000000F593500021083002F012BB86
:10EE200000F2545007F068BB10B5044607F054FCDC
:10EE300090F921308BB190F8403373B194F9783563
:10EE40005BB1064B1B68DB6A93F89C302BB904F26C
:10EE50005450BDE8104007F067B910BDCC25002024
:10EE600070B5044600F590700FF0B8FF94F8E433E5
:10EE70001C4904EB0312D2F894010A68824210D0B4
:10EE8000B02202FB034294F8285492F8C12145B9FC
:10EE9000022A06D9144E08603278012A02D9013AB2
:10EEA000327070BDFDD104F54055D5F870222AB9F5
:10EEB000D5F8742212B905233370F2E7B02202FBB1
:10EEC000034303F5E6730FCB05F51A7585E80F00CC
:10EED000236804F54951DB6C00222831204698470D
:10EEE0000023E9E71C5A00200C2200207047000094
:10EEF00037B5044642F022FC42F0D8F904F500553B
:10EF00004721002042F0D4FA4821012042F0D0FAF3
:10EF1000B5F8C41101EB810101EB8101490089B20F
:10EF2000472042F02DF9B5F9C831B5F9CA110F4D96
:10EF3000C91A01EB810101EB8101490089B2482026
:10EF400042F01EF942F02AFB42F010F804F52C5072
:10EF500001A90430019538F05BFC04F52C5001A99F
:10EF60001030019538F054FC03B030BDCDCCCC3D11
:10EF7000F0B52DED028B00F5005785B0B7F8C8212C
:10EF8000B7F8CA3104466425482012FB05F613FB86
:10EF900005F542F0E5F804F5405304F50750183044
:10EFA000B0EE408ADFED230A93EDBE0A0190002106
:10EFB0004BF07CFB07EE906A38EE000AF8EEE77A39
:10EFC0000198B4EEE70AF1EE10FA25D98DED020AA8
:10EFD00007EE905A9DED027AF8EEE77AF4EEC77AE2
:10EFE000F1EE10FA03D8CDED027A4BF053FA482037
:10EFF0009DED020A42F0A0F897F81D3B04F52C5055
:10F00000103083B10C4B039303AA02A938F004FC1F
:10F0100005B0BDEC028BF0BD0190CDED027A4BF056
:10F0200039FA0198D4E702A938F096FB012387F852
:10F030001D3BEDE70AD7A33C0AD7A33C00F540539C
:10F0400000F50050D0ED6C7A90ED6E6A93EDBE7ACB
:10F0500067EE867AF0EEC76AF4EEE76AF1EE10FA30
:10F0600004D59FED180A482042F066B8DFED167A05
:10F07000B5EEC07AF1EE10FA20EE270A10DDB0F8F6
:10F08000C831642213FB02F307EE903AF8EEE77AF8
:10F09000F4EEC07AF1EE10FA02D59FED0C0AE2E729
:10F0A000B0F8CA31642213FB02F307EE903AF8EE8F
:10F0B000E77AF4EEC07AF1EE10FA02DD9FED040A71
:10F0C000D1E77047000000000000C84200A00CC655
:10F0D00000A00C4610B5044600F5405304F500545A
:10F0E00000F50750DFED100A93EDBE0A002118303D
:10F0F0004BF0DCFAB4F9CA01B4F9C8313221C21AB2
:10F100001B1A4A434B4301EE102A00EE903A80202E
:10F11000B8EEC11AF8EEE00A16F028FFBDE810407C
:10F12000482042F009B800BF0AD7A33C00F50053BD
:10F1300093F9A831012B03D0022B03D0FFF718BF9E
:10F14000FFF77CBFFFF7C6BFF0B52DED028B00F5D2
:10F1500000563223B6F8C451DFED310A15FB03F532
:10F1600000F50B5700F5405393EDBF0A83B0002123
:10F17000044638464BF09AFA9FED2A1ADFED2A0A28
:10F18000BF2016F0F3FE4720B0EE408A41F0E8FFC2
:10F190009FED241ADFED240A30EE080AC02016F095
:10F1A000E5FE6B4207EE903AF8EEE77AB4EEE70A36
:10F1B000F1EE10FA26D98DED000A07EE905A9DED7A
:10F1C000007AF8EEE77AF4EEC77AF1EE10FA04D896
:10F1D0003846CDED007A4BF05DF947209DED000AF1
:10F1E00041F0AAFF96F81C3B04F52C5004307BB18B
:10F1F0000E4B019301AA694638F00EFB03B0BDEC3B
:10F20000028BF0BD3846CDED007A4BF043F9D4E7E0
:10F21000694638F0A1FA012386F81C3BEEE700BFEF
:10F220000AD7A33C00A08C4600A08CC60AD7A33CFA
:10F2300000F540539FED117AD3EDBF7A00F50050F1
:10F2400067EE877A90ED6D6A90ED6B7A27EE067A1D
:10F25000F0EEE76AF4EEC76AF1EE10FA04D59FED1E
:10F26000080A472041F068BFF5EEC07AF1EE10FAC7
:10F27000CCBF9FED040A9FED040AF2E70AD7233CB6
:10F280000000000000A08C4600A08CC610B504460B
:10F2900000F5405304F50054DFED110A93EDBF0A69
:10F2A000002100F50B504BF001FAB4F9C4314FF6D0
:10F2B000CE71322213FB02F213FB01F301EE102A8E
:10F2C00000EE903AF120B8EEC11AF8EEE00AB1EE85
:10F2D000400A16F04BFEBDE81040472041F02CBF1D
:10F2E0000AD7A33C00F5005393F9A931012B03D0B1
:10F2F000022B03D0FFF728BFFFF79ABFFFF7C6BF67
:10F30000FEF702BE70B500F5005088B090F9D1014B
:10F310000C46D8B105210E4842F0CEFA0921064626
:10F320000B4842F0C9FA01210390094842F0C4FA9F
:10F3300004AD00210346039A00912846314606F0A9
:10F34000C7F995E80F0084E80F00012008B070BDF0
:10F35000205A002037B50C460022054611460F48BA
:10F3600042F0B6FA62680D48012142F0C9FAA2687B
:10F370000A48052142F0C4FAE2680848092142F02F
:10F38000BFFA05F5075001240DF1070111308DF882
:10F39000074033F06BFC204603B030BD205A0020FC
:10F3A00037B503680191DD6C04460FF055FD90F808
:10F3B000C412019AB02303FB0101AC3120462B4655
:10F3C00003B0BDE8304018477FB5044604F59356B6
:10F3D000684608360D4606F05BF96946304601F08E
:10F3E000B1FE48B929462046FFF7B4FF064650B99A
:10F3F0000026304604B070BD2946304601F06CFD51
:10F400000028EFD1F4E795E80F0004F549542834BB
:10F4100084E80F00EDE7000010B5074B1B680446B9
:10F42000D86A036801211B68984704F57C600121B4
:10F43000BDE8104035F098BFCC25002010B5074B33
:10F440001B680446D86A036800211B68984704F5C6
:10F450007C600021BDE8104035F086BFCC2500203F
:10F4600010B5044655F05AF804F500540021C4F8CC
:10F47000A803472041F0ECFF0021482041F0E8FFBD
:10F4800042F08CF8BDE8104041F070BD70B5044604
:10F4900004F5005304F5405583F84421D5F878323B
:10F4A0008B420846164627D0C5F878120B685B6871
:10F4B000984710B32046FFF7AFFFD5F878020368EE
:10F4C0001B6898473246C1B204F57C6036F024F9D7
:10F4D00004F52C500021203004F580543FF0E4FE68
:10F4E00004F58D63D3ED007A9FED067AF8EEE77AA6
:10F4F00067EE877AC5EDBB7A70BD2046FFF79EFFA9
:10F50000DBE700BF0AD7233CF7B5044600F590506F
:10F5100014302FF077FF5F4B04F5345001223C305C
:10F520009A71DA7104F5866704F07EFD04F52C55B6
:10F530000823C4F844343846203504F0E9FB284653
:10F540003CF012FE284640F0C9F907F0C5F8202328
:10F55000036307F0C1F808F037F904F59356022366
:10F56000C4F8743104F5907008360EF03DF9304659
:10F5700000F078FE04F58053002283F87125B4F979
:10F58000A43004F698001BB9B4F8A230A4F8A43053
:10F59000B4F8A41016F05AF8304600F05DFF384673
:10F5A000012104F045FA3C4B00933C4B019302AB24
:10F5B00013E9060004F57C6035F0CAFE40F006FD54
:10F5C0009922292141F012FC40F000FD40F0A6FCF8
:10F5D00004F500562046FFF78BFC96ED677ADFEDC9
:10F5E000307AF0EEC76AF4EEE76AF1EE10FA04F54D
:10F5F000405747D8D6ED687ADFED2A6AB0EEE76A61
:10F60000B4EEE66AF1EE10FA3CD8DFED276A27EE99
:10F61000267A67EEA67ABDEEC77AFDEEE77A87ED29
:10F620009C7AC7ED9D7AD7F8703243B9D7F8743217
:10F630002BB904F5495128312046FFF763FE1B4BD7
:10F640001B68986A03684FF47A715B68984796F96B
:10F65000CE112046FEF7D0FE014610B904F54A51FE
:10F6600004311F222046FFF711FFD6ED697AF5EE2F
:10F67000C07AF1EE10FA0BDD204603B0BDE8F04091
:10F68000FFF7EEBE0A4A0521284638F023FCCAE7F8
:10F6900003B0F0BDB55A0020D025002001F30008CA
:10F6A0000000B442000034438096184BCC25002063
:10F6B00024E5080808B50A2922D8DFE801F00D1969
:10F6C00011151D2121212121060000F549513C3150
:10F6D000FFF7DCFE012008BD00F54A510431F7E7D1
:10F6E00000F54A512431F3E700F54A512831EFE79C
:10F6F00000F54A512C31EBE700F54A510831E7E7B4
:10F700000020E8E700F57C6036F0AEBC014803213C
:10F7100042F034B8205A002070B505462DED028B1A
:10F7200005F5405454F0F0FED4F8D432DFED1D7AE4
:10F73000C31A08EE103AB8EE488A28EE278AF1EE8E
:10F74000047AB4EEE78AF1EE10FA29D504F52D73A8
:10F750000FCB04F5317686E80F00D4EDB80A94EDAE
:10F76000B70A05F54B5068EE200A28EE000A04306F
:10F7700006F01EFADFED0C7A94EDB97A27EE277ABF
:10F78000D4EDB27AF8EEE77A0123E7EE087AFDEEDF
:10F79000E77AC4EDB27A84F8B032BDEC028B70BD6A
:10F7A0000023F8E7BD3786350000C84230B585B084
:10F7B0006D460446284605F06BFF04F59350294634
:10F7C000083001F09BFC50B104F54054002384F84C
:10F7D000123395E80F0004F51A7484E80F0005B0A1
:10F7E00030BD0000F8B52DED028B00F54054054604
:10F7F00094F8B032002B5ED0D4F8782200F54A534A
:10F80000243300F5495600F54B579A4206F1280675
:10F8100007F1040717D094F80C33DA0713D43946EC
:10F82000304606F0B3F89FED277AF6EE007AE0EE68
:10F83000077A9FED257AFDEEE77AF8EEE77A67EE34
:10F84000877AC4EDBB7A3946304606F041F905F5B2
:10F85000005584EDBC0A95F9AA31DFED1C6AD4F895
:10F860007802012B05BFD4F8C832D4F86C22D4ED4D
:10F87000BA7A9B1A08BF07EE903AF8EEE77A87EE5D
:10F88000A67A84EDC17A03681B689847022812D0D3
:10F8900094F80C339B070ED495F9AA31D4EDBC0A29
:10F8A0009FED0B8A53B994EDC00A74F065FB20EE0E
:10F8B000080A84EDBD0ABDEC028BF8BD94EDC10AC7
:10F8C000F3E700BFA00CB3450AD7233C0000C842B1
:10F8D000E02E654273B50446FFF71EFF2046FFF792
:10F8E00065FF04F500552046FFF77CFFD5ED697AEA
:10F8F000F5EEC07AF1EE10FA09DC244B1E68F06ACE
:10F900000368DB699847012816D102B070BD54F036
:10F9100005FED5F8A83395ED697ADFED1D6AC01AAA
:10F9200007EE900A27EE267AF8EE677AF4EEC77AA9
:10F93000F1EE10FAE1D5E8E7F36A93F89C10E9B923
:10F9400095F9CF31012B10D19FED120A472041F0DC
:10F95000F3FB9FED100A482041F0EEFB41F01EFE44
:10F9600002B0BDE8704041F001BB4720019141F079
:10F9700051FD0199482041F04DFDEFE704F5405459
:10F98000D4F8780203689B689847E7E7CC25002005
:10F9900000007A440000000037B54B68054613B9F3
:10F9A0008A68002A49D005F540540A20C4F8BC32C0
:10F9B0008B68C4F8C032CA6892FBF0F2C4F8B8226F
:10F9C0000B6993FBF0F3C4F8E832B1F91630DFEDC0
:10F9D0001C7A07EE103AB1F91830B8EEC77A87EE04
:10F9E000276A07EE103AB1F9143084EDB86AB8EE20
:10F9F000C77AC7EE276A07EE103AB8EEC77AC4EDA9
:10FA0000B96AC7EE275AC4EDB75A54F07DFDC4F861
:10FA1000D40254F083FD0221C4F8D8022846FFF72F
:10FA200071FE50B105F54B531C330093D4E9AF126E
:10FA3000D4F8B8322846FEF731FA03B030BD00BF23
:10FA40000000C84210B52DED028B044691ED018AED
:10FA5000DFED207A94F8413428EE278A00F586609D
:10FA6000242202FB0303F0EE480A93ED090A03F097
:10FA700087FCB4EE400AF1EE10FAF0EE400A1FD611
:10FA80009FED157AF0EEC07AF4EE477AF1EE10FAB7
:10FA900016DC04F54053D3EDC27A93F80C2377EECD
:10FAA000807A5107C3EDC07A0AD5F1EE407A002181
:10FAB0006FF38202C3EDC27AC3F8001383F80C23FC
:10FAC000B0EE480ABDEC028B2046BDE81040FEF7C0
:10FAD000C1B900BF0000C842FFFF7F7FB1F900300D
:10FAE00007EE903AF8EEE77A00F5405010B5C0ED19
:10FAF000BB7AB1F9023007EE903AF8EEE77A0023CC
:10FB0000C0F8F032C0EDBD7AB1F9002090F80C33A6
:10FB100047F6FF74121B18BF012262F3000380F83E
:10FB20000C33B1F9023090F80C231B1B18BF0123D2
:10FB300063F3410280F80C2310BD000010B500F5FE
:10FB40004054D4F8D80250B154F0E8FCD4F8D8327C
:10FB5000C01A41F2873398428CBF00200120014B2C
:10FB6000187110BDB55A002070B52DED028B00F54F
:10FB700000541646B4F9CA2194ED700A01EE102A19
:10FB8000B4F9C82100F54053D3EDBD7AD3EDBB8A5B
:10FB900000EE902ADA20B8EEC11AF8EEE00A30EE54
:10FBA000270A0D4616F0E2F9B4F9C821B4F9CA31B2
:10FBB00007EE902AF8EEE77A9B1A30EE670A07EE16
:10FBC000903A30EE000AF8EEE77AB7EE008A80EE5F
:10FBD000277A37EE487A86ED007A94ED6F0A38EE90
:10FBE000800A16F02FF9B4F9C43107EE103A30EE5E
:10FBF000000AB8EEC77A0120C0EE077A77EEC87A1D
:10FC0000BDEC028BC5ED007A70BD000070470000AE
:10FC100000207047704700000020704700207047A8
:10FC200000207047002070479FED010A704700BF19
:10FC3000000000009FED010A704700BF00000000B7
:10FC4000002070477047000010B50446143000F0E3
:10FC500019F804F12C0000F015F804F1740054F0C8
:10FC600069FC04F1F40054F065FC4FF0FF33C4F874
:10FC70005031204610BD0000014B1868704700BF8E
:10FC8000245A002070470000F0B52DED048B91B090
:10FC900004466D46284605F0FBFC94F8BC33002B67
:10FCA00072D004F57A730FCB85E80F0094F8F8331F
:10FCB000D4EDEC8A94EDED8A94EDEE9A002B63D0AE
:10FCC00094F8D033002B5FD02D22002104A8D4F863
:10FCD000C073D4F8C463D4F8C853D4F8CC4376F0D6
:10FCE00031FBA3238DF8103095238DF81130462376
:10FCF0008DF8123054F01AFC9FED250A9FED257AFD
:10FD0000CDF8171068EE807ACDF8130067EE877A89
:10FD1000FDEEE77A17EE903A68EE007A29EE000AD7
:10FD200067EE877AADF81B30FDEEE77A20EE070A22
:10FD300017EE903AADF81D3016F0AEF8DDED017A11
:10FD40009FED157ACDF82D70BCEEC00AF8EEE77A7B
:10FD500010EE103A67EE877AADF81F3017EE903A42
:10FD6000CDF82130029BCDF82530039BCDF829300A
:10FD7000CDF83160CDF83550CDF8394036F0AAF9DC
:10FD80002D2204A935F008FB11B0BDEC048BF0BDA9
:10FD9000E02E65420000C8420AD7233C30B52DED65
:10FDA000028B8BB0044624220D4601A8002176F078
:10FDB000C9FAA3238DF8043095238DF80530482324
:10FDC0009FED1F8A8DF8063054F0B0FBD4ED817A98
:10FDD0002B68CDF80F3067EE887A95ED020ACDF8E2
:10FDE0000B1017EE903AD4ED827ACDF8133067EE0F
:10FDF000887A6B68CDF8173017EE903ACDF8070087
:10FE0000CDF81B3016F01EF810EE103A94ED830A70
:10FE1000CDF81F3020EE080A16F014F810EE103A54
:10FE2000CDF8233094F80C338DF8273036F052F9A2
:10FE3000242201A935F0B0FA0BB0BDEC028B30BD25
:10FE4000E02E654230B587B014460D4618220021D9
:10FE5000684676F077FAA3238DF8003095238DF865
:10FE6000013049238DF8023054F060FBA3680393FE
:10FE7000E36804936368CDF807100593CDF8030099
:10FE80008DF80B5036F026F91822694635F084FAC1
:10FE900007B030BD10B58EB0044602A805F0F8FBDF
:10FEA00002A9204601F02AF9002845D001F044FBC0
:10FEB000694600F0BBFF1F22002106A876F042FA37
:10FEC000A3238DF8183095238DF819304A238DF827
:10FED0001A3054F02BFBDDED037A9FED1B7A049B67
:10FEE000CDF82330F8EEE77A059BCDF8273067EEA2
:10FEF000877ACDF81B0017EE903ADDED007ACDF849
:10FF00002B30F1EE677A17EE903ACDF81F102046AD
:10FF100001A9CDF82F3000F0FDFB78B1DDED017ABD
:10FF2000F1EE677A17EE903ACDF8333036F0D2F82A
:10FF30001F2206A935F030FA0EB010BD36F0CAF80F
:10FF4000DFED027AEEE700BF0AD7233C5241C07FC3
:10FF50000023036043608360C36003614361836186
:10FF6000C36103627047000090F8C432B02202FB04
:10FF7000030390F8082393F8A13012B1012B28BF96
:10FF800001231846704700002DE9F04F04468BB05E
:10FF90004FF0000A0D461BF0E1FF84F814A204F5AF
:10FFA00006704FF07E5753F017FC4FF47A73A4F8A5
:10FFB000623284F86852C4F84872C4F84C72C4F8CB
:10FFC000507204F51B70002505F062FB04F52B79D7
:10FFD0000323C4F8803204F53476C4F89452C4F88C
:10FFE0009852C4F89C52C4F8A052C4F8A452C4F861
:10FFF000A8524846FFF7ACFF04F5487B3046FFF7B0
:020000040801F1
:10000000A7FFC4F81453C4F81853C4F81C53584637
:10001000FFF79EFFC4F84453C4F84853C4F84C5348
:10002000C4F85053C4F85453C4F85853C4F85C533C
:10003000C4F86053C4F86453C4F86853C4F86C53EC
:10004000C4F87053C4F88C53C4F89053C4F8945354
:10005000C4F8A853C4F8A453C4F8A053C4F8B053C8
:10006000C4F8B453C4F8B853C4F8CC53C4F8C85354
:10007000C4F8C453C4F89C73C4F8C07304F5757015
:1000800005F006FB04F57A7005F002FB04F58063C9
:10009000C4F8FC531D6004F5816304F583601D60A2
:1000A0005D609D6005F0F4FA04F22C4304F26448AC
:1000B0001D605D609D60684BC4F83C3404F50D73B1
:1000C000C4F8403404F50E73C4F8443404F50F73D7
:1000D000C4F8483404F51073C4F84C3404F24523D2
:1000E000C4F8503404F51173C4F8543404F58B6328
:1000F00040461D605D609D60FFF72AFF04F591603A
:10010000FFF726FF04F5976304F23C421D605D6033
:100110009D6004F2C44304F2A4501D605D609D60C4
:1001200004F59A631D605D609D6004F2DC431D6010
:100130005D609D6004F2EC431D605D609D6004F2B3
:10014000FC431D605D609D6004F5A463C2F8D4703B
:10015000C2F8D8701D605D609D6004F22C531D6074
:100160005D609D6004F5A9631F605D6004F26C53DF
:100170001D605D609D6004F5AF631D605D609D6006
:1001800004F5B2631D605D609D6005F081FA04F2C4
:10019000B45324221D605D6004F2BC5351461D60BF
:1001A0005D6004F2C45340461D605D6076F0CAF89D
:1001B00004F2E450C8F82070C8F81070C8F8007055
:1001C000FFF7C6FE04F5C16304F5C7601D605D60FE
:1001D0009D6004F214631D605D609D6004F5C4635E
:1001E0001D605D609D6004F22C631D605D609D601C
:1001F00005F04EFA194B1A491C60204631F03EFFBB
:1002000051462422584676F09DF8C4F84073C4F84D
:100210003073C4F8207304F5257207CA04F52873F7
:1002200083E80700484694EDAA1AD4EDA90A94ED94
:10023000A80A16F05FFA3546494668466E4616F03B
:100240007BF90FCE0FC50FCE0FC533682B6020464C
:100250000BB0BDE8F08F00BF64E70808285A002003
:1002600014E6080810B5044688B001F0EFF994F9D7
:100270003232012B02D1274804F0A0FB022B0AD115
:10028000032384F8323204A9012304F111008DF80C
:10029000103032F0ADFC94F8323284F8903204F22F
:1002A0003C4001F089F994F93132642B30D1652357
:1002B00004A904F231208DF8103032F0D7FC04A9E3
:1002C000204631F0B1F918B304238DF8183000231B
:1002D000CDE9013303930F230593694604A831F058
:1002E00075FB059B28B108AA02EB8302009942F82E
:1002F000581C0133112B0593EFD951F0B7FF9DED39
:10030000031ADDED020A9DED010A652151F06CFF33
:1003100008B010BD74E5080870B500F5257600F545
:1003200028758CB004463146284617F0CFFDE0B959
:1003300096E8070085E8070004F52B7194EDAA1AEA
:10034000D4EDA90A94EDA80A0191084616F0D2F955
:1003500002AD019902A816F0EFF80FCD04F5347440
:100360000FC40FCD0FC42B6823600CB070BD00000C
:1003700013B540F2411200F50671044601A812F0CF
:1003800075FA04F23C4001F0FFFA20461BF0C4FF6E
:1003900001A812F08DFA02B010BD0000F8B50B688C
:1003A000C0F804324B68C0F808328B68C0F80C32D1
:1003B00001F10C0607460C4600F548750FCE0FC537
:1003C0000FCE0FC533682B6004F1300207CA07F562
:1003D000457383E8070004F13C0207CA07F551732F
:1003E00083E8070004F1480207CA07F5547383E85D
:1003F0000700543494E8070007F5577383E80700B3
:10040000384601F037FA3846BDE8F84001F01ABA2C
:1004100013B5044600F23C40019002F0ABFE04F537
:10042000BB610198009102F003FA0099204602B0E6
:10043000BDE81040FFF7B2BF4A78064BC2F3401246
:100440001A754A78C2F380125A750A78C2F30012FC
:100450009A757047B55A002013B540F2F52204464C
:1004600000F5067101A812F001FA002104F23C40E7
:1004700001F0FCFC94F8603223B120461CF0F8F83F
:1004800084F8600201A812F013FA02B010BD000057
:1004900038B590F80C3305460C462BB1032B0BD026
:1004A00095F86832DB070CD405F5C7630FCB84E8F9
:1004B0000F0095F8480603E01BF084FF0028EFD0FA
:1004C00038BD0020FCE7000000F23C4090ED350A0A
:1004D0007047000000F23C4090ED360A7047000083
:1004E00010B490F80C230C462AB1032A0AD000203D
:1004F0005DF8044B704700F5B26007C884E8070058
:100500000120F5E75DF8044B1BF044BF90F884032D
:10051000431E58425841704738B590F80C330D4689
:100520008BB900F23C4001F0A1FA044610B9002456
:10053000204638BD01F0EEF9D5ED007A27EE800AAD
:1005400085ED000AF4E7D0EDE07AC1ED007A90F88D
:100550007C43002CEBD090EDDE7ADFED086AB4EE40
:10056000E67AF1EE10FAF7EE006AB8BFB0EE667AFE
:1005700067EE877AC1ED007ADAE700BF0000003449
:1005800090F80C33032B01D11BF084BE0020704780
:1005900090F80C23032A01D11BF09EBF00F23C40CF
:1005A00001F0C6BE30B590F80C3385B004460D4658
:1005B0008BB1032B18D004F5257017F0C1FC284629
:1005C00001A98DED010ACDED020A8DED031A17F098
:1005D00011FB012006E000F23C4001F0F1F9002897
:1005E000E9D1002005B030BD90F86032002BF8D082
:1005F0001BF05AFFDFE700007FB590F80C2332B103
:10060000032A4FF0000309D0039304930CE000F297
:100610003C4007B05DF804EB01F0ACBA03A90393CA
:10062000049305931BF02CFE9DED030ADDED040AF7
:1006300007B05DF804FB000007B590F80C3333B148
:1006400000F57F7003B05DF804EB17F0DFBB00F23C
:100650003C4001F08FFA68468DED000ACDED010AAD
:1006600017F0D4FB03B05DF804FB000090F80C0316
:10067000003818BF0120704708B590F80C23032AF2
:1006800005D0BDE8084000F23C4001F05DBA1BF027
:10069000F7FD012008BD000010B590F80C230C46B2
:1006A0001AB1032A07D0002010BDBDE8104000F2A7
:1006B0003C4001F0EDB91BF0F9FD012084ED000A8A
:1006C000F2E7000030B590F80C3385B005460C46D3
:1006D00023B1032B09D0002005B030BD00F23C400F
:1006E00005B0BDE8304002F0D3B8002302A9029360
:1006F00003931BF0ADFD0028EDD001A928461BF0A7
:10070000B3FD0028E7D0029B2360039B6360019B3D
:10071000A360E1E790F80C231AB1032A05D000206A
:10072000704700F23C4002F0D9B81BF09DBD0000BC
:1007300090F932323BB990F8683213F0010F14BFD0
:10074000032000207047032070470000F7B50446DF
:10075000FFF7EEFF0546002862D0032839D194F850
:1007600060326BB394F86832D8072BD501A92046C4
:100770001CF0A8F8BDF80430002B18BF002594F831
:10078000146206F0FD06012E4AD10023032D0193C9
:1007900007D101A920461CF0A1F820461BF0A8FEB5
:1007A000064604F23C4002F025F908B994F8090322
:1007B0009DF80430D90703D55A0701D59F0632D4D6
:1007C00000252DE020461BF01DFD002808BF002558
:1007D000D5E70025D3E713F0020F2EE094F9443259
:1007E00023B99DF80430DB092FD0E9E7002EF8D0BB
:1007F0000EF032FBFFF7B8FB022807D99DF8053051
:100800009806DDD59DF80430D906D9D5FB6A93F852
:100810009C30002BE5D118E0DA0601D41B0718D56F
:10082000284603B0F0BD0028FAD094F80923B4F9A3
:100830004C36002ACFD013F0010FF1D1154B1F68B1
:10084000FB6A93F89C30002BC8D19DF804309C07BC
:10085000E2D405F041FF05F03DFE0028B0D10EF0D6
:10086000FBFAFFF781FB0228AAD90EF0F5FA90F8FF
:10087000C432B02202FB030090ED2F7AF0EE007A32
:10088000B4EEE77AF1EE10FA9AD59DF80530DB095F
:10089000C6D195E7CC2500202DE9F04790F86032CD
:1008A00092B00446002B00F0948020461CF016F90C
:1008B0002046FFF74BFF03287BD104F5487800273B
:1008C000414620460097019702971BF0E3FD6946D9
:1008D00020461BF0D5FD009BC4F80432019BC4F8F0
:1008E0000832029BC4F80C32204600F0C3FF2046B9
:1008F00000F0A8FF14F03CFE054620461BF09AFCD1
:100900000028A8BFC6B203AA4FF0FF312046BCBFE3
:1009100095F8129395F813630397A8BFB14604970F
:1009200005971BF0D1FC03A817F00AFB4FF00C0A47
:100930000AFB095084EDD10AC4EDD20A84EDD31A22
:1009400004F5517100F5117017F00AFB04F55777A3
:100950000AFB065584EDC50AC4EDC60A84EDC71A24
:100960003A464FF0FF31204605F5C4751BF0C0FC38
:1009700095E8070006AE86E807003946304617F0CE
:1009800055FB04F52B72414609A815F065FD31466B
:1009900009A815F0E3FC09A9204684EDD40AC4EDAA
:1009A000D50A84EDD61A1BF099FF09A92046FFF756
:1009B00043FD94F84E36002B3AD109A804F068FEA6
:1009C00009A920461BF00AFD90B3012384F84E3696
:1009D0002EE0D0F864321BB953F0A0FDC4F86402D5
:1009E000154B1B68D86A03685B68984788B153F059
:1009F00095FDD4F86432C01AB4F86232984204D932
:100A000020461BF035FE84F8600294F860327BB11A
:100A10004BE753F083FDD4F86432C01A41F28733B8
:100A20009842E4D835F056FB35F03AFB0028DED189
:100A300012B0BDE8F08700BFCC25002090F80C3341
:100A400023B1032B4FF0000007D0704790F93222FA
:100A5000032A04D10A70012070470870FBE718468A
:100A60007047000073B50D460DF107010446FFF70E
:100A7000E5FF064628B19DF807302BB1032B09D0BE
:100A80000026304602B070BD04F5C7630FCB85E881
:100A90000F00F6E7294620461BF094FC94F86062AC
:100AA000EFE700007FB50E460DF103010446FFF7A6
:100AB000C5FF054618B90025284604B070BD9DF84D
:100AC000033083B1032B16D004F5257017F038FAE4
:100AD00001A930468DED010ACDED020A8DED031A14
:100AE00017F088F8E8E7314604F23C4000F068FF70
:100AF0000028E9D1DFE794F86032002BDBD03146E3
:100B000020461BF0D1FCDFE737B50D460DF107019C
:100B10000446FFF793FF28B19DF8073023B1032B5C
:100B20000FD0002003B030BD04F5BB631B682B6001
:100B300004F2DC5304F5BC641B686B602368AB6093
:100B4000F0E7204629461BF09BFC94F86002E9E799
:100B500010B50446FFF7ECFD18B1032807D00020BC
:100B600010BD04F23C40BDE8104000F053BF94F8C3
:100B70006032002BF3D020461BF044FB0028EED05F
:100B800094F8143203F0FD03012BE9D194F80C031F
:100B9000C31E58425841E3E710B50446FFF7C8FDAD
:100BA00080B1032810D194F8600250B153F0B6FC24
:100BB000D4F86432C01A44F62063984294BF0020EF
:100BC000012010BD0120FCE70020FAE708B502462D
:100BD000FFF7AEFD032804D110461BF07FFE012075
:100BE00008BD0020FCE7000030B585B00446019147
:100BF000FFF742F80199054610B9002005B030BD55
:100C00000191FFF70BF801990028F6D02846FFF76D
:100C100009F80028F1D0B4F84C365907EED494F80E
:100C20000933002BEAD00B4A1268D26A92F89C5022
:100C30006DB103A92046FFF7C9FF30B19DF80E3012
:100C40009A07DBD5C3F38000D8E72846D6E71846D5
:100C5000D4E700BFCC2500202DE9F04190F80C33FB
:100C60008CB00027032B06460C46154600970197CB
:100C7000029719D11BF0DEFA6A4680464FF0FF3129
:100C800030461BF035FBB8F1FF3FA7606760276077
:100C90000DD114F06DFC2B4690F81313224613F07F
:100CA000F5FC0CB0BDE8F0814FF0FF38EBE714F035
:100CB0005FFC2B4622465FFA88F113F0E7FC95EDC6
:100CC000000A684617F078F903A920468DED051A49
:100CD0008DED030ACDED040A17F0A8F906F52B7285
:100CE00006F5487103A815F0B7FB214603A815F0D7
:100CF00035FB84ED021A84ED000AC4ED010A95ED7E
:100D0000007ADFED037AA7EE271A84ED021AC8E70E
:100D10000AE81C4137B5054600F5067140F6033276
:100D200001A811F0A3FD2846FFF702FD044640B1DB
:100D300003280AD0002401A811F0BAFD204603B010
:100D400030BD28461BF002FBF5E728461BF0FEFAF3
:100D50000446F0E708B50246FFF7EAFC10B10328A5
:100D600006D008BDBDE8084002F23C4000F01CBEC1
:100D7000BDE8084010461BF0BDBD00000B4610B496
:100D800011462BB1032B09D000205DF8044B7047AE
:100D90005DF8044B00F23C4000F01CBE5DF8044BD3
:100DA0001BF01CBB13B50446FFF7C2FC0A46014604
:100DB00020460192FFF7E2FF70B9084B019A1B68C9
:100DC000DB6A93F89C0038B194F80C13204602B00B
:100DD000BDE81040FFF7D2BF02B010BDCC25002007
:100DE00037B504460D4640F2B25200F5067101A82F
:100DF00011F03CFD294620461BF00EFB94F80C3305
:100E0000032B054610D148B104F583612046FFF756
:100E1000C9FF84F82804204600F05CFD01A811F009
:100E200047FD284603B030BD0025F7E770B590F8C0
:100E30007C32DB0786B004460D460CD402F04EFF30
:100E4000437C242202FB0300D0ED0B7AF1EE677A9B
:100E5000C5ED007A3BE002A804F01AFC01A9204687
:100E6000FFF758FCE8B90DF0F7FF94F94432022B74
:100E70000646E3D1FFF778F80228DFD996F8C402D6
:100E80009FED147AB02303FB0066D4F87032D6F8D5
:100E9000B0209B1A07EE903AF8EEE77A67EE877A71
:100EA000D6E702A92046FFF77DFF0028DBD0D4F863
:100EB0007022039BDFED076A9DED017A9B1A07EE16
:100EC000903AF8EEE77AA7EEE67A85ED007A06B07A
:100ED00070BD00BF0AD7233CF0B50C4687B000F5C3
:100EE0000671064640F6863201A811F0BFFCA368E1
:100EF00053B9E36843B9636833B9002701A811F017
:100F0000D7FC384607B0F0BD204604F097FC002817
:100F1000F3D094E80F0002AD85E80F0000212846C9
:100F200004F04EFC07460028E7D096F87C32DB0739
:100F300004D435F0CFF8192135F008F895E80F0002
:100F400006F51B7C8CE80F0096F87C3243F0010319
:100F500086F87C32304600F0BDFC3DF0ABFD46210A
:100F60003EF0A2F93DF0A6FD45213EF09DF9054B6E
:100F7000A2681B68DB6A1A61E2685A6162689A615A
:100F8000BCE700BFCC25002038B5144B1B68DD6AD8
:100F90002B6804465B6828469847F0B12B690BB96B
:100FA0006A69D2B1C4F874326B69C4F87832A9693D
:100FB000002204F51B7004F071FB94F87C3223F0DE
:100FC000030343F0030384F87C323DF073FDBDE876
:100FD0003840034A062136F07DBF38BDCC250020BD
:100FE0009CE5080810B588B004460593FFF7A0FB00
:100FF0000328059B4FF000000AD10690079006A831
:1010000002900B9801900A98009020461BF056FA27
:1010100008B010BD38B50446FEF72EFE0546D0B127
:1010200094F80C33032B03D095F84E41204638BD7D
:1010300020461BF0BBF9FF280446F5D001462846A0
:10104000FEF7F0FD0028EFD021462846FEF7E6FD2A
:101050000028E9D0EAE70446E8E7000008B590F880
:101060000C33032B05D014F083FA90F91203C0B2AD
:1010700008BD1BF0DFF8431CF9D1F4E708B590F880
:101080000C3383B1032B03D1BDE808401BF0CAB871
:1010900033F0F4FB40F6ED424FF4801133F0A6FB41
:1010A0004FF0FF3008BD1846FCE7000090F80C3305
:1010B000032B01D11BF05EBE7047000090F80C338B
:1010C000032B01D11AF0FCBF704700001BF082B85F
:1010D00010B504461DF090FE2046FEF7D5FD2046D3
:1010E000BDE81040FEF7D6BE90F80C330BB1032BD1
:1010F00001D11BF0BBBE00207047000030B500F5E9
:10110000757304460D460FCB85E80F0094F8E40391
:1011100030BD0000D0F880330B6090F87C0370473E
:10112000D0F888330B6090F88503704730B500F530
:10113000677304460D460FCB85E80F0094F8AC03A7
:1011400030BD000030B500F5836304460D460FCB7B
:1011500085E80F0094F8280430BD000010B500F2B7
:101160002C4203460C4607CA84E8070093F838046B
:1011700010BD00002DE9F0432DED028B8BB005462C
:101180000E461746FFF746FF014680462846FFF702
:101190002BFD0446002848D0FEF76EFD4146FEF7C1
:1011A00043FD86ED000A95F93032002B3ADD0DF053
:1011B00053FEFEF7D9FE012834D90DF04DFE90F80C
:1011C000C432D5EDDE7ADFED5D8A96ED000AB022FD
:1011D00002FB030095F93032D0ED2F0A07EE103AEA
:1011E000F4EEE87AB8EEC77AF1EE10FAB7EE008ABC
:1011F000B8BFF0EE487A37EE201A20EE270A70EEDC
:10120000C70A40F2B63014F0B1FED5EDDE7AF4EE46
:10121000E87AF1EE10FAB8BFF0EE487A80EE277A5D
:1012200086ED007A01233B7003E095F8083333B96B
:10123000387020460BB0BDEC028BBDE8F08395F80A
:101240000C334FF00009CDF80490CDF80890CDF89C
:101250000C9043B1032B10D0CDF81090CDF8149022
:10126000CDF818907CB902233B703246414605F216
:101270003C4001F083FB0446DBE701A928461BF054
:1012800089F80446E8E795F80C33002BEBD004A965
:101290002846FFF763FF04460028E4D001A904A80C
:1012A00016F074FE07A8CDED080A8DED091A8DED34
:1012B000070A17F07FFA04A8B0EE408A17F07AFA0E
:1012C00095F93032002B30DD07EE903AF8EEE77AF0
:1012D0004FF47F7070EE670A37EE801AF5EEC00AA1
:1012E000F1EE10FA48BFDFED160AF4EE410AF1EE16
:1012F00010FAB0EE480AC8BFB0EE601A14F036FE1D
:10130000B0EE408AD5EDDE7A9FED0C7AF4EEC77A26
:10131000F1EE10FAB7EE007AB8BFF0EE477A88EE39
:10132000277A032386ED007A7DE7B5EEC08AF1EED9
:1013300010FA48BF9FED028AE4E700BF00000034C6
:101340000000000010B50446FFF788FE84F80D0386
:101350002046FFF783FE84F80E032046FFF77EFE4B
:1013600084F80F032046FFF789FE04F55A7184F8CC
:1013700010032046FFF7B4F884F8740300F0CAFAAB
:1013800004F5617284EDDE0A04F560712046FFF712
:10139000F1FE04F5627184F87C032046FFF7BCF887
:1013A00004F5637184F885032046FFF7E9F804F536
:1013B000677184F898032046FFF7F4F804F56C7120
:1013C00084F8AC032046FFF79FFB04F5707184F8A6
:1013D000BC032046FFF766FB04F5757184F8D00363
:1013E0002046FFF755F804F57A7184F8E4032046A7
:1013F000FFF738FB84F8F8032046FFF7FDF804F503
:10140000806384EDFF0A2046C3ED000AFFF714F95C
:1014100004F2044383ED000A04F2144204F58161EE
:101420002046FFF719FC04F583612046FFF7BAFC5C
:1014300004F22C4184F828042046FFF71DF984F8B3
:10144000380410BD37B50D46044600F0FFF81DB94D
:1014500014F08EF813F04AF84FF4BE7204F50671DA
:1014600001A811F003FA94F869322BB92046FFF76E
:101470008BFD012384F86932224B1D68A86A03683A
:101480009B6998472046FEF747FF2046FEF7C0FFBE
:10149000204600F051FA2046FFF7FEF9286B30B1E4
:1014A0000368D4EDD20ADB6894EDD10A9847D4F8EA
:1014B000100208B153F0A0FF204600F07DF820464E
:1014C000FFF744F994F8903284F80C0383420ED06D
:1014D00084F8900298B10C4D0C4B032808BF1D46B0
:1014E0003DF0E8FA0A4A2B46062136F0F3FC204686
:1014F000FFF728FF01A811F0DBF903B030BD054D5F
:10150000EEE700BFCC250020DFB8080893E5080807
:10151000B4E5080898E50808D0EDDE7A9FED057A75
:10152000F4EEC77AF1EE10FAB7EE000AA8BFB0EEFB
:10153000670A704700000034014B1868704700BF0D
:10154000285A00204FF0FF307047000001207047FC
:10155000704700000020704700207047704700006F
:10156000704700000020704700207047002070473F
:10157000002070470020704700207047002070470F
:10158000012070470368D3F8943018470020704753
:1015900000207047002070470020704700207047EF
:1015A00000207047002070470020704700207047DF
:1015B00000207047704700007047000008B513F026
:1015C000D7FF90F8130308BD08B513F0D1FF90F8CA
:1015D000120308BD30B52DED028B9FED1A1ADFED19
:1015E0001A0A91ED000A87B005462D200C468DEDB4
:1015F000011ACDED000A14F0B9FC9DED011ADDEDE4
:10160000000AF0EE408A2E2094ED010A14F0AEFCA0
:101610009DED011ADDED000AB0EE408A2F2094ED19
:10162000020A14F0A3FC03A905F52570CDED038A89
:101630008DED048A8DED050A31F0FCFB07B0BDECA1
:10164000028B30BDC2B8323EC2B832BE10B50446BD
:1016500052F064FFD4F8F4321BB1C21AB2F57A7FAB
:1016600012D30A4A1268D26A92F89C2002B15BB97E
:10167000C4F8F40294F8314213F07AFF80F80D4375
:1016800005F02AF880F8254010BD00BFCC250020C9
:101690002DE9F0432DED028B91ED007AD1ED037A27
:1016A00087B08DED047AB0EEC77AB5EEC07AF1EE70
:1016B00010FADDE91087DDF84C90CDED057A0C4687
:1016C00015461E4606DCF0EEE77AF5EEC07AF1EE3E
:1016D00010FA02DD04A816F0EBFB6B20B7EE001A3F
:1016E000FFEE000A9DED050A14F040FC6C2089ED28
:1016F000000AB7EE001AFFEE000A9DED040A14F08E
:1017000035FC04A888ED000A16F05AFBB7EE008AF3
:10171000002852D00023C9F8003088ED008AD4EDAB
:10172000067A67EEA77AF4EEC87AF1EE10FA4ADB91
:101730000023336085ED008ADFED3F0A96ED000A55
:101740007C20B7EE001A14F011FC86ED000A95ED2E
:10175000000A7D20B7EE001AFFEE000A14F006FC26
:1017600085ED000AD4ED067A129BDFED346AF1EEC6
:10177000677AC3ED007A96ED007AF0EEC77AF4EE60
:10178000E67AF1EE10FA2BD503AB02AA01A92046A6
:1017900015F010F89DED018AB0EE480A72F0CAF912
:1017A00085ED000AB0EE480A72F01AFB87ED000AD8
:1017B00007B0BDEC028BBDE8F08304A816F0ECFA8C
:1017C0000028A7D1ABE738EE670A14F001FB86EDDD
:1017D000000A94ED087AC7EE007AC5ED007AABE70F
:1017E00094ED076AC6EE077AC7ED007A96ED007AA7
:1017F000B0EEC77AB4EEE67AF1EE10FAC4D495ED05
:10180000007ADFED0F6AB0EEC76AB4EE666AF1EEF9
:1018100010FAB9DCB4EE477AF1EE10FAB4D6B0EEB5
:10182000E77AB4EE667AF1EE10FAADDCF4EE677AA0
:10183000F1EE10FABCD7A7E700000000000000346A
:10184000FFFF7F7F1FB500F51773039300F5167335
:10185000029300F51573019300F51473009300F5DE
:10186000127200F5137300F54871FFF711FF05B010
:101870005DF804FB9FED156A90ED817ADFED146A47
:10188000D0ED837A27EE067A67EE867A27EE267AFF
:1018900067EEA67ABDEEC77AFDEEE77A80ED7E7A36
:1018A00090ED827A27EE067A17EE903A27EE267AA6
:1018B000002BB8BF03F50C43BDEEC77AB8BFA03309
:1018C00080ED7F7AC0F80032704700BFE02E65429D
:1018D0000000C8421FB50E4B1B680446B3B16846F2
:1018E00003F0D6FE69462046FFF72CFC20B16A467D
:1018F00000212046FEF7A6FA94F87C32DB0705D5D6
:1019000004F51B7201212046FEF79CFA04B010BDBD
:10191000D45C002008B502F0E1F9BDE8084001F010
:101920006FBD000010B580F8F812044652F0F6FDC5
:10193000C4F8FC0210BD000010B590F8F83204465F
:1019400053B152F0EBFDD4F8FC32C01AB0F57A7FF7
:1019500084BF002384F8F83294F8003353B152F076
:10196000DDFDD4F80433C01AB0F57A7F84BF0023BC
:1019700084F8003310BD000000F5AA700B4607C8BC
:1019800083E80700012070470023C0F89C30C0F8AE
:101990009830C0F89430C0F8A830C0F8A430C0F82F
:1019A000A030C0F8AC30704770470000024B0B60AD
:1019B0004FF07C53136070470000484270470000AE
:1019C00008B50B4600F12801184615F05DFD012011
:1019D00008BD000010B500F5B4700C460FC884E8CF
:1019E0000F00204603F044FE30B1FFF7A5FD00F5DF
:1019F0001B700FC884E80F00204603F039FE80F00A
:101A00000100C0B210BD000010B5044604F0E4F8B7
:101A1000204610BD10B5D0F8603104465BB152F0DD
:101A20007DFDD4F86031C01A41F28833984294BFEA
:101A30000020012010BD0120FCE7000013B5009339
:101A400003680192D3F890309847DDE900210446FD
:101A500028B90448044B0068C06A11F0E5F8204634
:101A600002B010BDCC250020D4E6080813B504460A
:101A70000191FEF701F92368019A1B6D014608B137
:101A800090F84E11204602B0BDE810401847000003
:101A900030B585B0002301930293039303680D468C
:101AA000DB6D01A99847044620B1039B2B602046BB
:101AB00005B030BD02F012F9417C01F0DDFD0446B5
:101AC0000028F4D002F00AF901F03CFDB1EE400A22
:101AD00085ED000AEBE7000090ED007ADFED0F7A6C
:101AE000B0EEC77AB4EEE77AF1EE10FA14D590EDC5
:101AF000017AB0EEC77AB4EEE77AF1EE10FA0BD5C0
:101B000090ED027AB0EEC77AB4EEE77AF1EE10FA11
:101B10004CBF0120002070470020704700000034B7
:101B200010B5FEF7A9F8044658B190F84E11FEF72B
:101B300075F830B194F84E112046BDE81040FEF71C
:101B400071B8002010BD000038B50D460DF084F9C5
:101B50000446FEF709FA022881BF94F8C402B023B4
:101B600003FB0040D43089BF07C8002085E8070088
:101B7000012038BD2DE9F0432DED028B8FB00368B5
:101B80000025DB6C0395049505950695029502A941
:101B900004469847064638B1FFF7BCFEDDED027AF1
:101BA00027EE800A8DED020A0DF056F9FEF7DCF9FA
:101BB0000746002E50D0DDED027AD4ED646A94ED34
:101BC000657A23680B9527EE877A67EEA67A8DED06
:101BD000097ACDED0A7A0C950D959B6C0BA92046E0
:101BE00009AD98470BA9284616F060F8012F8DED36
:101BF000030ACDED040A40F2B3800DF02DF990F800
:101C0000C432DFED5B7AB02505FB030090ED308A2E
:101C100028EE278AB0EE480A71F08CFFF0EE408A79
:101C2000B0EE480A72F0DCF8CDED0B8A8DED0C0AAF
:101C30000DF012F990F8C43205FB030090ED2F0A65
:101C40000BA816F053F809AD8DED050ACDED060A87
:101C500005A896BB03C885E00128CED89DED020AF1
:101C6000B5EEC00AF1EE10FA7FDD07AED4F894218C
:101C7000D4F8903107923046089316F055F823684F
:101C80000B950C950D959B6C0BA920469847DDEDA7
:101C9000077A9DED0B7A77EE877A9DED0C7ACDED84
:101CA000077ADDED087A77EE877A09ABCDED087A11
:101CB00096E8030083E8030049E0236993ED000AF6
:101CC000B7EE008A38EE408A16F010F804F5BC79B9
:101CD0008DED090A4846B0EE480ACDED0A0A16F025
:101CE00005F80BA92846CDED0C0A8DED0B0A15F071
:101CF000DDFF04F5C47603AFC4ED5F0A314684ED21
:101D00005E0A384615F0E2FF04F5C0788DED090A49
:101D10004046B0EE480ACDED0A0A15F0E7FF0BA9E0
:101D200028468DED0B0ACDED0C0A15F0BFFF97E8A4
:101D3000030084ED600AC4ED610A86E803004946A9
:101D4000404615F0B3FF8DED090ACDED0A0A9DED71
:101D5000090ADDED0A0A0FB0BDEC028BBDE8F08385
:101D6000DDE9030185E80300F1E709950A95EEE74F
:101D700035FA8E3C10B590F84213044604F0C6F8CC
:101D80007C23C0B203FB0044D4F8A00010BD0000C7
:101D9000044B026F1B68DB6A5A60426F9A60826F65
:101DA000DA607047CC250020F0B58FB0044613F000
:101DB000DFFB002302930393049390F8121301AB0B
:101DC00002AA054612F008FC04F19407D8B39DED71
:101DD000010AB5EEC00AF1EE10FA34DD02A816F0E1
:101DE000FBF804F1B00684ED2C0AC4ED2D0A84ED55
:101DF0002E1A3946304616F0FFF804F17C013046C1
:101E000016F0AEF804F1880105A88DED050ACDEDB8
:101E1000060A8DED071A16F0A3F808A88DED080A3A
:101E20009DED010ACDED090A8DED0A1A16F0C4F8F0
:101E30000BA904F128008DED0B0ACDED0C0A8DEDF8
:101E40000D1A14F063FD95F812030C2303FB0050E8
:101E5000394600F5117016F083F884ED2C0AC4EDB4
:101E60002D0A84ED2E1A0FB0F0BD00002DE9F047C9
:101E7000824B00251F682DED028BC0F89C50C0F8E6
:101E80009850C0F89450C0F88450C0F88050C5678E
:101E9000C0F89050C0F88C50C0F88850C0F8B850C6
:101EA000C0F8B450C0F8B0500446F86A03688AB06D
:101EB0005B680E46984704F12809002854D052F078
:101EC0002DFB42F20F7398424ED8FB6A9FED6C8A4D
:101ED00093ED010A84ED1C0AD3ED020AC4ED1D0A3C
:101EE00093ED031A484684ED1E1A14F003FC3CF0EF
:101EF000E1FDD4ED1E7A67EE887A054617EE900A6A
:101F0000FAF7FAFAD4ED1D7A67EE887ACDE9040182
:101F100017EE900AFAF7F0FAD4ED1C7A67EE887A99
:101F2000CDE9020117EE900AFAF7E6FA554ACDE933
:101F300000010621284635F0CDFF94ED1E8AB0EE53
:101F4000480A71F0F7FD84ED650AB0EE480A71F0B9
:101F500047FF84ED640A52F0E1FAC4F864010AB064
:101F6000BDEC028BBDE8F087A6B194ED1C0AB4EE7F
:101F7000400AF1EE10FA0DD6D4ED1D0AF4EE600A17
:101F8000F1EE10FA06D694ED1E1AB4EE411AF1EEF7
:101F900010FA52D713F0ECFA90F813334FF00C0A02
:101FA0000AFB030303F5C473074693E8070007AE73
:101FB00086E807004FF01508B2EE028AF2EE068AB4
:101FC000304616F0F7FBB4EEC80AF1EE10FA38D539
:101FD00008F1FF3818F0FF083CD1304616F0EAFB54
:101FE000F1EE047AB4EEE70AF1EE10FA43DD9DED6E
:101FF000090ADDED087A9DED078A20EE000AA7EEBA
:10200000A70A72F003F9F0EE400AB0EE480A71F048
:10201000B3FFDDED090A84ED1D0A9DED080AF1EE1E
:10202000600AB1EE400A71F0A7FF84ED1C0A9FED33
:10203000161AD4ED1D0A94ED1C0A484614F05AFBFA
:102040007BE7304616F0B6FBB4EEE80AF1EE10FA84
:10205000BEDCC2E7384612F081F9384612F046FA83
:1020600097F813330AFB037303F5C47393E807006F
:1020700086E80700A4E725676567D8E7CC25002038
:10208000E02E6542E0E60808000000000021FFF7AE
:10209000EDBE000037B5044608461546019116F01E
:1020A00089FBB7EE007AC7EE007AB4F8D030019819
:1020B0000133A4F8D03094ED337A37EE277A84EDEB
:1020C000337AB0EE007AF4EEC77AF1EE10FA06D564
:1020D000B6EE007AF4EEC77AF1EE10FA0DDC9FED61
:1020E0000E7AF4EEC77AF1EE10FA13D59FED0B7A63
:1020F000F4EEC77AF1EE10FA0CDDB0EE670A15F0D7
:102100005BFF012085ED000AC5ED010A85ED021A8D
:1021100003B030BD0020FBE700247449BD3786358D
:1021200070B52DED028B00F1280600F134058AB060
:1021300029460446304615F0BBFFB6EE008A20EE75
:10214000088A2846B0EE480A15F036FF07A930463F
:10215000CDED080A8DED091A8DED070A15F016FF71
:1021600030468DED010AB0EE480ACDED020A8DED44
:10217000031A15F021FF07A928468DED070ACDEDBA
:10218000080A8DED091A15F001FF04A901A88DEDCB
:10219000040ACDED050A8DED061A15F09DFF3246B5
:1021A00001A920468DED070ACDED080A8DED091A2B
:1021B000FFF770FF58B952F0B1F90121C4F860017E
:1021C0002046FFF753FE0AB0BDEC028B70BD2A46D5
:1021D00004A92046FFF75EFF0028ECD004F140027E
:1021E00007A92046FFF756FF0028E4D0EBE70000E0
:1021F00030B52DED028B0D4683B091F842130446A5
:10220000284603F083FEC1B27C2000FB01519031CF
:1022100004F1280014F0FEF868468DED000ACDEDBB
:10222000010A15F0F3FDDFED1C7AB4EEE70AF1EEDA
:1022300010FA05D59FED190A03B0BDEC028B30BD35
:10224000684615F035FE684615F0BAFD0028F1D154
:10225000284694ED428A03F0CDFFF0EE400AB0EE3E
:10226000480A13F081FD80B9284603F0C3FF84EDCE
:10227000420AB0EE408A71F05DFC84ED430AB0EE94
:10228000480A71F0ADFD84ED440A04F58671684694
:1022900015F074FDD0E700BF00000034000000001E
:1022A0009FED0C7AB4EEC70AF1EE10FA0BD4DFED15
:1022B0000A7AB4EEE70AF1EE10FA07DCC0EE077A0C
:1022C000B0EE670A7047F7EE007AF9E7F2EE047AAB
:1022D000F6E700BFF3665F3F58A00B4108B51C301E
:1022E00015F094FDF1EE007AB4EEE70AF1EE10FA83
:1022F0009DBFF1EE027A37EEC00ADFED047A9FED62
:10230000040A98BF20EE270A08BD00BFCDCC4C3E82
:10231000CDCCCC3D08B5836993F9000038B10CF001
:102320009BFDFDF721FE012894BF0020012008BD80
:10233000F8B52DED028B054604F0CEF904F0CAF88D
:102340000446B8B3FFF7F8F890F8093393B328467A
:10235000FFF7E0FF064668B30CF07EFD90F8C4324C
:10236000B02707FB030090ED2F7AF0EE087AB4EE69
:10237000E77AF1EE10FA1DD495ED1E8A0CF06CFD93
:1023800090F8C432DFED1E7A07FB030090ED300AAF
:1023900098EE270A13F06CFDDFED1A7AB0EEC00A52
:1023A000B4EEE70AF1EE10FA08DC52F0B7F8344662
:1023B000C5F85001BDEC028B2046F8BD05F5AA70AA
:1023C00016F0F8F9B0EE408A0CF046FD90F8C432F1
:1023D0009FED0D7A07FB0303D3ED2F7A67EE877A23
:1023E000B4EEE78AF1EE10FADFD552F097F8D5F89F
:1023F0005041001BB0F5FA6F8CBF00240124D9E7CF
:10240000E02E654200003442CDCC4C3F10B50A4B63
:102410001B68DB6A93F89C3004465BB952F07EF887
:10242000D4F86431C01A44F61F6398428CBF002070
:10243000012010BD0020FCE7CC250020F8B52DEDD3
:10244000068B04460CF008FD054604F045F90646E7
:1024500006F02EFE002840F0AA802046FFF768FF15
:10246000002800F0A7803046FFF784FCD4F8DC3069
:10247000984200F018813046FFF77CFCD4F8DC303D
:10248000DFED8E7AC31A08EE903AF8EE688A30468D
:1024900068EEA78AFFF76EFC94F8BC30C4F8DC0045
:1024A000F3B9304604F028F8D0B104F1280796F8C3
:1024B00042233946304603F0A1FED4ED1D0AB0EEAA
:1024C000401A384694ED1C0A14F014F90023C4F89D
:1024D0009030C4F88C30C4F88830012384F8BC30C4
:1024E00020463146FFF784FE95F8C40205EB00153F
:1024F000B0EE408A2B6FC4F8E03004F1B000D4EDA8
:10250000129A16F057F96368DFED6D7A93ED007A51
:10251000B4EEE77AF1EE10FA68EE299AB0EE40AA2E
:1025200001D5C3ED007A2046B0EE4A0AFFF7B8FEA7
:10253000636820EE299A93ED000A29EE009AFFF7CE
:10254000CDFE29EE009A204684ED249AFFF75EFF27
:1025500038B1D4ED247AB2EE007A67EE877AC4ED12
:10256000247AF0EE007AF4EEE78AF1EE10FA10D554
:10257000DFED547AB4EEE7AAF1EE10FA09D5DFEDFB
:10258000527A69EEA79AD4ED2A7AE9EEA87AC4EDD8
:102590002A7A9FED4E0A94ED367ADFED4D7AB0EE51
:1025A000C88A28EE008AA7EE278A84ED368ABDEC19
:1025B000068BF8BDFEF7C0FF90F80933002B72D0F0
:1025C0002046FFF7A7FE00286DD095F8C42205EB42
:1025D0000213196FD4F8E0308B4264D0B02606FBAA
:1025E000025292ED2F7AF0EE087AB4EEE77AF1EE2D
:1025F00010FA58DBCB1AC4F8E01008EE903A95F8C0
:10260000C4329FED341A94ED1E0ADFED337A06FBD7
:102610000353D3ED309A69EE819AF8EE688A39EE69
:10262000C00A68EEA78A13F08DFCB0EE409A71F0F4
:10263000D7FB94F8BC30B0EE408AF3B1F3EE047AE5
:10264000F4EEE78AF1EE10FA17DC95F8C40206FB07
:10265000005595ED2F7AF2EE027AB4EEE77AF1EEBC
:1026600010FAFFF64AAFDFED1D7AB0EEC99AB4EE6C
:10267000E79AF1EE10FAFFF640AF9FED198AD4ED1C
:102680001D0A94ED1C0AB0EE691A04F1280014F03A
:1026900031F8012384ED248A84ED238A84ED228A93
:1026A00084F8BC3029E7BDEC068B04F188009FED6F
:1026B0000D0ABDE8F84015F0D3BC00BFBD37863524
:1026C000CDCC4C3DC2B8B23E0AD7233CCDCC4C3E1B
:1026D000CDCC4C3F35FA8E3C6F12833A1904863FBD
:1026E00000000000EC51783F30B50C2303FB0101E2
:1026F00001F1C003144693E807008BB004AD85E8F0
:10270000070094E8070083E807002846FFF7E4F98C
:1027100007AB58B194E8070083E807009DED070A6E
:10272000DDED080A9DED091A0BB030BD95E80700F4
:10273000F2E70000F0B52DED028BD0F818318B6078
:10274000D0F81C31CB6085B004460D4601F0C6FAC6
:1027500006460CF081FBA36993F90030022B074673
:102760004BD1FDF701FC022847D997F8C432B022BB
:1027700002FB0373D3F8B0100022284602F08EFF4C
:10278000D4ED4A0A94ED490A284603F011FA94F868
:102790002C3163B351F0C2FE9FED228A97F8C41228
:1027A0008DED018A01AA064638460BF0D9FBD4F814
:1027B00020019FED1D0A361A07EE906AF8EE677A3F
:1027C0004FF4876027EE800AB6EE001AF0EE480A52
:1027D00013F0CCFBDDED017A30EE270A04F1F000B6
:1027E0008DED010A15F082FA284603F0E1F994F81C
:1027F0002C0105B0BDEC028BF0BD707C242303FBE3
:10280000006696ED0B8AFEF797FED0ED9C7A9FED61
:10281000077AF8EEE77AE8EE077AFDEEE77A17EE48
:10282000901AA9E7000000006F12833A0000C84226
:10283000F8B5036F0B60436F4B60836F8B6000F1E3
:102840004C050E46074601F10C040FCD0FC40FCD09
:102850000FC42B68236007F1B00207CA06F13003EA
:1028600083E8070007F1940207CA06F13C0383E8F6
:10287000070007F11C0207CA06F1480383E80700B6
:1028800006F160013846FFF755FF86F87000F8BD85
:1028900030B589B0044668460D4602F0F9FE694637
:1028A0002046FFF797F818B90024204609B030BD3C
:1028B00004A802F0EDFE204604A9FFF73BFF044602
:1028C0000028F1D004A9684603F0CAF885ED000A93
:1028D000C5ED010A85ED021AE7E700001FB50023E8
:1028E0000C4601A9019302930393FFF7D1FF08B1AE
:1028F000039B236004B010BD30B585B001AD00234B
:102900000C462946019302930393FFF7C1FF034648
:1029100018B195E8030084E80300184605B030BDFF
:10292000F8B506460F461546FDF7A6F9044690B1E0
:102930003946FDF773F970B120463946FDF772F953
:10294000044640B1FDF798F93946FDF76DF985ED7C
:10295000000A2046F8BDFEF7EFFD90F8083343B1BA
:102960003046FFF7D7FC044618B1D6F84C312B603F
:10297000EFE7D6F84C312B600024EAE770B52DED77
:10298000048B1646FFF7CCFF054670B3FEF7D4FD67
:1029900090F930424CB30CF05FFAFDF7E5FA0128EC
:1029A00023D9E4B207EE904AB8EE678A0CF054FAE5
:1029B00090F8C43296ED009AB02202FB0300D0EDED
:1029C0002F8AFEF7A7FF38EE281A78EEC80A40F2E1
:1029D000614029EE000A13F0C9FAB0EE408AFEF712
:1029E00099FFC8EE007AC6ED007ABDEC048B28464C
:1029F00070BD000008B503F06FFEBDE8084003F0AD
:102A000069BD000010B5044615F082FB50B904F111
:102A10000C0015F07DFB28B904F11800BDE810404A
:102A200015F076BB012010BD38B500F1280504462D
:102A30002846FFF7E7FF28B120460121BDE83840CE
:102A4000FFF714BAD4ED107AB7EE007AF4EEC77A35
:102A5000F1EE10FA06D5BFEE007AF4EEC77AF1EE89
:102A600010FA12DC2046FFF75BFB2846FFF7CAFF8F
:102A70000028E1D1D4ED107AB2EE047AF0EEE77AD4
:102A8000F4EEC77AF1EE10FAD6DC38BD10B5044684
:102A900015F090FE2046BDE8104015F0F5BA000094
:102AA0002DE9F04F2DED048B9FEDC48A95B00446BF
:102AB000F0EE408A8DED028A8DED038A8DED048A59
:102AC000FFF7BCFC12F054FD0023054695F8792170
:102AD000012AA8BF012293423FD20021284611F0CB
:102AE000A9FB01230028F1D008AB0BAA002128463E
:102AF0008DED0B8A8DED0C8A8DED0D8A11F0C6FDE2
:102B00009DED080AB5EEC00AF1EE10FA23DD0BA820
:102B100015F062FA11A904F128008DED110ACDED2E
:102B2000120A8DED131A13F019FC0EA88DED0E0A82
:102B3000B0EE680ACDED0F0A8DED101A15F03CFAD3
:102B400011A904F1E4008DED110ACDED120A8DED0D
:102B5000131A15F051FA0123B8E795F813130C2353
:102B600003FB015104F1280B01F5C471584613F021
:102B7000F5FB84ED070A94ED3F0AC4ED080A70EEF8
:102B8000288A84ED091AC4ED3F8A0CF065F90646DF
:102B9000FEF7D2FC90F8093300932046FFF7BAFB0A
:102BA00080B13046FDF7E0F902280BD996F8C4222F
:102BB0006169B02303FB026391F9001093F8D2001E
:102BC00088425FDA94ED3F7ADFED7D7AB4EEE77A02
:102BD000F1EE10FA5DD4D4ED538AFEF7A1FF38B1BF
:102BE000FDF74AF890F84E11FDF71EF8F0EE408A16
:102BF000236C626BA16A1393B0EE680A11A812925B
:102C0000119115F0D9F904F5AA7102A88DED020A07
:102C1000CDED030A8DED041A15F0EEF951F07EFCAE
:102C20000023074684F814312046FFF773FB002881
:102C300065D096F8C422B02302FB033232445268B6
:102C4000C4F8182196F8C42202FB033333449B686E
:102C5000C4F81C3151F062FC0123C4F8200184ED5A
:102C6000498A84ED4A8A84F82C31D4F80031002B4B
:102C700058D102AB93E80700C4F80071F03484E83F
:102C8000070006E006EB0212176FD4F80021BA42E3
:102C900004D115B0BDEC048BBDE8F08FD43393E8BC
:102CA000070094F814310DF1080C8CE807001BB9EB
:102CB00004F1F00383E807000123604684F814312F
:102CC00004F5AA7115F062F911A904F14C008DED1B
:102CD000110ACDED120A8DED131A13F06DFBB5EE4E
:102CE000C00AF1EE10FA8DED110AD8BF9FED330A3C
:102CF000CDED120A8DED131A84ED530A94E794ED8D
:102D00003F7AD4ED497ADDED026AE6EE877ADDEDB1
:102D1000036AC4ED497AD4ED4A7AE7EE267AC4ED27
:102D20004A7AA2E7D4ED3F7A224B8DED058AF5EE83
:102D3000C07AF1EE10FA8DED068A0793A9D99FEDBE
:102D40001E7A94F8143167EE877AB7EE007AC7EEF0
:102D5000279A1BB9009B002B00F0AA80E36804F1BE
:102D6000F00102A8D3ED008A15F010F969EEA88AE7
:102D70008DED110A11A8B0EE680ACDED120A8DEDA5
:102D8000131A15F019F90EA905A88DED0E0ACDED4F
:102D90000F0A8DED101A15F02FF905A8FFF776FE32
:102DA00005A815F0CFF9D8B151F0B8FBC4F860010F
:102DB0006FE700BF000080BF0AE81C410000000070
:102DC000CDCC4C3ECDCC4C3FCDCC4C3D920A06BF39
:102DD000920A063FC2B8B23E728A0E3C5B82183934
:102DE000012301930023CDE90833CDE90A33CDE96E
:102DF0000C335FED0E8A4FF0FF3A04F1E40895F8CA
:102E00007921012A1046A8BF0120834257D201230D
:102E1000002AFAD095F835130029F6D0B0EE690AE9
:102E2000404615F01DF9019B0DF12C09002B41D0F6
:102E3000424600212046FFF757FC8DED0B0ACDEDF1
:102E40000C0A8DED0D1A4846FEF746FE70BB48464B
:102E5000FFF71CFE484615F075F938BB05A9484632
:102E600015F03AF9484605A98DED080ACDED090A95
:102E70008DED0A1A15F01CF908A8B0EE409A15F06D
:102E800099FCBAF1000F06D1F4EEC08AF1EE10FA07
:102E9000D8BFB0EE680AB5EEC09AF1EE10FAF7EEC0
:102EA000008A58BFF0EE408A4FF0000A0123A6E7DF
:102EB000009B96E798E8070089E80700C3E7BAF1A6
:102EC000000F7FF471AF002384F804312046FFF730
:102ED0002FFA38B12046FFF71DFA002840F025816F
:102EE0008DED0A8A95F8123395F878219A4240F2CE
:102EF00033812B4493F83433002B00F02D8195F867
:102F0000133395F879219A4240F226812B4493F8A5
:102F10003533002B00F0208108A9584613F04CFAF5
:102F20008DED080ACDED090A8DED0A1A08A815F0F5
:102F3000EFF8002840F0178108A815F003F90028E1
:102F400040F011815FED627A94ED357A68EEA78AE0
:102F50005FED647AE7EE278A04F1B000C4ED358AAC
:102F600015F028FCA3685FED687A93ED007AB4EE63
:102F7000E77AF1EE10FAF0EE408A00F1F880204690
:102F8000B0EE680AFFF78CF908A815F015F8A368E9
:102F90008DED110ACDED120A8DED131A93ED000A95
:102FA00011A815F009F8204684ED1F0AC4ED200A87
:102FB00084ED211AFFF72AFA28B1B2EE000A04F1D3
:102FC0007C0015F04DF8009BB3B33046FCF7CCFF06
:102FD000012831D996F8C402B02303FB006696EDB0
:102FE0002F7AF0EE087AB4EEE77AF1EE10FA23D5F4
:102FF00095F813030C2303FB005595ED627AF1EE6F
:103000000C7AB4EEE77AF1EE10FA15DBD4ED1D7A06
:103010001FED927AF4EEC77AF1EE10FA0CDD1FED97
:10302000947AF4EEC77AF1EE10FA05D5B6EE000AFE
:1030300004F17C0015F014F85FED9A7AF4EEE78A5B
:10304000F1EE10FA22D51FED9C0A08A814F0B4FF87
:103050000EA88DED0E0A94ED3F0ACDED0F0A8DED11
:10306000101A14F0A9FF11A904F1A0008DED110AA6
:10307000CDED120A8DED131A14F0BEFFD4ED2B7AAC
:1030800094ED3F7A77EE877AC4ED2B7A94ED2B7A24
:10309000F1EE047AB4EEE77AF1EE10FA3BDB12F0CF
:1030A00067FA5FEDB27A94ED2B1A94ED280A21EEBF
:1030B000271A40F2C530F1EE410A8DED011ACDED2F
:1030C000000A12F053FF9DED011ADDED000A84EDB8
:1030D000280A40F2C63094ED290A12F047FF9DED10
:1030E000011ADDED000A84ED290A40F2C73094EDA3
:1030F0002A0A12F03BFF04F1A00184ED2A0A04F130
:10310000940014F079FF84ED2A8A84ED298A84EDF5
:10311000288A84ED2B8A0023C4F8E430C4F8E83010
:10312000C4F8EC3084ED3F8AA3E5E368F7EE000ACB
:1031300093ED000A12F018FE00283FF4D1AE94ED92
:103140001C0AB0EEC00A70F04BFEDDED0A7A27EEE5
:10315000800A8DED0A0AC5E68DED0A8A8DED098A91
:103160008DED088AE2E62046FFF75EFC1CE6C3ED23
:10317000007A04E72DE9F04D2DED048B9EB0044656
:1031800012F0F6F9D0EDC87A90ED618AF4EE487A43
:10319000F1EE10FA48BFB0EE678ADFED5C7AB4EE6C
:1031A000E78AF1EE10FA0EDD0023C4F8E430C4F82B
:1031B000E830C4F8EC300023C4F8FC301EB0BDEC9D
:1031C000048BBDE8F08D2046FEF7EEFD2046FEF7AD
:1031D000A7FFB0EE480A2046FFF762FC2046FFF743
:1031E00023FCFEF7A9F914AD00F5347204F12801AF
:1031F00014A813F031F90FCD04F14C060FC60FCD12
:103200000FC62B68336004F1740204F1780304F1F3
:10321000700104F14C0013F0CDFA94ED1E8AB0EE6B
:10322000480A70F087FC84ED650AB0EE480A70F039
:10323000D7FD204684ED640AFEF7AAFDFEF77CF96F
:1032400004F5B471FDF77EFF51F068F9D4F89831B8
:10325000C31A632BB2D9C4F8980132F03BFF9FED3B
:103260002C9A054651F062F9D4ED1C7A67EE897A02
:10327000074617EE900A0E46F9F73EF9D4ED1D7A8F
:1032800067EE897A824617EE900A8B46F9F734F991
:1032900094ED1E0A20EE090A41EC180B12F0D2FD43
:1032A000D4F85C0110EE108AF9F726F9CDE9120185
:1032B000D4F85801F9F720F9CDE91001D4F85401F8
:1032C000F9F71AF9CDE90E01D4F8D800F9F714F995
:1032D000CDE90C01D4F8D400F9F70EF9CDE90A01D3
:1032E0004046F9F709F90B4B01930B4B0093CDE9DD
:1032F00008018DED068BCDE904ABCDE90276074BD5
:10330000074A0849284632F071FC57E7CDCC4C3EBD
:10331000E02E654245E708084FE708080CE7080873
:1033200016E7080898E5080808B52DED048BB0EEFF
:10333000609AF0EE408A00F011F9B0EE408A89EE12
:10334000280A70F083FEDFED0B7A20EE270A70F07A
:1033500015FEDFED097A38EE278ADFED087A28EED0
:10336000278AF7EE007A37EEC00A28EE000ABDEC95
:10337000048B08BD41D3423E33938843A1D81943FF
:10338000FFF7D2BF08B52DED048B9FED189AF0EE34
:10339000E07AF4EEC97AF1EE10FAF0EE408AB0EE7F
:1033A000608A1ED400F0DAF8DFED117A9FED117A11
:1033B00070EE277A9FED100AE8EEC77A9FED0F7A3C
:1033C00027EE800AC8EE007A87EE270AB4EEC90A13
:1033D000F1EE10FA05DBBDEC048BBDE8084070F09F
:1033E00015BFBDEC048BB7EE000A08BD0000003429
:1033F00033938843F4FDD43B48A18F43CDCC9C3F0D
:10340000427CD0ED257A242101FB020292ED0B0AC9
:10341000D2ED090A30EE270AFFF7B4BF38B52DED1B
:10342000088BDFED21AA9FED21AA9FED21BA054669
:10343000B0EE409AF0EE609AB0EE408A1524013C5E
:10344000A4B25CB3F0EE490A2846B0EE480AFFF792
:103450006BFFF0EE490A70EE698A284638EE2A0AB8
:10346000FFF762FFB0EEE87A70EE697AB4EECA7ADE
:10347000F1EE10FA77EEE87A10D468EEAA8A40F2FC
:10348000631088EEA70AB0EE4B1A38EE400AF0EE51
:103490004A0A12F06BFDB0EE408AD0E7B0EE480A5F
:1034A000BDEC088B38BD00BFCDCCCC3D0AD7233C4A
:1034B00000247449002343608360C3600361436157
:1034C0008361C361002380F82030704790F820208A
:1034D000531CDBB2062B80F8203000EB820288BF41
:1034E000002382ED010A88BF80F820307047000079
:1034F0004FF0FF3310B543610E4BC0F8A8300023E6
:10350000044680F8C830A830FFF7D4FF0A4BC4F84F
:10351000A83004F5867050F05FF9084B08491C602C
:1035200020462EF0ABFDD4F89030C4F894302046FD
:1035300010BD00BF6CE908087CE908082C5A00207F
:1035400014EA080808B5A83033F0F6FDDFED027A7A
:1035500020EE270A08BD00BF00007A4490ED3C0A27
:10356000DFED057AB0EEC07AB4EEE77AF1EE10FA4C
:1035700048BF90ED3D0A70470000003473B5D0F8A5
:10358000A43004460E4663B150F0C8FFD4F8A4300E
:10359000C01A42F20F73984203D894ED280A02B081
:1035A00070BD114B1D687DB195F84E112846FCF792
:1035B00039FB48B195F84E1101AA2846FCF728FBC3
:1035C00010B19DED010AEAE7242101FB064494EDC8
:1035D0000A0ADFED067AB4EEE70AF1EE10FA58BFF8
:1035E000B0EE670ADBE700BF245A002000000C425F
:1035F00008B561B10378022B02D9064850F05EFF8E
:103600005A1C027000EB83004160012008BD08468F
:10361000FCE700BF34E808082DE9F84305460E46EC
:103620009146002400F13C082B78A34211DD0023D1
:103630004A46314601200EF08DFF2423634307469E
:10364000002158F803000EF095FF874204D00134A2
:10365000EAE70020BDE8F8830120FBE7054B1B6883
:103660002BB141694A1C02D0184632F0FDBC002043
:10367000704700BFD45C002002290BD8242303FB31
:10368000010191F8390030B191F83A0018B191F880
:103690003B007047002070472DE9F047044650F08A
:1036A0003DFFD4F8F86042F21073861B9E4288BF3B
:1036B000C4F8F80000274FF0240942F2107A237C66
:1036C000FDB2AB421CD929462046FFF7D5FF70B1A9
:1036D00009FB054898ED0D0AD8ED097AD4ED250AC5
:1036E00030EE270A2046FFF799FE88ED0C0A564572
:1036F00004D909FB054030302EF098FE0137DEE793
:10370000617C2046FFF73AFF84ED3D0ABDE8F08773
:1037100070B5044686B050F001FFD4F89830C31A53
:10372000B3F57A7F05464FD3344B94ED257A1B6869
:10373000DFED336ADB6AD4ED247A93F89C60B0EE57
:10374000C76AB4EEE66AF1EE10FA32D5B0EEE76A77
:10375000B4EEE66AF1EE10FA2BD502A801F098FF5C
:1037600096BBFDF7E9FE02A9FDF7ECFC60B3DDEDC9
:10377000037A9FED247AF8EEE77A67EE877AC4ED54
:10378000257AC4F89850FDF7D7FEFDF7C3FA204616
:10379000FFF782FF3BF08EF90546D4F89400F8F766
:1037A000ABFE194ACDE900010621284634F092FB10
:1037B0000AE037EE676AF7EE005AB0EEC66AB4EE7A
:1037C000E56AF1EE10FA01DC06B070BDB0EEE76A12
:1037D000B4EEE66AF1EE10FAF6D4002ECFD0204611
:1037E000903080ED007A2EF021FE3BF063F9074A1D
:1037F000012106B0BDE8704034F06CBBCC25002040
:10380000000000340AD7233C75E8080850E808088F
:10381000F0B52DED048B85B004464FF4537200F5DE
:10382000867103A80FF022F8D4ED227AD4ED236A32
:103830009FED796A637C37EEE67A2422B0EEC77A90
:10384000B4EEC67AF1EE10FAC1BF9FED747A67EE5E
:10385000877A9FED737AE6EE877A02FB03430025B1
:10386000C4ED237A93F839602378E9B28B4206D904
:1038700004EB81030135586851F0B0FEF4E7DFED49
:10388000698A9FED698A9FED699A0027237CFDB2C2
:10389000AB4264D9242303FB054393F83920002A63
:1038A0005BD0D3ED0C7AF4EEE87AF1EE10FA0BDB94
:1038B000F4EE677AF1EE10FA06D6F0EEE77AF4EE5F
:1038C000487AF1EE10FA04DD242303FB05435A6A1B
:1038D0001A63242303FB0543D3ED090AD3ED0D7AC4
:1038E00093F8382070EEA70AA2B993ED0C0A20468F
:1038F000FFF746FDD4ED257A30EE670AB4EE400AB4
:10390000F1EE10FA16D7242303FB0545002385F8B2
:103910003A3022E0012A09BFD3ED0C7A93ED0B0A6D
:1039200077EEE00AD4ED3B7A04BF80EE897A87EE29
:10393000270AE3E7F0EEC07AF4EE487A2423F1EEAA
:1039400010FA03FB0545E1DC012385F83A30D4ED9C
:10395000237A37EE800A85ED0B0A013796E7627C01
:1039600020461146FFF788FE48B1242101FB0242A0
:1039700092ED0B0AD16904F1A80033F0BDFB94F974
:103980009C10277C002907DBB94205DACAB2114630
:103990002046FFF771FE68B900226274D5B2AF42CB
:1039A00009D929462046FFF767FE01320028F5D0E5
:1039B000657400E062742046FFF7AAFE2046FFF718
:1039C0004DFE10B1204652F007FA637C242505FB1A
:1039D000034393F83930B34216D032F07BFB4FF6F5
:1039E000FF7132F041FB78B1607C05FB004494F834
:1039F0003930002B14BF00220422019232F06AFBFE
:103A0000019A122132F0C2FA03A80EF051FF05B05C
:103A1000BDEC048BF0BD00BF0AD7233C0AD7A33C02
:103A200048E17A3F00000034FFFF7F7F0020194605
:103A30002DE9F04F0446007C0F4687B004F13A03AD
:103A400000220121D5B2A84203F1240305D903F8CD
:103A5000231C03F8241C0132F4E76F4B1E68F06A44
:103A600003685B68984740B13BF024F86B4A062135
:103A700007B0BDE8F04F34F02DBA3BF01BF8684AB0
:103A8000062134F027FA002303A904F188000393E8
:103A90002FF082F80A2550F041FD80462046FFF7BE
:103AA000B7FE50F03BFDA0EB0800B0F5FA7F02D95D
:103AB0005C4800F083FFB06A03680A215B6898479E
:103AC000617C2046FFF7D8FD0028E7D0B06A036884
:103AD00064215B68013D984715F0FF05DBD1524B2F
:103AE00005951B888DF80650CDE90355ADF80430D7
:103AF000052550F013FD80462046FFF789FE50F063
:103B00000DFDA0EB0800B0F5FA7FD1D8617C20460E
:103B1000FFF7B2FD0028EFD094F810B00DF10C08BB
:103B2000A14601AA4FF0000A5FFA8AF18B4516D927
:103B30002046FFF7A1FD50B1D8ED007A99ED097A42
:103B4000137877EE877A0133C8ED007A13700AF1A3
:103B5000010A08F1040809F124090132E4E7B06A16
:103B6000036864215B68013D984715F0FF05C0D1EB
:103B7000A9464FF02408237C5FFA89F6B34226D980
:103B800006AB334413F8143C33B908FB064686F8F9
:103B90003B3009F10109EEE7002FFAD007EE903A29
:103BA00006AA02EB8602F8EEE77A12ED030AD4EDDC
:103BB000250A204680EE270AFFF730FC08FB064066
:103BC00002A930308DED020A2EF0E6FFE1E7617CBC
:103BD000DFF85C902046FFF7D1FC002684ED3D0A1B
:103BE0004FF02408237CF7B2BB420FD908FB0743F0
:103BF00093F83B3043B13AF05DFF7B1C4A46062107
:103C000034F068F90135EDB20136EBE70DB907483C
:103C10004FE707B0BDE8F08FCC25002090E80808FA
:103C2000BBE80808D1E8080848A408080DE9080816
:103C3000EBE8080808B5037C022B02D9034850F0D2
:103C40003DFC5A1C0274184608BD00BF2CE9080848
:103C500038B5057C02460024E1B28D4206D91046F3
:103C6000FFF70AFD01340028F6D138BD281E18BF21
:103C70000120FAE770B50D4609780729044606D8F1
:103C8000027E437E22B901228A401343437670BDEF
:103C9000002BFCD000262278F3B29A42F7D904EB2D
:103CA0008303294658680368DB6898470136F2E7C2
:103CB00037B50D460192FFF7CBFF0199044630B9A5
:103CC0000448054B00682A46C06A0EF0ADFF204646
:103CD00003B030BDCC250020970C0A08014B1868B2
:103CE000704700BF2C5A002010B50446006810B180
:103CF00003685B689847204610BD000010B5044675
:103D0000006810B103685B689847204610BD00004A
:103D100070B5D0ED247A9FED637AF0EEE77AF4EE99
:103D2000C77A0123F1EE10FA8AB00446037609D46B
:103D30009030002309A9059009932EF02DFF0598D6
:103D40002EF074FB0026E6632666C4F884607622B3
:103D500031462046FFF760FC054600283CD0CDE9FF
:103D60000666079A0992002309A92046CDE9073380
:103D700051F0AEFF01462046FFF73AFC09A8FFF7D5
:103D8000B3FF08A8FFF7B0FF07A8FFF7B7FF15B10B
:103D900006A8FFF7B3FF2378032B56D0237C032B11
:103DA00053D094F99D10002925DAD4F80031DA04B3
:103DB0005DD40025637EEB40DB07EAB25DD40135BC
:103DC000082DF7D1237823B1237C13B16368002B2E
:103DD0003BD1354800F0F2FD344B1B685968042292
:103DE0000B68CDE90102324A00921E680246762332
:103DF00007A8B047B5E77722C9B22046FFF70CFC09
:103E0000054620B30023CDE90633079B0993002222
:103E100009A92046CDE9072252F012FD01462046AD
:103E2000FFF7E6FB09A8FFF75FFF08A8FFF75CFFB5
:103E300007A8FFF763FF15B106A8FFF75FFF237818
:103E4000032B02D0237C032BAFD10AB070BD174BDC
:103E50001B68596804220B68CDE90102144A0092DC
:103E60001E6894F89D20772307A8B047CDE7637EAE
:103E7000002B9ED1012363769BE73820059201F049
:103E8000A3FE064618B1059A214652F077FD314649
:103E90002046FFF7ADFB2378032BD6D0237C032BE2
:103EA0008DD1D2E70000003440E90808CC2500207D
:103EB000801A060090F81835934207D902F59E72D1
:103EC00050F8220010B103689B6A18470020704721
:103ED0002DE9F34105466E4686E80C00134B45F884
:103EE000043B04460F4600F5C87828462C3500F000
:103EF0008DFCA845F9D196E8030004F21C53C4F8E0
:103F0000147583E80300089BC4F82435084920464B
:103F10002EF0B4F8074B1A6812B1074850F0CEFAE9
:103F200020461C6002B0BDE8F08100BF34ED0808F7
:103F3000FCEB0808305A002040EB08082DE9F0415E
:103F4000A2B00C4607A92DF06FFB002855D0002128
:103F50000D220CA80591ADF818100B9172F0F2F932
:103F60002B4B611C1F68C9B20BAD0129F86A0A9579
:103F700046D1284B062205A90EF056FE264B01938A
:103F800005AB0093002411222946244BF86A8DF8D2
:103F900019400EF049FE04AA0DF10F0128468DF8D4
:103FA0003C4004942EF0D6FC38B31D49DFF86C80F9
:103FB000482210A872F07CF9062610AC2268531E25
:103FC000049AC2F3513202EB831223798DF8243024
:103FD000A368019305AB009308924346112229463A
:103FE000F86A0EF021FE0021B7EE000A07A82DF0B6
:103FF0001DFD013E04F10C04E0D122B0BDE8F081CA
:104000000091084B062205A90EF00EFEB6E700BF90
:10401000CC250020D1DA080871EB08086BEB080802
:104020004CA4080864EB08082DE9F04F90F81865D7
:1040300085B00446002E59D17F2380F828350DF134
:104040000F01042328308DF80F302EF0E1FD04F528
:10405000C87504F59E68271D5FFA86FA1822FF21AD
:10406000284672F06FF985F857A097F92490B9F1B6
:104070000A0F59D03DDCB9F1040F0FDCB9F1020F82
:104080000FDD442001F0A0FD834620B13B462A46C7
:10409000214652F0FFFCC8F800B002E0B9F1090F68
:1040A00036D0D8F8000050B1E96DC5F8589031B15C
:1040B000244B43F826102EF0EFF92EF0E5F958F8CE
:1040C000040B0AF101095FFA89F940B103689B68A2
:1040D000984784F8189551462046FFF72FFF013680
:1040E000092E05F1600507F12C07B5D105B0BDE833
:1040F000F08FB9F1190FD4D1482001F065FD834646
:104100000028C8D03B462A46214653F03DFBC2E773
:10411000382001F059FD83460028BCD03B462A4692
:10412000214653F011F9B6E7302001F04DFD8346EA
:104130000028B0D0CDF800A03B462A46214653F0D7
:10414000A5FAA8E7345A002090F818358B4283BFAF
:10415000602303FB010090F8D501002070470000A8
:1041600090F818358B4283BF602303FB010090ED6C
:104170006A0A9FED010A70470000000090F81835A8
:104180008B4206D901F59E7150F8210008B152F01A
:1041900015BE9FED010A70470000000010B490F8B2
:1041A00018458C420A4614D901F59E7450F82440F3
:1041B0007CB1E468246A640603D55DF8044BFFF71C
:1041C000DDBF602101FB020393ED6A0A5DF8044B39
:1041D00070479FED010AF9E70000000090F81835DC
:1041E0008B420BD901F59E7150F8210038B1C3689C
:1041F0001B6A1A4214BF012000207047002070473C
:1042000070B590F81835934204460E46154601D80D
:10421000002070BD02F59E7350F823000028F7D0EF
:1042200003689B6998470028F2D0602202FB05448E
:10423000D4F8AC313360ECE770B590F818359342A0
:1042400004460E46154601D8002070BD02F59E7347
:1042500050F823000028F7D003689B69984700288E
:10426000F2D0602202FB0544D4ED6C7AF4EE677A5A
:10427000F1EE10FAE8D6C6ED007AE6E770B590F8F0
:104280001835934204460E46154601D8002070BDED
:1042900002F59E7350F823000028F7D003685B698D
:1042A00098470028F2D0602202FB0544D4F8B431CC
:1042B0003360ECE790F8183593420ED902F59E73FF
:1042C00050F823305BB1602303FB020292F8E40153
:1042D00030B1D2F8E0310B607047002070471846CB
:1042E0007047000008299DBF2C2303FB0100406894
:1042F000002070472DE9F04F4B4B2DED028B1B68D2
:10430000DB6A93F89C3089B00446002B00F086806D
:10431000DFF82CB19FED458A4FF0000994F818356D
:104320005FFA89F5AB4279D905F59E7354F82300FD
:1043300000285DD003685B6B9847602303FB05434F
:10434000074693F8D431834252D2032861D8DFE87C
:1043500000F04F025259364E4FF000083AF0AAFBD7
:1043600094F81825AA4284BF602202FB05424FF050
:10437000600105F1010301FB05458CBFD2F8A821BE
:1043800018EE102A8246D5F8B001CDE90632F8F7CA
:10439000B3F8079ACDE904011046F8F7ADF8069B8B
:1043A0000096CDE902015A460421504633F092FDB1
:1043B0000123204A84F8293585F8D471D372D4F8C2
:1043C00024354BB3002255B25957481C03D0414500
:1043D00002F10102F7D194F92835AB4208DBD4F899
:1043E0002035D4F81C0542463146984784F82855B4
:1043F00009F1010992E72C2303FB05430E4E93F9C3
:104400002B80ABE72C2303FB05430C4E93F92C8048
:10441000A4E70026B046A1E71D46DCE709B0BDECE5
:10442000028BBDE8F08F00BFCC250020000000000B
:1044300085EB0808B55A0020BA170A087CEB080873
:1044400094EB080890F818358B4207D901F59E7156
:1044500050F8210010B10368DB691847002070474D
:1044600008299CBF602303FB010000F5C87070475A
:1044700090F81835934207D902F59E7250F8220041
:1044800010B103685B6A1847002070472DE9F04FB0
:10449000002493B005460E46174621462F2206A853
:1044A000059405F59E6971F04DFF05F1280A4FF05E
:1044B0002C0B05F5F4730BFB04F259F8040B1AF9F5
:1044C0000210E5B230B951B90134092CF3D14FF0E3
:1044D000010813E0602262439A58914212D01548B5
:1044E000154B006801930135EDB20095134BC06A7E
:1044F000324639460EF098FB4FF00008404613B0A4
:10450000BDE8F08F05A93322039352F039FD039BD8
:10451000804605A90028D7D1064801910135EDB2A2
:1045200000680095054BC06A324639460EF07CFBA8
:10453000E4E700BFCC250020CAEB0808BCEB080864
:104540002DE9F04FDFF88090DFF880A0DFF880B031
:104550008DB00646002796F81835FCB2A3422ED936
:10456000602505FB046595F8DC3133B395F8DD1162
:1045700019BB4FF001082022444404A889F819808F
:1045800071F0E0FE07EE904A4AF21043F8EEE77A47
:1045900003AA4C21ADF8283050462423CDED037AF0
:1045A00035F098FB3AF086FA9BF80030054A009403
:1045B000042133F08FFC85F8DD810137CBE70DB0A6
:1045C000BDE8F08FD4EB0808B55A0020615D0020EB
:1045D000052300202DE9F04F2F4B1E6885B00446BF
:1045E00046B1D0F81415304631F03EFD10B13046DA
:1045F00030F09CFC4FF092FF4FF0000801904FF01C
:104600002C0A4FF0600B94F818355FFA88F5AB422E
:1046100039D904EB8507D7F8F00488B30AFB0543C2
:104620000BFB054993F92820D9F8E8118A4227D1D4
:1046300032B30268D2689047D7F8F0040268126B70
:10464000904799F8D52112B1019BC9F8D831BEB174
:10465000D4F81415304631F007FD88B14FF066FFED
:10466000CDE9021002460B46D7F8F004294652F075
:104670007FFEDDE90232D7F8F004294652F0F6FE5B
:1046800008F10108BFE72046FFF734FE204605B0D9
:10469000BDE8F04FFFF754BFD45C00202DE9F04790
:1046A0004FF000082DED028B04468946B0EE408A9B
:1046B000474601264FF0600A94F818355FFA88F5EE
:1046C000AB421AD929FA05F3DB070AD505F59E7323
:1046D00054F8230078B10368B0EE480A9B6B984702
:1046E00006400AFB054508F1010895F8D4319F42C0
:1046F00038BF1F46E0E70646F3E727B97F23A4F853
:104700002835034BDF72BDEC028B3046BDE8F087E5
:10471000B55A002090F818358B4207D901F59E71E3
:1047200050F8210010B10368DB6B18470020704778
:104730000B46114690F818259A4207D903F59E7347
:1047400050F8230010B103681B6C18477047000035
:1047500070B504460E46002594F81835E9B28B4230
:1047600005D932462046FFF7E3FF0135F4E770BD77
:104770002DE9F84390F818550246002400F1280668
:104780002C2700F5F4784FF06009E1B28D420FD983
:1047900007FB04F309FB04F0F35658F800008342CA
:1047A00009D11BB11046FFF7CFFC10B10134ECE783
:1047B0000120BDE8F8830020FBE7000010B590F869
:1047C00018258A42044617D9602202FB010393F898
:1047D000D431022B03D004D9032B18BF0023184671
:1047E00010BDFFF797FF48B92046FFF7C1FF00282B
:1047F0000CBF06230123F2E70023F0E70623EEE7D0
:10480000014B1868704700BF305A002010B50349AB
:1048100004462DF033FC204610BD00BFACED080867
:1048200010B50446203043F001FA044B04491C60E3
:1048300020462DF023FC204610BD00BF585A002012
:1048400020EF0808F7B5B7EE000A0022022104465F
:104850002DF004FA204652F0E7FF43F0CBFA144B58
:104860001D680646E86A03685B6A98470B460221A2
:1048700002460091304643F0EFF9B4F94A60002E49
:1048800014DDEF6A3B6838465B68B4B2984728B1DC
:1048900097F84D3013B1C92EA8BFC824A86A036881
:1048A0005B68214603B0BDE8F040184703B0F0BD97
:1048B000CC25002010B5044652F084FF2046BDE808
:1048C000104052F0AFBF00002DE98048284BDFF8C0
:1048D000A490DFF8A4A0DFF8A4B01446012293B09E
:1048E00005460E461A704FF000084FF017FED9F833
:1048F00000300393A0EB080241F287339A42074647
:104900001FD9CDE9005603985346342205A9C06A41
:104910000EF08AF9214605A804944EF0DBFFCDE99C
:10492000005603985B46342205A9C06A0EF07CF954
:1049300004943AF0BFF8049B05AA022133F0B0FAC0
:10494000B8463AF0B7F839F0B3F93AF0B3F83AF0BC
:10495000C5FF0A2105A80DF06FFF039B986A036845
:1049600005215B68984705A80DF072FFBDE700BF01
:104970005C5A0020CC2500209CEE0808C52A0A08B5
:104980000FB400B595B016AA002152F8043B03926B
:1049900005A83C220193049171F0D4FC054A019BC7
:1049A000402104A84EF03EFF039A034804A9FFF7F4
:1049B0008BFF00BFA4EE0808BAEE08080FB407B5D5
:1049C00004AA034852F8041B0192FFF77DFF00BFC1
:1049D000CCEE08080146D0E9070300B11847002BC8
:1049E000FCD17047B0F9023002889A4314BFC3F378
:1049F000C00000207047000038B507230380022262
:104A000000230525C0E90532C0E90D33C0E91033A4
:104A1000C0E92C330C490362C0F89C5004462DF0C9
:104A20002DFB0A4B196811B109484FF047FD94F965
:104A300010001C602A4611F0D7FA637C207403F042
:104A400010036361204638BD70F00808605A0020EA
:104A5000B0EF0808012343610423C36470470000DA
:104A6000002343610423C364704700000123C3642F
:104A7000704700000223C364704700000323C3642F
:104A80007047000010B5C36993B190F9514090F997
:104A900050309C4207DA074B07480068C06A0EF0A6
:104AA000C3F8002010BD036A012B01D8034BF3E7C4
:104AB0000120F7E7CCEF0808CC250020D8EF080844
:104AC000F8B504463BF082FA3BF06CFA3CF02AF968
:104AD00007463BF07BFA3BF06FFA3CF023F90646C1
:104AE0003BF074FA3BF04AFA3CF01CF905463BF007
:104AF0006DFA3BF04DFA3CF015F90246606C50B18E
:104B000001285FD1012E5DD1012A5BD1012D14BF97
:104B100000200820F8BD012F28D176B9012A61D1E3
:104B2000012D63D1627CD70705D494F9511094F913
:104B30005020914210DA0220ECE7022E16D1012A11
:104B400050D1012D52D1627CD60741D494F9511035
:104B500094F9502091423BDB6269216C8A421AD061
:104B6000002A33D0012A08BF0A20D3E7002D3BD00A
:104B7000012E0BD1012A09D1022DEDD12046FFF7DC
:104B800031FF002814BF04200320C3E7E2B1022A4A
:104B9000E2D10620BEE7E26CA16B8A42BAD0012ABC
:104BA0001DD1617C0D0715D4617C490710D4022A00
:104BB00012D1617C0B070DD4627C12F0040F18BF78
:104BC0000220A7E70020A5E70520A3E70920A1E729
:104BD00001209FE710469DE7042A9BD1ECE7032ABA
:104BE000E5D1E1E7002DD1D1072093E7002DB3D126
:104BF000FAE700004B6A022B4FF0000303D080F865
:104C00004830436470478A68032A05D0042A05D0D7
:104C1000002380F8483070474364F9E70B680A7B4B
:104C20005B78012A03F00F0305D0022AF0D1002B94
:104C3000EED00262ECE7002BEAD005230362E7E73F
:104C4000FFF7D8BF037C033B022B94BF0120032056
:104C500070470000037C033B022B94BF012004201B
:104C600070470000C06910B103681B6A184770479D
:104C700070B50446C069036800215B6C9847E06921
:104C8000036801219B6C9847E06903680021DB6B96
:104C90009847E5692B682846D3E90D63984740F4A7
:104CA000407081B22846B0470A23E0691A464FF4A3
:104CB000E1310DF087FEE0690368BDE870401B6AD2
:104CC00018470000033904299ABF024B58560020A8
:104CD000704700BF68F00808F7B5C36904466BB3B6
:104CE000E2B9012915BF0023012303270427CC20A3
:104CF0008DF804008DF805100BB18DF80620002604
:104D000030467D1EF3B2AB4206F1010609DA02AA73
:104D1000134413F8041C11F02BFAF3E701230427C2
:104D2000E5E702AB1D443A4605F8040CE069036868
:104D300001A9DB689847E0690DF0A0FE03B0F0BD63
:104D400010B5C4693CB18469012C06D1C262CAB2F3
:104D50002146FFF7C1FF204610BD0020FCE7000000
:104D6000042910B5044604DC02290DDC01290ED00B
:104D700010BD0A29FCD1FFF765FFE2680146204615
:104D8000FFF7DEFF032306E0437C9B07F0D5FF23FC
:104D9000A4F8523004232362EAE7000010B590F82B
:104DA000513080F85030044643F076F920B100F5D8
:104DB0008050002380F884346369012B0DD163880F
:104DC0005B060AD52046FFF73DFFE2680146204614
:104DD000FFF7B6FF0323236210BD0223FBE70000A9
:104DE000013938B50446062969D8DFE801F0042006
:104DF00031688B8BB60090F95030002B5FDC0133AB
:104E000080F85030C2680221FFF79AFF94F95030C1
:104E1000002B0ADD43F040F920B100F5805001235A
:104E200080F884340523236249E00423FBE790F9EA
:104E30005030002B08DD013BC26880F85030022161
:104E4000FFF77EFF0623EEE7BDE83840FFF7A6BF79
:104E500090F9503090F95210012B20DD90F910009C
:104E6000484D421EC2EBC202AB18AA5C2AB353FAE9
:104E700081F394F853205B78013B9A421DD10528B9
:104E80001BD0A26800212046FFF75AFF002384F8B8
:104E9000533094F85030013B84F850300FE00CD17F
:104EA00090F910203748531EC3EBC303C35C23B1F2
:104EB000013B994201D1052A02D100290BDA38BD04
:104EC000E26800212046FFF73BFF94F85030013B99
:104ED00084F85030B6E794F910302A4A013BC3EB0E
:104EE000C30313440B445B78002BE8D0A268002175
:104EF0002046FFF725FF94F950300133022BA8BF5D
:104F00000223C9E701218268FFF71AFF94F95030A4
:104F10001C49012B94F9103011DD013B94F852002B
:104F200094F85320C3EBC3030B44034401325B7872
:104F3000B2FBF3F103FB112284F85320BFE7013BDE
:104F4000C3EBC30394F95220CB5C013292FBF3F123
:104F500003FB112284F85220B1E790F95030002B66
:104F600009DD013B80F850300023C26880F85330DF
:104F70000221FFF7E5FE94F95030002B9FD194F801
:104F80005130A5E70D22002010B54369012B0446DE
:104F900010D143885B060ED5437CD90607D4FFF7B2
:104FA00051FEE268014652002046FFF7C9FE032386
:104FB000236210BD0BB10223FAE743885A06FAD5E3
:104FC000437CDB06F7D5FFF745FEE2680146520059
:104FD0002046FFF7B5FEEEE7042910B5044604DCD1
:104FE00002290DDC01290ED010BD0929FCD1FFF7E3
:104FF00031FEE26801462046FFF7A2FE02230EE0E2
:10500000437C9B07F0D52046FFF724FEE26801466B
:105010002046FFF795FEFF23A4F8523004232362B5
:10502000E2E7000010B504464FF078FAA36AE26A9E
:10503000C31A934207D3226AA0620023022AE362C2
:1050400002D0032A10D010BD6269012A0AD16388F8
:1050500013F0400F0CBF00210A212046BDE810408C
:10506000FFF77EBE1946F8E7616949B9638813F016
:10507000400F18BF09212046BDE81040FFF7ACBF24
:105080001946F8E773B50B685B78836143885B0466
:105090005EBF0B685B884380B0F90230002B04468A
:1050A0001ADD0123036239F005FD05462046B4F9F7
:1050B0000260FFF797FC68B92388B3430CBF022353
:1050C00000230093094A33460621284632F002FFA6
:1050D00002B070BD0523F4E739F0ECFC044A04216A
:1050E00002B0BDE8704032F0F5BE00BFECEF08083A
:1050F0001DF00808FFF7C6BF70B50446D0F8B80029
:105100000E46E8B1D4F8A83023B1D4F8A420CB1AC5
:10511000934221D3B4F8AC509DB12046FFF7A8FDCF
:10512000D4E9260194F8A020FFF7D6FDB4F8AC30FE
:10513000C4F8A8600020013B84F8A100A4F8AC30BA
:1051400070BD042304F19400C4F8B830FFF742FCAA
:10515000C4F8B8502846F3E70120F1E738B5002439
:10516000054620466B7BA34205DD2B68195D10F0D8
:10517000FFFF0134F6E738BD2DE9F041C36904466D
:10518000002B43D04FF0CAF901462046FFF7B4FF89
:1051900000283BD0E06903685B699847402828BF36
:1051A00040200025064604F19407A846AE422DD0C3
:1051B0004FF0B4F901462046FFF79EFF30B3E06997
:1051C00003689B69984794F8A130C0B20BB9CC280A
:1051D0001AD1D4F89420D05494F8A13094F8A22095
:1051E0000133DBB29A4284F8A1300DD13846FFF783
:1051F000B5FF00280CBF02230323C4F8B83038469B
:10520000FFF7E8FBC4F8B8800135CFE7BDE8F081CF
:10521000074A002352F83300884203D102EBC3034C
:10522000187970470133042BF4D10020704700BF78
:105230003022002038B5037300234373049B0361BD
:105240001546BDF81430856001F154020446C0E9EA
:105250000021038300F11C03DDE9060183E803005C
:10526000012363624FF05AF9294660612046FFF737
:10527000CFFFA073204638BD2DE9F0438FB016ACA8
:10528000064634F8049B0F4690461D46FFF7EAFC9D
:1052900094E8030002AB83E803003A46CDE90059E5
:1052A0004346314604A804ACFFF7C4FF0FCC06F117
:1052B00094050FC50FCC0FC594E80300424685E85E
:1052C0000300394630460FB0BDE8F043FFF704BD98
:1052D00010B586B0094B0593049006AA12E90300A5
:1052E00001AB83E8030000224FF6FF7300931146E1
:1052F0004FF47A63FFF7C0FF06B010BDF550010808
:1053000013B51A4B0446186820B100221A212EF05A
:105310007DFCE061E36953B101230DF1070104F164
:1053200010008DF807302DF073FC2DF0ADF894F9D6
:10533000103013B9E36102B010BDE269002AFAD05F
:10534000022B01D0052B03D14FF6FF73A4F8503088
:105350002046FFF78DFC4FF0E1F86368A06220461D
:10536000E36202B0BDE81040FFF7B2BF845B0020EB
:1053700030B587B004AB83E80600054693E8030028
:1053800001AC022384E805000421009301224FF4BC
:10539000C8732846FFF770FF07B030BD30B587B03F
:1053A00004AB83E80600054693E8030001AC84E8FB
:1053B0000500022200924FF4C87304212846FFF72B
:1053C0005BFF07B030BD000010B586B006AC04E945
:1053D0000C0061B10124446401AC84E80C00022497
:1053E000CAB200944FF4C8732146FFF745FF06B0D8
:1053F00010BD000070B586B004AB83E8060002253E
:105400004564044693E8030001AE86E805004FF4C6
:10541000C8730095002203212046FFF72DFF06B038
:1054200070BD000010B5012380F848304B1E88B0D5
:105430000446C262072B31D8DFE803F0040E1818C7
:1054400018181825164B00901A460146019308B00B
:10545000BDE81040FFF78CBF114B02901A46014681
:10546000039308B0BDE81040FFF798BFFFF72AFC90
:105470000B4B0494014622462046059308B0BDE834
:105480001040FFF7A1BF064B0793069008AB13E946
:10549000060008B0BDE81040FFF7ACBF08B010BD73
:1054A000414C01084B1E10B50446092B20D8DFE8FB
:1054B00003F00C233636363636053636642208219C
:1054C0002046BDE81040FFF7ADBF90F9503083B9DA
:1054D00042F0E2FD20B100F58050012380F88434D1
:1054E000642201212046FFF79DFF012384F85030FC
:1054F00010BD64220321E3E790F95030002BF7DD63
:1055000042F0CAFD20B100F58050002380F88434B9
:10551000642202212046FFF785FF0023E6E764228C
:10552000CEE7000013B504460191FFF75BFA01993D
:1055300028B1204602B0BDE81040FFF7B3BF238872
:10554000B4F90220934305D1204602B0BDE81040D3
:10555000FFF746BC02B010BD70B504464EF0DEFF4A
:1055600094F8482022B9A36AE16AC31A8B4202D296
:105570000023236370BDC4E90A022046FFF7A0FAA6
:10558000236B626983420146236AE06C0ED1656B2E
:10559000AB420BD1A56B854208D194F93C6094F9DC
:1055A0005050AE4202D1256C9542E3D0C4E90C13B1
:1055B000A063013B94F8500084F83C002264052B62
:1055C000D8D8DFE803F003080D1213182046BDE811
:1055D0007040FFF7D9BC2046BDE87040FFF7C0BB64
:1055E0002046BDE87040FFF7F7BC01212046BDE82A
:1055F0007040FFF797BF0221F8E7000010B50D4B90
:105600001B68DB6A93F89C30044623B12046BDE852
:105610001040FFF707BD42F03FFD28B100F5805371
:1056200093F86434032BF1D82046BDE81040FFF70F
:1056300093BF00BFCC25002038B5C36904467BB1B9
:1056400090F9103063B1FFF797FD4EF067FF636A82
:10565000C31A642B054603D92046FFF7CFFF6562C6
:1056600038BD0000014B1868704700BF605A002029
:1056700008B50449102270F00BFEB0FA80F0400922
:1056800008BD00BF645A00201022002170F05ABEED
:1056900010B50446FFF7F8FF204610BD03784160BF
:1056A00023F00D03022A037008D0032A0AD0012A2E
:1056B00003D1DBB243F0010303707047037843F07A
:1056C0000803F9E7037823F0050343F00503F3E744
:1056D00073B504460E4615460193FFF7D5FF2046E5
:1056E000C4E90265069A0199FFF7D8FF02B070BDC0
:1056F0000078420704D4030704D400F00100704787
:105700000320704702207047F0B585B00546164665
:10571000FFF7EEFF88420F4605D16B683360012426
:10572000204605B0F0BD032801D10024F8E7032985
:10573000FBD001280BD0022816D018BB6D68012FB2
:1057400022D0022F2ED0002FEFD13560E7E7FBF7F4
:10575000F3FE90F87C32DB07E7D56D68FBF7ECFED3
:10576000D0F870321D44EAE76846FFF78DFFFBF77B
:10577000E3FE6946FBF7E6FC04460028D0D06D68DE
:10578000019BEFE70025DAE7FBF7D6FE90F87C42B5
:1057900014F00104C9D0FBF7CFFED0F87032ED1A37
:1057A0003560BDE76846FFF76FFFFBF7C5FE69464A
:1057B000FBF7C8FC04460028B2D0019BEFE70000CD
:1057C00073B501AA05460E46FFF79EFF044620B1B9
:1057D000019932462846FFF761FF204602B070BDAE
:1057E00013B5144601AAFFF78FFF48B1DDED017A2A
:1057F0009FED047AF8EEE77A67EE877AC4ED007AD7
:1058000002B010BD0AD7233C07EE900A9FED090AAB
:10581000F8EEE77A08B527EE800A6EF08BF9DFED37
:10582000067AB4EEE70AF1EE10FAD8BFB0EE670AD6
:1058300008BD00BF50E0EF300AD7233C10B5044646
:10584000806810F03DFD20B1E068BDE8104010F028
:105850004BBD10BD0D4B83424FF000038B4106DA68
:1058600000F1255000F5311000F5E0507047084B6D
:1058700098424FF0FF3371EB0303BEBF00F1564077
:1058800000F5130000F52440704700BF00D2496BBB
:10589000002EB69490EA010F01D4401A7047C31746
:1058A000401A63EBE1710D4B83424FF000038B41D3
:1058B00006DA00F1255000F5311000F5E050704790
:1058C000074B98424FF0FF3371EB0303BEBF00F16B
:1058D000564000F5130000F52440704700D2496B94
:1058E000002EB69470B52DED028B84B00446684648
:1058F0000D46FFF7C9FEFBF71FFE6946FBF722FCCA
:10590000064608B3A368029ADFED128A03999B1A30
:1059100007EE903AF8EEE77A67EEA87AC5ED007ADE
:10592000E068FFF7B7FF08EE100AA068024402EB38
:10593000D272B8EEC88A5010FFF766FF28EE288AA8
:1059400028EE000A85ED010A304604B0BDEC028B5A
:1059500070BD00BFF67C8E3F37B500230C4601AA10
:10596000022105460193FFF7CFFE10B9002003B0D6
:1059700030BD21462846FFF7B5FF0028F6D0DDED03
:10598000017AF8EEE77AC4ED027AF0E738B52DED4A
:10599000028B0C460246C168E068FFF77BFF956802
:1059A000A46808EE100A601900EBD0704010641B68
:1059B000FFF72AFF07EE904AF8EEE77AF8EEC80AFA
:1059C00087EE807ABDEEC70A10EE103A5B4200EE19
:1059D000103AB8EEC00A6EF0CFFADFED087A30EE7A
:1059E000270ABDEC028BB5EEC00AF1EE10FA44BFF7
:1059F000DFED037A30EE270A38BD00BFDB0FC93F69
:105A0000DB0FC94030B52DED028B0B4685B08C689D
:105A1000D0E90251D868FFF73DFF08EE100A60197F
:105A200000EBD0704010FFF7EFFE641B07EE904ACA
:105A3000F0EE400AB8EEC88A9FED060AF8EEE77A63
:105A400028EE008A27EE800A68EE200A05B0BDEC39
:105A5000028B30BD8262363C82B002B0FFF7D2BF0B
:105A6000F0B52DED028B0D4689B08C680646D0E965
:105A70000271E868FFF70EFF08EE100AE01900EB6C
:105A8000D0704010FFF7C0FE73686A689FED0E1A71
:105A90009B1A07EE903AE41BB8EEE77AF0EE400A64
:105AA00007EE904A9FED090AB8EEC88AF8EEE77A49
:105AB00028EE008A27EE011A27EE800A68EE200AF7
:105AC00009B0BDEC028BF0BD0AD7233C8262363CA4
:105AD00010B52DED028B84688A680B46111B08EE09
:105AE000901AC168D868FFF7D5FE224402EBD27243
:105AF00008EE100A5010FFF787FEB8EEC88AF8EEDD
:105B0000E88A28EE000A20EE000AA8EEA80A6EF045
:105B10007DFBBDEC028BDFED027A20EE270A10BD83
:105B20008262363C094B984206DDC0F1D64000F552
:105B3000930000F5A4407047054B9842BEBFC0F1EA
:105B4000144000F5360000F53850704700E9A435E0
:105B500000175BCAF8B52DED028BDFED148A0768DC
:105B600020EE280A0646FDEEC07A0D4617EE904A52
:105B700004EBD47007EB6000B0EE608AFFF744FEE0
:105B800028EE288A3819C8EE007AFFF7CBFF30607C
:105B900017EE900AF7F7DAF92B68C01841EBE371BA
:105BA000FFF758FEBDEC028B2860F8BD02AAB34295
:105BB00000F10C010830FFF7CDBF00000148FFF7EE
:105BC00063BD00BF645A00200121884238BF0846E7
:105BD0006CF052B9FFF7F8BF08B16CF051B97047DB
:105BE000FFF7FABF00214FF0FF3310B50022036327
:105BF000044601600171C0F80510417280F825105B
:105C000000F13C0300F50B70D9709A60DA601A61FC
:105C10005A619A61DA611A625A629A62DA631A64A4
:105C20005A649A64DA641A655A659A65DA65DA66BE
:105C30001A675A677C339842E6D1214604F51670FC
:105C400007F0AAFA044B1A6822B904491C602046DE
:105C50002CF014FA204610BD745A0020A8F208084F
:105C600073B5D0F83C3201919942044613D0D0F874
:105C70004032994218D0D0F844328B4216D10220DB
:105C80000AE0D4F8343253B3D4F838324BB34FF07F
:105C9000030002B070BD002094F822308342F8D88F
:105CA000431C84F82230F4E70120F5E7D0F8306295
:105CB000002EE6D194F841233546B6009AB1A319D7
:105CC000C3F83012A319019AC3F83C2294F8223089
:105CD000AB429CBF6B1C84F822302846D9E70126D2
:105CE000E8E70226E6E704F50C7001A930442DF040
:105CF00061F8E7E738B504460D462CF0D1FF291DC1
:105D0000201D2CF0CDFF05F1080104F108002DF055
:105D1000A1F805F1140104F114002DF09BF805F130
:105D2000200104F120002DF095F805F12C0104F17B
:105D30002C002CF049FF05F1300104F130002DF06A
:105D400051F805F13C0104F13C002DF083F8AB6BF8
:105D5000A3636B6B636338BD2DE9F043A1B00023EF
:105D6000002500F13C0706468DF807500393049385
:105D7000059306930793089309930A930B93109343
:105D800011931293139314931593169317931893D7
:105D90001C931D931E9300F50F78B94658F8043BE9
:105DA000F3B1F26E934223D0D6F8E820934221D08B
:105DB000D6F86421934213D10221EBB299420FD05D
:105DC000C1EB411109EB8104214601A8FFF792FFC5
:105DD00039462046FFF78EFF01A93846FFF78AFFB4
:105DE0000135032D07F17C07D8D121B0BDE8F08340
:105DF0000021E2E70121E0E72DE9F04706460F46E2
:105E00001546804604464FF0000A39463046FFF7F3
:105E100027FF626FBA425FFA8AF90ED1C3B2022B32
:105E20000BD87C2202FB0A66012086F83E0086F829
:105E30003F3085F80090BDE8F0870AF1010ABAF119
:105E4000030F04F17C04E0D1002439463046FFF70B
:105E500007FFD8F86C205FFA84F912B9C3B2022B9D
:105E600022D90134032C08F17C08EED100244FF034
:105E70007C0906F13E0A39463046FFF7F1FE03463B
:105E800009FB04F05FFA84F81AF8002012B9DBB2BB
:105E9000022B12D90134032CEDD196F823000428EB
:105EA00014D919484EF00AFB7C2000FB0464012041
:105EB00084F83E0084F83F30BBE70644012086F8B2
:105EC0003E0086F83F3085F80080B4E706F5437160
:105ED000002251F8043BBB42D4B208D1A04202D800
:105EE000631C86F8233003342C700020A3E73BB9F1
:105EF000421C06EB800086F82320C0F80C73F2E702
:105F00000132052AE5D1F0E7E0F00808C9B200EB5C
:105F10008101D1F83C3253B1026F93420AD0D0F8DC
:105F2000EC20934208D0D0F86821934206D04FF07D
:105F3000030070470020704701207047022070471F
:105F400059B190F82030032B07D05A1C80F820203C
:105F500000EB830041610120704700207047000082
:105F60002DE9F8430F469146044600F5BA7894F8B7
:105F70003E5035B97C344445F9D100252846BDE86A
:105F8000F88300234A46394601200CF0E3FA002149
:105F90000646E06E0CF0EEFA8642EBD1EEE700002A
:105FA0002DE9F043DFF87C8085B0044600F50F76DC
:105FB00000257C27B14656F80C3CD9F800209342C6
:105FC000E9B206F1040619D1C3B12046FFF79EFFDE
:105FD000C0B207FB004090F83E307BB903A9A9F19D
:105FE0000C0003932CF0E6FE38F064FD56F8043CF8
:105FF000009342462B46012131F06CFF0135032D01
:10600000D8D104F16C0504F5F074296821B9AB68A6
:1060100013B128462BF024FB7C35A542F5D105B001
:10602000BDE8F083FCF0080838B504461546FFF7D4
:106030006DFFC0B2022808D87C2303FB004029462C
:106040005030BDE838402CF0F5BE38BD38B50446B8
:106050001546FFF75BFFC0B2022808D87C2303FB7C
:10606000004029465C30BDE838402CF0E3BE38BD26
:1060700037B50D4604468DED010AFFF747FF022DA7
:1060800007D8C0B27C2303FB004001A968302CF084
:1060900083FD03B030BD000038B50546FFF736FF7D
:1060A000C4B2022C13D8C4EB4414A4003C3504F150
:1060B0000800284400212BF0D3FA04F1340104F144
:1060C000300029442844BDE838402CF073BE38BD68
:1060D00070B505460E461446FFF718FFC3B2022BF3
:1060E0000DD87C2000FB035394E80700443383E879
:1060F000070031462846BDE87040FFF7CDBF70BDB0
:1061000037B504461546FFF701FFC0B2022809D88B
:106110007C2303FB00400DF1070140308DF8075050
:106120002CF0BEFD03B030BD10B500210446FFF7D2
:10613000B3FF20460121FFF7AFFF20460221BDE853
:106140001040FFF7A9BF00001FB590F92C3004469E
:1061500023B390F921300BB36846FFF799FAFBF7A8
:10616000EBF96946FAF7CAFFC0B1DDED037A9FED9E
:106170000C0AF8EEE70ADDED027AF8EEE77A012381
:10618000C0EE800A84F83D3387EE800A07F046FAB5
:10619000DFED047A20EE270A84ED0A0A04B010BD70
:1061A0008096184B35FA8E3C024690F9210058B182
:1061B00092F8400340B1114491F92C0220B192F9B8
:1061C0002400033818BF01207047000038B590F84C
:1061D000223005465BB100242346E1B22846FFF792
:1061E000E3FF08B10133DBB20134032CF5D11846CB
:1061F00038BD000090ED0A0A7047000038B50C4623
:10620000D1ED066A11460546FFF780FEC3B27C2039
:1062100000FB0353D4ED087AD3ED260A94ED076A08
:10622000D3ED255A93ED245A26EE600A67EEA00AB4
:10623000A5EEA70AF0EE607AE5EE867AB7EE007A70
:10624000A6EEE67A67EEE60AB1EE400AE5EE070A48
:106250006DF092FE9FED071ADFED070A40F61C0075
:106260000FF084FED5ED0A7ABDE8384030EE270AFB
:106270000FF068BEDB0F4940DB0F49C02DE9F0414C
:1062800090F822308B4204460D4602D20020BDE831
:10629000F081FFF73BFEC0B204F13C06C0EB4010BA
:1062A00006EB8000083012F085FADFED157AB0EECB
:1062B000C00AB4EEE70AF1EE10FAE7D42946204608
:1062C000FFF724FEC5B27C2000FB05473B6F002B87
:1062D000DCD0032DDAD000FB05603030D7F86C80BD
:1062E0002BF0A2FFD7E91B32934201D1984505D08C
:1062F0007C2000FB0544C4F86C80C7E70120C6E79A
:10630000000000342DE9F74F04460E46174600F50D
:106310000F7A4FF0000B5AF8049B5FFA8BF8B9F133
:10632000000F26D041462046FFF73EFF08B3414606
:106330002046FFF7EBFD7C23C0B203FB004090F842
:106340003E505DB908F101031B4ADBB239463046C5
:106350004DF068FA284603B0BDE8F08F5AF8102CCB
:10636000914506D0154A394630464DF05BFA002576
:10637000F0E70BF1010BBBF1030FCCD14FF000089C
:1063800094F822305FFA88F18B420DD920460191B2
:10639000FFF774FF054620B901992046FFF704FF77
:1063A00020B908F10108EBE70125D3E7044A394693
:1063B00030464DF037FACDE724F1080839F10808E6
:1063C0005EF108082DE9F0412DED048B90F84213A1
:1063D0009FED348ADFED348A9FED349A82B0064611
:1063E000FFF794FD06F13C07C5B27C2000FB057564
:1063F00054354FF0000896F822205FFA88F39A424D
:106400004ED919463046FFF7CFFE10B908F1010802
:10641000F1E719463046FFF779FDC4B27C2000FB56
:106420000474D4ED157AF0EEE77AF4EEC87AF1EE62
:1064300010FA04F154040ED5D4ED017AF0EEE77AA7
:10644000F4EEC87AF1EE10FA05D5002002B0BDECEA
:10645000048BBDE8F0812946204612F0C3F9B4EE62
:10646000E80AF1EE10FAF0DC2946204611F0E2FCD1
:10647000B4EEC90AF1EE10FAE7DC2146284611F025
:1064800025FC68468DED000ACDED010A11F0BEFC39
:10649000DFED077AB4EEE70AF1EE10FAB6DDD4E7E5
:1064A0000120D3E700000034DB0FC93F920A863F8A
:1064B00000004843022910B5044608D8FFF726FD1E
:1064C0007C23C0B203FB004494F83D0010BD0020C3
:1064D000FCE7000013B590F8421301910446FFF762
:1064E000E9FF30B10199204602B0BDE81040FFF746
:1064F0005BBE02B010BD0000F7B590F92150044614
:10650000002D73D090F84053002D6FD090F84213B7
:10651000FFF7D0FF94F83D33064613B92046FFF746
:1065200013FE002594F82020EBB29A4207D904EB21
:1065300083030135586903689B689847F2E74DF07B
:10654000EDFF0027224604F5BA7140F2F315D2F8A8
:106550009C30C31AAB428CBF0023012382F83D302C
:106560007C32914247EA0307F1D194F92430032B9E
:1065700007D194F83C33002B3BD0D4F838030028E3
:1065800049D167B1236B013309D02FF0A3FD216BF3
:106590002FF06AFD18B12FF09DFD2EF0DBFD94F970
:1065A0002C32002B3AD194F92D32CBBB94F92E32F8
:1065B00013B1022384F8423394F842132046FFF7C4
:1065C00079FF8642054611D02FF084FD4FF6FF710A
:1065D0002FF04AFD50B1002D14BF00220422019279
:1065E0002FF078FD019A03212FF0D0FC284603B04C
:1065F000F0BD012384F83C330420FFF7E5FA05469B
:1066000010B1214606F05EFE94F92430C4F83853E8
:10661000032BB2D0B5E706F063FEB2E70023C9E76B
:106620000123C7E738B590F921300446D3B190F87B
:106630004053BDB1FFF76AFCC0B2022812D87C23D8
:1066400003FB0044D4ED1A7A9FED087AF4EEC77A82
:10665000F1EE10FA06D4B7EE087AF4EEC77AF1EE4E
:1066600010FA00DD0025284638BD00BFABAA2A3F3E
:1066700070B5D0F8085315F4003504460E460DD118
:1066800090F840335BB90A78072A07D8012303FA48
:1066900002F290F83F33134380F83F3370BD94F813
:1066A0002020EBB29A42F9D904EB830331465869B2
:1066B0000368DB6898470135F1E7000038B5054607
:1066C0006C242B591BB1002128192AF0C9FF7C34F6
:1066D000B4F5F07FF5D138BD014B1868704700BFA5
:1066E000745A00202DE9F04FAA4BD3F800800446DD
:1066F000D8F8040003688DB09B68984700250746CA
:106700004FF0010909FA05F33B4240F0828201355E
:10671000202DF7D1D8F804000368DB6898470025DE
:1067200007464FF0010909FA05F33B4240F0B382F6
:106730000135202DF7D1D8F8040003689B689847ED
:10674000002507464FF0010909FA05F33B4240F0E6
:10675000E1820135202DF7D1D8F80400DFF840B2EE
:1067600003689B68984700250490049A0123AB4076
:10677000134240F00B830135202DF6D1D8F80400E8
:10678000DFF81CB20368DB68984700250490049A80
:106790000123AB40134240F0C9830135202DF6D1CF
:1067A000D8F804000368DB689847002507464FF0D7
:1067B000010909FA05F33B4240F083840135202D9D
:1067C000F7D1D8F804000368DB689847002507462E
:1067D0004FF0010909FA05F33B4240F0B18401355D
:1067E000202DF7D1D8F8040003689B68984700254E
:1067F00007464FF0010909FA05F33B4240F0DF84F8
:106800000135202DF7D1D8F8040003689B6898471C
:10681000002507464FF0010909FA05F33B4240F015
:106820000E850135202DF7D1D8F8040003689B6848
:106830009847002507464FF0010909FA05F33B4246
:1068400040F03D850135202DF7D1D8F804000368CC
:10685000DB689847002507464FF0010909FA05F360
:106860003B4240F068850135202DF7D14A4B089313
:1068700008AF0425D8F8040003689B6898470026F1
:1068800083460123B34013EA0B0F40F08F85013696
:10689000202EF6D1D8F804000368DB68984700265C
:1068A00083460123B34013EA0B0F40F0C485013641
:1068B000202EF6D1013D15F0FF0507F10107D9D1D2
:1068C000D8F8040003689B6898474FF00109074611
:1068D00009FA05F33B4240F0F2850135202DF7D14E
:1068E000D8F804000368DB689847002507464FF096
:1068F000010909FA05F33B4240F01D860135202DC0
:10690000F7D1D8F8040003689B689847002507462C
:106910004FF0010909FA05F33B4240F04886013582
:10692000202DF7D1D8F804000368DB6898470025CC
:1069300007464FF0010909FA05F33B4240F0738620
:106940000135202DF7D1154B0793D8F804000368C3
:106950009B689847002583460123AB4013EA0B0F41
:1069600042D000275FFA85F9D4F8083313F4803A4F
:1069700032D107AB4946DB5D04931A462046FFF748
:10698000EFFA049B0646002800F08986CDE908AAA4
:1069900008E000BFCC2500200C0D0E0F2021222383
:1069A000801A0600099B0B93002201210BA8CDE958
:1069B000092204F003FE01462046FFF7C1FA0BA8A6
:1069C000FDF792F90AA8FDF78FF909A8FDF796F9E6
:1069D00016B108A8FDF792F994F82330052B00F0C2
:1069E00048810137042FBFD10135202DB4D1D8F80B
:1069F00004000368DB689847002583460123AB4009
:106A000013EA0B0F38D000275FFA85F9D4F8083362
:106A100013F4803A28D107AB4946DB5D04931A464C
:106A20002046FFF79DFA049B0646002800F04686A4
:106A3000CDE908AA0022099B0B9311460BA8CDE9CA
:106A4000092204F0BBFD01462046FFF779FA0BA8A6
:106A5000FDF74AF90AA8FDF747F909A8FDF74EF92D
:106A600016B108A8FDF74AF994F82330052B00F079
:106A700000810137042FC9D10135202DBED1D8F8AE
:106A8000040003689B689847002682460123B340B0
:106A900013EA0A0F31D010255FFA86F9D4F80833CB
:106AA00013F0080B20D12A4649462046FFF758FA32
:106AB0000746002800F01186CDE909BB0A9B002299
:106AC00001210BA8CDE90A2301F00AFC014620466A
:106AD000FFF736FA0BA8FDF711F90AA8FDF70EF932
:106AE00017B109A8FDF70AF994F82330052B00F037
:106AF000C0800135EDB2142DD0D10136202EC5D184
:106B0000D8F8040003689B68984700268246012352
:106B1000B34013EA0A0F34D014255FFA86F9D4F88B
:106B2000083313F4001B24D12A4649462046FFF7B8
:106B300017FA0746002800F0E385CDE908BB099B5A
:106B40000B93002201210BA8CDE9092201F0DAFF05
:106B500001462046FFF7F4F90BA8FDF7C5F80AA88F
:106B6000FDF7C2F809A8FDF7C9F817B108A8FDF7A5
:106B7000C5F894F82330052B7BD00135EDB2182DE4
:106B8000CDD10136202EC2D1D8F804000368DB68CD
:106B90009847002682460123B34013EA0A0F34D0F7
:106BA00014255FFA86F9D4F8083313F4001B24D1B6
:106BB0002A4649462046FFF7D3F90746002800F049
:106BC000AF85CDE908BB0022099B0B9311460BA8AA
:106BD000CDE9092201F096FF01462046FFF7B0F902
:106BE0000BA8FDF781F80AA8FDF77EF809A8FDF7C4
:106BF00085F817B108A8FDF781F894F82330052B24
:106C000037D00135EDB2182DCDD10136202EC2D1AD
:106C10002FE0D4F8083313F0010A25D15FFA85FB81
:106C20001E2259462046FFF79BF9064620B3CDE9C0
:106C300008AA099A0B920023082201210BA8CDE98A
:106C4000093303F089FA01462046FFF779F90BA8CA
:106C5000FDF74AF80AA8FDF747F809A8FDF74EF82E
:106C600016B108A8FDF74AF894F82330052B7FF4F5
:106C70004EAD0DB0BDE8F08FD8F8041004220B68BB
:106C8000CDE90102A84A0092D3F800A05A461E237B
:106C900009A8D047CDE7D4F8083313F0010A24D16E
:106CA0005FFA85FB1E2259462046FFF759F9064632
:106CB00008B3CDE908AA099B0B93062200210BA873
:106CC000CDE9091103F048FA01462046FFF738F9EB
:106CD0000BA8FDF709F80AA8FDF706F809A8FDF7C3
:106CE0000DF816B108A8FDF709F894F82330052B24
:106CF0007FF41EADBDE7D8F8041004220B68CDE97F
:106D00000102894A0092D3F800A05A461E2309A81E
:106D1000D047D0E7D4F8083313F4805A21D15FFA72
:106D200085FB0D2259462046FFF71AF90646F0B1B9
:106D3000CDE909AA0A9B0022CDE90A2301210822F4
:106D40000BA804F077FA01462046FFF7F9F80BA8E4
:106D5000FCF7D4FF0AA8FCF7D1FF16B109A8FCF78D
:106D6000CDFF94F82330052B7FF4F3AC81E7D8F8FE
:106D7000041004220B68CDE901026B4A0092D3F89B
:106D800000A05A460D230AA8D047D3E7D4F8083309
:106D900013F480773FD15FFA85F90C2249462046EB
:106DA000FFF7DEF80646002800F08480CDE906777C
:106DB000079B0A934FF0000A692249462046CDF806
:106DC0001CA0FFF7CDF80746002800F08180CDE930
:106DD00008AA099B0B9300221A2309920BA90122EE
:106DE0000AA801F005F801462046FFF7A9F80BA80C
:106DF000FCF784FF09A8FCF781FF17B108A8FCF78E
:106E00007DFF0AA8FCF77AFF07A8FCF777FF16B109
:106E100006A8FCF773FF94F82330052B3FF429AF45
:106E2000D4F8083313F480777FF4A5AC5FFA85F9C2
:106E30000C2249462046FFF793F80646002856D014
:106E4000CDE90677079B0A934FF0000A682249466E
:106E50002046CDF81CA0FFF783F80746002854D041
:106E6000CDE908AA099B0B9300221A2309920BA9CA
:106E700001220AA800F0BCFF01462046FFF760F897
:106E80000BA8FCF73BFF09A8FCF738FF17B108A8CF
:106E9000FCF734FF0AA8FCF731FF07A8FCF72EFF28
:106EA00016B106A8FCF72AFF94F82330052B7FF4CF
:106EB00062ACDEE6D8F8041004220B68CDF800B00E
:106EC000CDE901024A461F6807A80C23B8476FE7BF
:106ED000D8F8041004220B68CDF800B0CDE9010207
:106EE0004A46D3F800A009A86923D04771E7D8F82B
:106EF000041004220B68CDF800B0CDE901024A4627
:106F00001F6807A80C23B8479CE7D8F80410042290
:106F10000B68CDF800B0CDE901024A46D3F800A0D5
:106F200009A86823D0479DE7801A0600D4F80833E3
:106F300013F480773DD15FFA85F90C22494620464B
:106F4000FFF70EF80646002800F08180CDE90677AD
:106F5000079B0A934FF0000A692249462046CDF864
:106F60001CA0FEF7FDFF074600287ED0CDE908AA49
:106F7000099B0B9300221A230BA90AA8099200F07F
:106F800037FF01462046FEF7DBFF0BA8FCF7B6FEF5
:106F900009A8FCF7B3FE17B108A8FCF7AFFE0AA8D2
:106FA000FCF7ACFE07A8FCF7A9FE16B106A8FCF793
:106FB000A5FE94F82330052B3FF45BAED4F80833DC
:106FC00013F480777FF4E9AB5FFA85F90C22494628
:106FD0002046FEF7C5FF0646002855D0CDE90677C6
:106FE000079B0A934FF0000A682249462046CDF8D5
:106FF0001CA0FEF7B5FF0746002853D0CDE908AA2C
:10700000099B0B9300221A230BA90AA8099200F0EE
:10701000EFFE01462046FEF793FF0BA8FCF76EFE3D
:1070200009A8FCF76BFE17B108A8FCF767FE0AA8D1
:10703000FCF764FE07A8FCF761FE16B106A8FCF792
:107040005DFE94F82330052B7FF4A7AB11E6D8F84A
:10705000041004220B68CDF800B0CDE901024A46C5
:107060001F6807A80C23B84772E7D8F80410042259
:107070000B68CDF800B0CDE901024A46D3F800A074
:1070800009A86923D04773E7D8F8041004220B68D5
:10709000CDF800B0CDE901024A461F6807A80C23CD
:1070A000B8479DE7D8F8041004220B68CDF800B06B
:1070B000CDE901024A46D3F800A009A86823D047C9
:1070C0009EE7D4F8083313F0200A24D15FFA85FB39
:1070D0001C2259462046FEF743FF064608B3CDE979
:1070E00008AA0022099B0B9311460BA8CDE909229F
:1070F00003F030FC01462046FEF722FF0BA8FCF708
:10710000F3FD0AA8FCF7F0FD09A8FCF7F7FD16B19E
:1071100008A8FCF7F3FD94F82330052B7FF44EAB61
:10712000A7E5D8F8041004220B68CDE90102B84A9B
:107130000092D3F800A05A461C2309A8D047D0E7F4
:10714000D4F8083313F0200A24D15FFA85FB1E22FD
:1071500059462046FEF704FF064608B3CDE908AAC3
:107160000022099B0B9311460BA8CDE9092203F0DD
:10717000F1FB01462046FEF7E3FE0BA8FCF7B4FD49
:107180000AA8FCF7B1FD09A8FCF7B8FD16B108A8DC
:10719000FCF7B4FD94F82330052B7FF420AB68E5B1
:1071A000D8F8041004220B68CDE90102984A009235
:1071B000D3F800A05A461E2309A8D047D0E7D4F838
:1071C000083313F0200A25D15FFA85FB1C225946AB
:1071D0002046FEF7C5FE064610B3CDE908AA099A77
:1071E0000B920023022201210BA8CDE9093303F001
:1071F000B1FB01462046FEF7A3FE0BA8FCF774FD89
:107200000AA8FCF771FD09A8FCF778FD16B108A8DB
:10721000FCF774FD94F82330052B7FF4F1AA28E5E0
:10722000D8F8041004220B68CDE90102784A0092D4
:10723000D3F800A05A461C2309A8D047CFE7D4F8BA
:10724000083313F0200A25D15FFA85FB1E22594628
:107250002046FEF785FE064610B3CDE908AA099A36
:107260000B920023022201210BA8CDE9093303F080
:1072700071FB01462046FEF763FE0BA8FCF734FDC8
:107280000AA8FCF731FD09A8FCF738FD16B108A8DB
:10729000FCF734FD94F82330052B7FF4C2AAE8E410
:1072A000D8F8041004220B68CDE90102584A009274
:1072B000D3F800A05A461E2309A8D047CFE7D4F838
:1072C000083313F0400A21D15FFA85FB0C2259469E
:1072D0002046FEF745FE0646F0B1CDE909AA0A9B15
:1072E0000022CDE90A23012106220BA800F046FD69
:1072F00001462046FEF724FE0BA8FCF7FFFC0AA877
:10730000FCF7FCFC16B109A8FCF7F8FC94F8233054
:10731000052B7FF497AAACE4D8F8041004220B687C
:10732000CDE901023A4A0092D3F800A05A460C2354
:107330000AA8D047D3E7D4F8083313F0400A20D185
:107340005FFA85FB0C2259462046FEF709FE0646E9
:10735000E8B1CDE909AA00220A9B11460BA8CDE9A4
:107360000A2300F00BFD01462046FEF7E9FD0BA8BD
:10737000FCF7C4FC0AA8FCF7C1FC16B109A8FCF78D
:10738000BDFC94F82330052B7FF46DAA71E4D8F886
:10739000041004220B68CDE901021D4A0092D3F8C3
:1073A00000A05A460C230AA8D047D4E7D4F80833E3
:1073B00013F0800A26D13B78F1B21A462046CDE977
:1073C0000413FEF7CDFDDDE90413814610B3CDE9CA
:1073D00009AA0A9B0022CDE90A2301210C220BA84D
:1073E00003F086F901462046FEF7AAFD0BA8FCF73C
:1073F00085FC0AA8FCF782FCB9F1000F02D009A8AD
:10740000FCF77CFC94F82330052B7FF440AA30E491
:10741000801A0600D8F80400B84AD0F800E00092BC
:107420004FF0040CCDE9019C0A46DEF800A00146AD
:107430000AA8D047CDE7D4F8083313F0800A26D144
:107440003B78F1B21A462046CDE90413FEF788FDD9
:10745000DDE90413814608B3CDE909AA0A9B00229D
:10746000CDE90A2300210C220BA803F041F90146C3
:107470002046FEF765FD0BA8FCF740FC0AA8FCF7C8
:107480003DFCB9F1000F02D009A8FCF737FC94F8D5
:107490002330052B7FF40BAAFFF7EBBBD8F80400D1
:1074A000964AD0F800E000924FF0040CCDE9019C20
:1074B0000A46DEF800A001460AA8D047CEE7D4F875
:1074C000083313F4004A20D15FFA85FB0C22594699
:1074D0002046FEF745FD0646F0B1CDE909AA0A9B14
:1074E000002201210BA8CDE90A2302F077FF014613
:1074F0002046FEF725FD0BA8FCF700FC0AA8FCF7C8
:10750000FDFB16B109A8FCF7F9FB94F82330052B15
:107510007FF4E3A9FFF7ADBBD8F8041004220B6891
:10752000CDE90102754A0092D3F800A05A460C2317
:107530000AA8D047D3E7D4F8083313F4004A20D17F
:107540005FFA85FB0C2259462046FEF709FD0646E8
:10755000F0B1CDE909AA00220A9B11460BA8CDE99A
:107560000A2302F03BFF01462046FEF7E9FC0BA888
:10757000FCF7C4FB0AA8FCF7C1FB16B109A8FCF78D
:10758000BDFB94F82330052B7FF4B8A9FFF771BB3E
:10759000D8F8041004220B68CDE90102574A009282
:1075A000D3F800A05A460C230AA8D047D3E7D4F852
:1075B000083313F4007A20D15FFA85FB3022594654
:1075C0002046FEF7CDFC0646F0B1CDE909AA0A9B9C
:1075D000002201210BA8CDE90A2303F087FC014614
:1075E0002046FEF7ADFC0BA8FCF788FB0AA8FCF7C9
:1075F00085FB16B109A8FCF781FB94F82330052B15
:107600007FF48DA9FFF735BBD8F8041004220B686E
:10761000CDE90102394A0092D3F800A05A4630233E
:107620000AA8D047D3E7D4F8083313F4007A20D15E
:107630005FFA85FB302259462046FEF791FC06464C
:10764000F0B1CDE909AA00220A9B11460BA8CDE9A9
:107650000A2303F04BFC01462046FEF771FC0BA801
:10766000FCF74CFB0AA8FCF749FB16B109A8FCF78C
:1076700045FB94F82330052B7FF462A9FFF7F9BA94
:10768000D8F8041004220B68CDE901021B4A0092CD
:10769000D3F800A05A4630230AA8D047D3E7D8F839
:1076A000041004200A68CDE9016014480090D2F863
:1076B00000A009A84A46D047FFF774B9D8F80410CB
:1076C00004200A68CDE901600C480090D2F800A0BF
:1076D00009A84A46D047FFF7ADB9D8F804100422EC
:1076E0000B68CDE90102054A0092D3F800B04A4682
:1076F0002B460AA8D847FFF7E1B900BF801A060059
:10770000D8F8041004220B68CDE901020C4A00925B
:10771000D3F800B04A462B4609A8D847FFF70FBA5E
:10772000D8F8041004220B68CDE90102044A009243
:10773000D3F800B04A462B4609A8D847FFF743BA0A
:10774000801A060073B50446FEF7CCFF94F8233088
:10775000052B32D0002594F83F33EB40DA07E9B22D
:1077600016D40135082DF6D194F82330052B24D0FA
:1077700094F8203013B194F82230F3B9104B11492A
:107780001B68986903681B6802B0BDE87040184721
:10779000D4F808339B030CD42C200191FEF714FA83
:1077A000064610B1019903F019FC31462046FEF758
:1077B000C7FB94F82330052BD3D102B070BD00BFB6
:1077C000CC25002078F108082DE9F04F90F9213000
:1077D00089B00446002B00F00481012300F50C75EC
:1077E00080F84133024600F50F712B462E46D06ECD
:1077F000002859D0002384F8413394F94030642B99
:107800005BD094F9BC30642B00F08D8094F9383152
:10781000642B00F08A80D4F830722FBB01A9204677
:1078200029F002FF00B30C230593012306978DF87E
:107830001830714B07936946BDF80430049704A8CB
:10784000ADF810308DF800702AF0C0F89DF90010E6
:1078500051B1022908DC38B1C9B27C2303FB0141D4
:107860006C3128462BF0BEFA94F841B3BBF1000FFF
:107870005DD0E36E6367D4F8E830C4F8F030D4F834
:107880006431C4F86C3194F8233003F1C30204EB83
:1078900082020021042B7CD852F8040B10610133C2
:1078A00042F8041CDBB2F5E753F8040B0028A1D121
:1078B0008B4202F17C029AD19FE7002066238DF86B
:1078C00010307C2303FB004004A940302BF0CEF99C
:1078D00004A9204629F0A8FE00289CD004238DF896
:1078E00018300023CDE90133039331230593694612
:1078F00004A82AF06BF8059B28B108AA02EB8302C2
:10790000009942F8E01C0133332B0593EFD94AF07C
:10791000ADFC9DED031ADDED020A9DED010A662125
:107920004AF062FC77E70120C8E70220C6E701279A
:10793000A94655F8043B23B1AB600137042FF7D1BA
:1079400097E7AA46B8465FFA88F3022BF5D8DAF82B
:10795000002055F8043C9A4205D104A95046CDF8C0
:1079600010B02BF03FFA5AF8043B08F101020BB9B2
:107970009046E8E704A906EB88000193CDF810B023
:107980002BF030FA019BAB6001A948462BF02AFA94
:10799000D3E794F8413313B92046FEF7DDF994F8A4
:1079A00022300BB3154B1B68986A036864215B682F
:1079B00098472046FEF7A0FD94F83E3003B9E366F1
:1079C00094F8BA300BB9C4F8E83094F836310BB9F2
:1079D000C4F86431F9F7B0FDF9F738FE0123A4F8D3
:1079E000403309B0BDE8F08F2046FFF7ABFE94F8B6
:1079F0002230002BE0D0D5E7D8860908CC2500201E
:107A00007047000001207047012070474368986864
:107A10007047000010B5054B03600446806A10B142
:107A200003685B689847204610BD00BF3CF6080815
:107A3000406803685B6A184733B46C46406884E862
:107A40000C0003689D6A94E80C00AC4602B030BCA0
:107A50006047000010B50446FFF7DCFF2046FEF744
:107A6000BBF8204610BD000040680AF0A5BC00002D
:107A7000406801230AF0A0BC40680AF079BC00000D
:107A800040680A220AF01EBC40680AF033BC0000BD
:107A900040680AF0B5BC000090F82E2022B190F8A2
:107AA0002D10002201F06EB97047000073B5044636
:107AB00005250026A06A8DF8076003680DF107020E
:107AC000DB680121984778B19DF807300C2B09D06D
:107AD000102B05D0092B07D184F8303002B070BDCF
:107AE0001523F9E71423F7E7013DE3D12846F5E72D
:107AF00010B4806A03681C690822A44601235DF85B
:107B0000044B31216047000010B4806A03681C698F
:107B10000122A44600235DF8044B32216047000097
:107B2000F0B50446806A036885B05B6998470546EE
:107B3000002800F08480A06A03685B6998470368A6
:107B40009B689847A06A03689B69984760B93D4B5A
:107B50003D491B68986903681B6898472B6828464D
:107B6000DB689847002667E02046FFF7CDFF002836
:107B7000F4D02046FFF79AFF0028EFD0A06A0368F0
:107B80000121DB6A98472046FFF7B2FF30B92D4B41
:107B90002E491B68986903681B68DEE7A06A0368C2
:107BA000DB69984730B9274B29491B6898690368F6
:107BB0001B68D2E7A06A94F83010012784F82E7071
:107BC00003685B6A9847A06A03689B6A984704F158
:107BD0002D020146204601F023F906460028BDD0BB
:107BE000A06A94F82D10036801919B6A9847019947
:107BF0000246204601F018F994F82C302BB194F885
:107C00002D103A46204601F023F994F82F2094F8DD
:107C10002D10204601F03EF92B682846DB68984776
:107C2000A06A029403681D6A0A4B039304AB13E92C
:107C30000C0042F21071A847304605B0F0BD064670
:107C4000FAE700BFCC250020A8F50808CEF5080803
:107C5000EDF508084D7D010870B5002586B0CDE929
:107C6000005500230446806A8DF80850059303935D
:107C7000049303686A469E6810210923B047A0B1A7
:107C80009DF8003013F0010615D194F8313001331E
:107C9000DBB2052B84F8313007D12046FFF734FFE3
:107CA0002046FFF725FF84F83160A06A03681B6B4C
:107CB000984706B070BD9DF8083084F831501B0716
:107CC000F3D4BDF901309FED1F6A06EE903ABDF97D
:107CD000033007EE103ABDF90530F8EEE66A07EE1C
:107CE000903ACDED036AF0EEE66AB8EEC77AF8EEA8
:107CF000E77AF4EEC66AF1EE10FA8DED047ACDED76
:107D0000057A0DD5B0EEC77AB4EEC67AF1EE10FA68
:107D100006D5F0EEE77AF4EEC67AF1EE10FAC4D4A6
:107D20009FED090A03A810F09BF9B2EE040A03A81C
:107D300010F096F994F82D200A2303A9204601F0AB
:107D40000FF9B2E7000000349A99193EFFF784BF9B
:107D500010B5044B044640F8043BFBF7CFFF204628
:107D600010BD00BF54F6080810B50446FFF7F0FF39
:107D70002046FDF731FF204610BD0000F7B503682F
:107D80000F4616461BB90024204603B0F0BD002460
:107D9000046008200193FDF717FF054620B1124B40
:107DA0000360019B4360019401A8FBF7A7FF002D2E
:107DB000E9D03420FDF708FF04460028E3D000F0A6
:107DC000E1FE0A4BA562236084F82C7084F82F60D2
:107DD0002046FFF7A5FE05460028D5D1236820469A
:107DE0005B6898472C46CFE754F608083CF608082D
:107DF0002DE9F74F046806460D4690469946002C3B
:107E00006CD00B68002B49D0236820465B6A9847EA
:107E100003689B689847012328680DEB0302002143
:107E20000AF0CAFA98B39DF80130EA2B2FD1DFF897
:107E3000F0B04FF0060A28680023802206210AF0DD
:107E400097FA20B3DBF80070B86A03680A215B6810
:107E50009847002328681A4606210AF089FAB0B12B
:107E6000B86A03680A215B689847012328680DEB0C
:107E7000030206210AF0A0FA48B19DF8014014F06F
:107E800040042FD00AF1FF3A1AF0FF0AD3D130682C
:107E900003685B6A98470368DB68984700241DE025
:107EA000022223460F2128680AF062FAB86A0368A2
:107EB00001215B689847306803685B6A98470368EC
:107EC000DB689847336834604A46414601A801930D
:107ED000FFF754FF044601A8FBF710FF204603B04C
:107EE000BDE8F08F224623460F2128680AF040FAA9
:107EF000B86A036801215B6898470223214630680D
:107F00000DEB03020AF058FA04460028C8D0B869FD
:107F1000024903681B689847B9E700BF14F60808D0
:107F2000CC25002090F82C10002200F02BBF000080
:107F300070B504468CB00426013E76B2731C4AD05C
:107F4000A06A15236A465D210AF036FA0028F3D0AC
:107F5000A06A152306AA5D210AF02EFA054600281C
:107F6000EAD0152206A968466EF092F90028E3D1FE
:107F70009DF8003084F82E309DF8073084F83030BA
:107F80009DF8143084F83A309DF813309DF8102095
:107F900084F83B309DF80F3043EA0223A3879DF815
:107FA000013084F82F309DF8083084F83130039B7D
:107FB0009DF80C20C3F30F2363869DF80B3043EA32
:107FC0000223A386049BC3F30F23E386019BC3F321
:107FD0000F23238707E0054B05491B689869036851
:107FE0001B689847002528460CB070BDCC250020A2
:107FF00088F608082DE9FF4104460023806A8DF8C1
:1080000007300368DFF868815B6A984703689B68FC
:108010009847A06A03680A219B6C9847A06A0A22C5
:1080200004210AF04FF90425013D6DB26B1C32D0DA
:1080300000234B21A06A82220AF09AF9D8F8006046
:108040000746B06A036802215B689847002FEBD0AF
:1080500001231A464B21A06A0AF08AF90746B06A42
:10806000036802215B689847002FDDD0A06A0123D6
:108070000DF1070240210AF09FF90028D4D09DF8A5
:108080000720322A10D0002DCED1B06936490368BE
:108090001D683223A847A06A03685B6A9847036893
:1080A000DB68984700255BE02046FFF741FF00288A
:1080B000F1D0A06A0123172251210AF059F90028B2
:1080C000E9D05222A06A012311460AF051F9002892
:1080D000E1D0A06A012338224C210AF049F9002896
:1080E000D9D0A06A03685B6A98470368DB68984741
:1080F000A06A05210AF0FEF8A36A04F12C0299682F
:10810000204600F08DFE054650B3A36A94F82C106B
:108110009A68204600F088FE94F8442094F82C10C9
:10812000204600F0B7FE94F845302BB194F82C109F
:108130000122204600F08CFEA06A036802219B6C9D
:108140009847A06A029403689E6A084B039304ABA5
:1081500013E90C0044F21B11B0474CF0DFF9206426
:10816000284604B0BDE8F081B0F60808DD820108B9
:10817000CC25002070B5858F90F93B60AD03B5FB31
:10818000F2F2A2F5804404FB04F2D51190F83A20F3
:108190000498D201624306FB05225212A03002F578
:1081A0008012424312134A43DB0003EB623000B2F9
:1081B00070BD000010B5448E53005C43B0F93830F8
:1081C000C91A838FD31AB0F93620B0F9340053435B
:1081D00004F500449B10C3EBC13300EB2440044979
:1081E00093FBF0F04FF400420DF0EEFE00B210BD34
:1081F0000080FFFF10B52DED028B8AB004460823E6
:10820000806A05AA42210AF0D7F818B1BDF81A20F1
:10821000D30719D4A06A0AF0F3F84CF07FF9236C65
:10822000C31AFA2B0CD92064002382224B21A06AA6
:108230000AF09EF80123A06A1A464B210AF098F82A
:108240000AB0BDEC028B10BDBDF9141094F93030AA
:108250000093920894F92E300392C9102046FFF73C
:1082600089FFBDF9161094F93130039A009308EE96
:10827000900A94F92F30C9102046FFF77BFFBDF913
:108280001810039A491008EE100A2046FFF792FFD3
:1082900007EE900AF8EEE88AF8EEE77AB8EEC88AB8
:1082A000B3EE000A07A8CDED097ACDED078A8DED72
:1082B000088A0FF0E9FEB2EE040A07A80FF0D0FE1C
:1082C0004CF02CF994F82C2020640A23204607A9AE
:1082D00000F046FEA06A0AF093F8B1E7FFF78ABF04
:1082E000F7B503680D4616461BB90024204603B0B7
:1082F000F0BD002707604820CDE90073FDF764FC5E
:10830000044650B100F03EFC0E4B2360019BA3627B
:10831000019784F8446084F8455001A8FBF7E4FC19
:108320006846FBF7E1FC002CDFD02046FFF762FE39
:1083300005460028DAD1236820465B6898472C461A
:10834000D4E700BFE8F6080810B5044B044640F82F
:10835000283BFBF7C9FC204610BD00BFE8F6080823
:1083600010B50446FFF7F0FF2046FDF735FC204628
:1083700010BD000090F82C10002200F003BD00009A
:10838000F8B504460D4617461E4600F0FBFB094BA8
:1083900023602B68A362002200232A6084F82D70DA
:1083A00084F82E6023656365A365E36523666366D1
:1083B0002046F8BD00F70808F8B51C4609331646F4
:1083C000DB086A46A2EBC30300AF9D46806AA31C8C
:1083D0006A4609F0F1FF054628B122460DF1020177
:1083E00030466DF065FF2846BD46F8BD2DE9F341E6
:1083F00006460F4614464CF091F8114BD3F8008016
:108400000546D8F82800036801215B6898470123D6
:108410000DF1070207213046FFF7CEFF60B19DF84E
:108420000730DA0702D4B7EB531F05D04CF076F8CB
:10843000431BA342E5D3002002B0BDE8F08100BF9A
:10844000CC2500202DE9F041DFF8608292B004468F
:1084500002AF002646F02002A06A0023D2B25021CB
:1084600009F086FF002800F00C810325013D6DB264
:108470006A1C00F00681D8F80030986A03684FF44F
:1084800096719B68984701230DF1060255212046FD
:10849000FFF792FF002800F0F4809DF8063013F0FB
:1084A000E00F40F0EE80DB07E0D502230DF106027D
:1084B00052212046FFF780FF002800F0E280BDF83F
:1084C000063001365BBA202E27F8023BC2D1BDF838
:1084D00024309DF826109FED6D7ADFED6D6A9FEDDB
:1084E0006D6A43F30B0207EE902A1B0903F47063D5
:1084F000BDF82620F8EEE77A0B4343F30B03C4EDF7
:108500000C7A07EE903A02F470639DF82820F8EE9A
:10851000E77A134343F30B03C4ED0D7A07EE903A69
:108520009DF92230F8EEE77AC4ED0E7A07EE903A24
:108530009DF92930F8EEE77A67EE877A07EE103A70
:10854000B8EEC77A9DF92A30C4ED0F7A27EE267A65
:10855000DFED517A84ED107A07EE103AB8EEC77A63
:108560009DF92B30E7EE267AC4ED117A07EE903AAA
:10857000F8EEE77A9DF9233067EEA67ADFED476AD9
:10858000C4ED127A07EE903A9DF92C3007EE103ABE
:10859000B8EEC77A9DF92E3027EE267AF8EEE77A04
:1085A00084ED147A67EE867A07EE103A9DF9303042
:1085B000C4ED137A07EE903AF8EEE77A9DF92D3084
:1085C00067EEA67AB8EEC77AC4ED167A27EE267A59
:1085D00007EE903A84ED157AF8EEE77A9FED307A5F
:1085E0009DF92F3067EE877AC4ED177A07EE903A3F
:1085F0009DF93130F8EEE77A06EE903A67EE877A29
:10860000F8EEE66AC4ED187ADFED267ABDF9383067
:10861000E6EE877A07EE103A9DF93230C4ED197A0A
:10862000B8EEC77AF3EE077AE7EE067A07EE103A6D
:10863000DFED1D6AC4ED1A7AB8EEC77A27EE267A06
:1086400084ED1B7A9DF9333007EE103AB8EEC77A05
:108650009DF9343027EE267A84ED1C7A07EE103A25
:108660009DF9353007EE903AB8EEC77AF8EEE77A22
:1086700027EE267A67EEA67A84ED1D7AC4ED1E7A7F
:1086800000E0002012B0BDE8F08100BFCDCC4C3E30
:108690000000803B0000003B0AD7233C0000003D67
:1086A0000000803817B7D1B80AD7A33ACC250020EC
:1086B00073B501230E460DF1070206210446FFF7AC
:1086C0007BFE18B90025284602B070BD9DF8073022
:1086D000013B012B0CD80023A06A1A46062109F0A1
:1086E00047FE0028EED0062200212046FFF77EFE3E
:1086F000A06A00233246062109F03AFE054600280A
:10870000E0D0262231462046FFF770FEDBE700006E
:1087100013B501230DF1070207210446FFF74CFEB4
:1087200010B9002002B010BD9DF807301B070CD512
:108730000023A06A1A46062109F01AFE0028F0D08C
:10874000062200212046FFF751FEA06A00230722DF
:10875000062109F00DFE0028E3D013220721204650
:10876000FFF744FE0028DCD0A06A00230522062182
:1087700009F0FEFD0028D4D0172205212046FFF77E
:1087800035FE0028CDD001212046FFF791FFC9E733
:10879000F7B50446806A5B4F03685B6A98470368D5
:1087A0009B689847A06A03680A219B6C9847A06A57
:1087B0000A22042109F086FD0525013D6DB26B1CDE
:1087C00000F09680A06A0023B6227E2109F0D0FD39
:1087D0000028F2D03B68986A036818215B686E46EF
:1087E00098470123324600212046FFF7E5FD002887
:1087F000E3D09DF80030332BDFD12046FFF722FE77
:10880000002875D0A06A00238022502109F0B0FD15
:1088100000286DD02046FFF77BFF002868D0A06AB3
:10882000002386222E2109F0A3FD002860D0A06A33
:1088300000232422042109F09BFD002858D0A06ABF
:1088400000230222062109F093FD002850D01422B3
:1088500002212046FFF7CAFDA06A00230722052156
:1088600009F086FD002843D001212046FFF720FFB4
:1088700000283DD0A06A036803219B6C9847A06A3A
:1088800003685B6A98470368DB689847A06A17210A
:1088900009F030FDA36A04F12C029968204600F02B
:1088A000BFFA054608B3A36A94F82C109A682046CC
:1088B00000F0BAFA94F82E2094F82C10204600F01C
:1088C000E9FA94F82D302BB194F82C1001222046AF
:1088D00000F0BEFAA06A03689F6A0B4B00940193F4
:1088E00096E80C0042F21071B847284603B0F0BD7C
:1088F000A06A03685B6A98470368DB6898470025AD
:10890000F3E700BFCC250020018B010810B586B02D
:108910000C236A4631210446FFF74EFD002800F083
:10892000DF809DF801309DF80020DFED717ADFEDEA
:10893000715A1B0403EB02239DF8022003EB026330
:108940001B1206EE903A9DF804309DF803201B049C
:1089500003EB02239DF8052003EB02631B1207EED5
:10896000103A9DF807309DF806201B0403EB022304
:108970009DF8082003EB02631B1206EE103A9DF8E7
:108980000A309DF809201B0403EB0223F8EEE66A87
:10899000B8EEC77A9DF80B2066EEA76A27EE277A15
:1089A000B8EEC66ADFED547A03EB02631B1226EEC3
:1089B000276A07EE903AF8EEE77A67EEA57AF5EEC9
:1089C000C07AF1EE10FA40F38D80DFED4C5A77EE6D
:1089D000E57AD4ED134A94ED0F5A94ED1C4AD4ED88
:1089E0001D3A94F82C20F7EE005A74EEA54AF0EEEA
:1089F000632AA4EEA75A0A2303A9D4ED107AD4ED72
:108A00000C4A77EEA57A2046E7EEA64AD4ED1A7A0C
:108A100075EE677A94ED145AF0EE646AD4ED174A55
:108A2000E5EE276AB0EE655AA7EEA45AC6EE854A6F
:108A300094ED115AD4ED0D6A35EE255AE5EE076A2C
:108A400094ED157AE7EE876A94ED187AB0EE655AE0
:108A5000A7EE875A86EE857A94ED125AD4ED0E6A07
:108A600035EE255AE5EE066A94ED166A94ED195A2C
:108A7000E7EE866AB0EE656AA7EE856AF0EE657A83
:108A800086EE863A94ED1B6AF0EE646AE6EE447A6E
:108A9000E6EE476A86EEA75AF0EE476AE4EE646AAD
:108AA000C6EEA75AD4ED1E6AD4EE262AE6EE636A15
:108AB000B2EE046A27EE667A65EE066AA2EEA47A42
:108AC000CDED036A65EE866ACDED046AC7EE276ACE
:108AD00076EE837A67EE867ACDED057A00F040FA7D
:108AE00006B010BD44BFDFED055A77EEA57A70E7FA
:108AF00047ABE73B5B9E803AF61BEB3B85EBCB41FC
:108B0000FFF704BF30B51346026885B00D461AB9A9
:108B10000024204605B030BD002101607C20019377
:108B20000392FDF751F8044620B1019B2A4603A9A0
:108B3000FFF726FC03A8FBF7D7F8002CE8D0204667
:108B4000FFF726FE05460028E3D1236820465B6830
:108B500098472C46DDE7000010B5044B044640F86A
:108B6000283BFBF7C1F8204610BD00BF00F70808FE
:108B700010B50446FFF7F0FF2046FDF72DF820461C
:108B800010BD0000064B10B503600446FDF7A4FDC0
:108B9000606004F108004AF01FFE204610BD00BFCF
:108BA00018F7080873B50646144675687C2303FB5E
:108BB0000253C4EB441405EB8404084693F8A41054
:108BC00001900FF0E3FA94F93C3001983BB97368D7
:108BD00093F8251002B0BDE870400FF0D7BA94F8B2
:108BE0004010F7E737B5446801917C2505FB024545
:108BF00095F83F3004EB8304D4F84C325BB14BF072
:108C00008DFCC5F89C000199D4F84C0203B0BDE876
:108C1000304003F079BE03B030BD00002DE9F04FC5
:108C2000C2EB421447684FEA840881460E4607F1BA
:108C30003C0B08F108018BB01546594430460FF043
:108C4000DBF9D9F8040029460BEB8404FDF7EAFCB4
:108C500038B17C2303FB057393ED1A0A30460FF0FD
:108C6000FFF97C2303FB057393ED146ADFED3A7A79
:108C7000D3ED156AB0EEC67AB4EEE77AF1EE10FAEB
:108C80000FD5B0EEE67AB4EEE77AF1EE10FA08D539
:108C900094ED077AB0EEC77AB4EEE77AF1EE10FA07
:108CA0001BD47C2303FB0573D86D196E5A6E9B6D24
:108CB000029003910490079101A831468DED016A5D
:108CC000CDED056A0692089209930DF047FB86EDFB
:108CD000000AC6ED010A86ED021A7C2303FB057724
:108CE0000023C7F88C30C7F88830C7F88430D9F82B
:108CF000040090F95C3208F13C0A08F14808DA44B3
:108D0000D84463B15DB9414600F5167004F0B4FA79
:108D1000414630460BB0BDE8F04F0FF06DB990F909
:108D20003430012B0BD190ED0E0A50460FF044F970
:108D300084ED120AC4ED130A84ED141AE8E7022B3D
:108D4000E6D1FBF75DFD002201A9FBF759FA0028E7
:108D5000DED09DED010AE8E70000003410B543685D
:108D60007C2404FB023407C904F1900383E8070064
:108D70004BF0D4FBC4F89C004BF0C6FBC4F8A00039
:108D800010BD0000F0B5074685B00D46164600F14F
:108D90000801A92203A809F069FD7C687C2303FB74
:108DA0000543D3F8B42022B903A809F081FD05B02A
:108DB000F0BDBEB196ED007AD3ED2A7A67EE877AE0
:108DC000C3ED2A7A96ED017AD3ED2B7A67EE877A96
:108DD000C3ED2B7A96ED027AD3ED2C7A67EE877A83
:108DE000C3ED2C7A7C2607EE902A06FB0541A831BC
:108DF000B8EE670A084601910FF046F901992A4634
:108E00003846FFF7ABFF06FB05410023C1F8B03041
:108E1000C1F8AC30C1F8A8300023C1F8B430C3E7C2
:108E20004068FCF7E9BF0000F7B5064640680192CC
:108E30007C2707FB01000D466C3001A9144629F080
:108E4000B1FF716807FB05152C6703B0F0BD00008A
:108E500007B540687C2303FB010393F93C30022BE8
:108E60000BD000F13C03C1EB411003EB80000DF18E
:108E700007018DF8072029F0EFFE03B05DF804FB31
:108E800043687C2202FB013191F93C00003818BF95
:108E90000120704743687C2000FB013181F8A42049
:108EA00070470000F8B5054608460F460FF04AF92E
:108EB00010B100242046F8BD38460FF029F90446C9
:108EC0000028F6D16B6893F934637EB138460FF011
:108ED00071FC95ED087ADFED1F7AF0EEC76AF4EECB
:108EE000E76AF1EE10FA03D585ED080A0124E1E7FF
:108EF00077EE407A30EE076AF0EEE77AC7EE866AE0
:108F0000F6B207EE906A9FED146AF8EE677A26EEE5
:108F1000866AF4EEC67AF1EE10FA48BFB2EE046A41
:108F2000DFED0E7A45BF6B6A66EE866AB0EE676A61
:108F300087EEA66A46BF01336B620124F7EE007A22
:108F400077EEC67A20EE060AA7EE270A85ED080A14
:108F5000B0E700BF0000003400004843CDCCCC3D5A
:108F60002DE9F74304460E4615461F46FFF71AFE45
:108F70002A4631462046FFF735FE314620462A462E
:108F8000FFF74CFE31462046FFF78CFF28B39B22AB
:108F900004F1080101A809F069FC64684FF07C093C
:108FA00009FB054808F1A808314640460FF024F8AF
:108FB00009FB0542D2F8B4100131C2F8B4104FB128
:108FC000B94207D34908C2F8B410B0EE000A4046CF
:108FD0000FF05AF801A809F06BFC03B0BDE8F0836C
:108FE00010B50446FCF792FFC0B23C34C0EB401011
:108FF00004EB800010BD0000F8B50A4E044600F5F1
:10900000167704F5137555F8040B08B103F0B0FF9B
:10901000BD42F8D13368986A036801215B689847BC
:10902000EFE700BFCC25002008B5FFF7E5FF000003
:10903000F0B5144E00EB810773780446D7F84C0264
:109040006FF3410387B00D467370C8B102F07EFB29
:1090500068B1737843F0100373702C440023A3723B
:10906000D7F84C0207B0BDE8F04002F0F3BAD7F8E9
:109070004C12684602F09AFB009B012BEDD1E8E709
:1090800007B0F0BDD45A002070B506460D46002446
:1090900045FA04F3DB07E1B202D53046FFF7C8FF1B
:1090A0000134032CF4D170BDFF21FFF7EDBF0000A8
:1090B00030B500F5137587B000F5167455F8041B2C
:1090C00021B9A542FAD1002007B030BD684602F0B0
:1090D0006DFB009B013B022BF3D80120F4E700005D
:1090E0002DE9F0472DED028B88B004460D469046E1
:1090F000B0EE408AFDF7DEF930B90026304608B000
:10910000BDEC028BBDE8F08729462046FDF74CF800
:1091100006460028F1D004EB8507D7F83C22D7F8A3
:1091200030329A4206D035F0C5FC5C4A03212EF05D
:10913000D1FEE2E7D7F84C3283B94FF49870FCF7D0
:1091400043FD814608B103F017F8C7F84C92B9F116
:10915000000F03D135F0AEFC514AE7E7B4F84A32CC
:10916000D90711D505F078FE90F8082390F8C4329D
:1091700032B9B02202FB030090F8A130012B03D8D2
:1091800035F098FC474AD1E72046FFF791FF20B918
:10919000454A537843F00203537094F9353053B382
:1091A00029462046FFF71CFF90F90030002B53D0D2
:1091B00029462046FFF714FF90F80490B9F12B0FD1
:1091C00019D829462046D7F84CA2FFF709FF94F991
:1091D000353090F90020022BD4BF00210121012B52
:1091E000D4BF00230123003A009118BF0122494651
:1091F000504602F043FA631900229A7275B3D4ED17
:10920000C10AB4F84822D7F84C0270EEA00A2B46E7
:10921000B0EE480A414602F051FA94F83E33002B72
:1092200031D1224A069412680127E773906A0268D6
:10923000156D1F4A0792029309224FF40063CDE98E
:10924000003208AA12E906001A4BA847C8B935F03F
:1092500031FC194A02216AE79946B2E729462046BD
:10926000FFF7BEFE90F90030002BC8D0D4EDC10A44
:10927000B4F84822D4F84C022B46B0EE480A4146D6
:10928000C9E784F83E7300230DF1170104F12400AF
:109290008DF8173029F0EAFC30E700BF28F70808FE
:1092A0005AF708087DF70808D45A0020CC2500207A
:1092B000299001089BF70808A6F708082DE9F04156
:1092C0002DED028B002443739DF8203083730546F7
:1092D0000F469046B0EE408A264647FA04F3DB0775
:1092E000E1B210D5B0EE480A42462846FFF7F8FE34
:1092F000064640B939462846FFF7C6FEBDEC028B4C
:109300003046BDE8F0810134032CE6D1F6E70000D9
:10931000F8B500242DED028B05460F46B0EE408ACD
:10932000427383732646E1B2B0EE480A3A462846B5
:10933000FFF7D6FE0134002818BF0646032CF2D1F1
:10934000BDEC028B3046F8BDF0B500EB81030D4655
:10935000D3F84C129BB0044611B900201BB0F0BDED
:109360000BA802F007FA6319987A0028F6D10B9A35
:10937000002A48D0042AF0D101229A720DAA07CA05
:1093800002AB83E8070010AA07CA05AF87E8070009
:1093900013AA07CA9DED180A08AE86E807001A4608
:1093A000294620468DED010AFCF792FE3A462946F1
:1093B0002046FCF739FE324629462046FCF746FE99
:1093C0009DED010A29462046FCF752FE9DF86430C7
:1093D00083B129462046FFF703FE90F900304BB1D8
:1093E00094F93530012B05DD9DF85D202946204696
:1093F000FCF786FE2046FFF75BFE20B9034A537850
:1094000043F0040353700120A8E700BFD45A0020A2
:109410002DE9F0410546884600F513770024012622
:1094200057F8043BE1B26BB148FA04F3DB0709D506
:109430002846FFF789FF002857F8040C08BF0026CC
:1094400002F008F90134032CEAD13046BDE8F0817E
:109450002E4B2DE9F04F1F68FB6A93F89C8087B074
:109460000446B8F1000F38D1DFF8A8A000F5137654
:1094700000F1030B054656F8040BA5EB04095FFA4F
:1094800089F9E8B102F04EF928B19AF8013043F0B9
:1094900008038AF8013056F8040C02F057F9F8B9BD
:1094A000637B6BB1AB7A5BB956F8041C684602F07B
:1094B0007DF9009B042B03D149462046FFF744FF6A
:1094C00001355D45D7D1124B204683F81280FFF756
:1094D000EFFD054630B10123237407B0BDE8F08FDE
:1094E0008046EDE7237C002BF7D0A37B002BF4D044
:1094F000B86A03684FF47A715B689847B86A036882
:109500009B6B294607B0BDE8F04F1847CC250020DB
:10951000B55A0020D45A0020F0B5002587B000F5D8
:1095200013762C46012756F8041B41B1684602F019
:109530003DF9009B1BB107FA05F31C43E4B201356A
:10954000032DF0D1204607B0F0BD00002DE9F04F0B
:109550002DED028B03270E7C9FED348A91B00546DA
:109560008846B946AC5D0134E4B2B4FBF9F303EBD1
:109570004303E41AE4B205EB8403D3F84C1209B9AF
:10958000AC554CE003A802F011F9DDF80CB00BF17A
:10959000FF33022BF4D830462FF02AFC82463046A7
:1095A00030F02AFB00F11B039A4508D230462EF01A
:1095B0009BFE002011B0BDEC028BBDE8F08FAC55D6
:1095C000284698F810A0FFF7A7FFDDED057A8DF883
:1095D0003100FCEEE77A9DF810208DF8332017EE6D
:1095E000903A8DF8343006AB03CB1B88ADF83D3094
:1095F0005C221B23CDE90032CDF83500CDF83910BF
:1096000009AABF2150468DED098A8DED0A8A8DED9C
:109610000B8A8DF830408DF832B02FF053FC013FAB
:1096200017F0FF079ED10120C4E700BF0000000033
:109630002DE9F04F0F7CA1B006468846032500EBCC
:10964000070999F805400134E4B20323B4FBF3F3AE
:1096500003EB4303E41AE4B206EB8403D3F84C12A1
:1096600011B989F805400AE011A802F083F8DDF885
:1096700044A0BAF1030F08DCBAF1000FF1DA013DA2
:1096800015F0FF05DDD1012012E0AAF10402032A42
:10969000F5D838462FF0ACFB8346384630F0ACFAAC
:1096A00000F13602934506D238462EF01DFE00200A
:1096B00021B0BDE8F08F89F80540304698F810B029
:1096C000FFF72AFFDDF848E0CDF80CE0DDF84CE0CC
:1096D000CDF810E0DDF850E0CDF814E0DDF854E00E
:1096E000CDF818E0DDF858E0CDF81CE0DDF85CE0DE
:1096F000CDF820E0DDF860E0CDF824E03219DDF8A7
:1097000064E01C9BCDF828E0DDF868E092F80AC020
:109710009DF874109DF87520CDF82CE00E93DDF8BF
:109720006CE01E9B8DF835008DF83C108DF83D20C7
:10973000CDF830E08DF834408DF836A08DF837C084
:109740002422CDF83E303623CDE90032C0212C232F
:1097500003AA58462FF0B6FB91E700007FB58A8B2D
:109760000B464AF2B9518A4205465FD04AF2BA51D5
:109770008A4274D04AF2B8518A420BD1474A1268E1
:10978000D26A92F89C203AB135F094F9444A052106
:109790002EF0A0FB042479E0D3ED007AF5EEC07A38
:1097A000F1EE10FAF6D49FED3F7AF4EEC77AF1EEBF
:1097B00010FAEFDC93ED017ADFED3B6A1C6993ED63
:1097C000030AB0EEC77AB4EEE67A93ED027AFCEEC5
:1097D000E77AB0EEC77AF1EE10FAB4EEE67A17EE59
:1097E000903A54BF01260026F1EE10FA54BF012230
:1097F0000022003C18BF012413F0FF0110D18DEDB1
:10980000030A0292FCF7CCFB9DED030A029A234661
:1098100031462846FFF77CFD0028BBD0002435E008
:10982000134600943246FFF749FDF5E7D3ED007A81
:10983000F5EEC07AF1EE10FAACD49FED1A7AF4EEA0
:10984000C77AF1EE10FAA5DCFCEEE77A17EE903A53
:1098500013F0FF0108BFFF21FFF7DAFDDCE7D3EDCE
:10986000007AF5EEC07AF1EE10FA93D49FED0D7AFE
:10987000F4EEC77AF1EE10FA8CDCFCEEE77A17EE24
:10988000904A14F0FF0404D1FFF70EFC204604B008
:1098900070BD2146FFF7F8FBC0E700BFCC250020D4
:1098A000D8F7080800007F4300000034F0B58BB003
:1098B0000E4614460746FFF793FB543007C884E86A
:1098C000070031463846FFF78BFB90ED057ADFED58
:1098D000267AB0EEC77AB4EEE77AF1EE10FA0546D2
:1098E00011D590ED067AB0EEC77AB4EEE77AF1EED4
:1098F00010FA08D590ED077AB0EEC77AB4EEE77AA1
:10990000F1EE10FA24D431463846FFF769FB016ABC
:10991000426A836AE869D5F814E0D5F818C009905E
:1099200001A8CDF804E0029103920491CDF814C08F
:109930000693079208930CF0BDFE98B1214601A84A
:109940000CF00CFD84ED000AC4ED010A84ED021A4E
:1099500031463846FFF744FB00F1080120460EF07F
:1099600065FB01200BB0F0BD000000342DE9F0478D
:109970002DED048BACB0B0EE608A0546B0EE409A97
:109980000F46F0EE418A9046FCF70AFBDFED8B7A3A
:10999000B0EEC87AB4EEE77AF1EE10FA4BD5B0EE3D
:1099A000E87AB4EEE77AF1EE10FA44D523AC20461B
:1099B000FBF76EFEF7F7C0FD2146F7F79FFB064663
:1099C00058BB05F049FA90F8083390F8C42233B137
:1099D000B02303FB020393F8A130012B07D84FF00B
:1099E000B00909FB020090F8A130022B0BD835F02A
:1099F00061F8734A03212EF06DFA30462CB0BDECAD
:109A0000048BBDE8F08705F027FA90F8C43209FB13
:109A10000300AC300FC884E80F00DDED257A9FED20
:109A2000691AB8EEE78ADDED267AF8EEE78A28EEC5
:109A3000018A68EE818A04AA03A902A8F0EE680AE6
:109A4000B0EE480A03F0D4FC064618B935F032F8F7
:109A50005D4ACFE79FED5D7ADDED027A9FED5C8A8E
:109A6000DFED5C8A8DED068A67EE877A242200217D
:109A700011A8CDED057A8DED078A6CF063FC9DEDA4
:109A8000031ADDED040ADFF858A121EE281A68EE6A
:109A9000E00AB0EE480A11A80CF02CFE05A911A8A6
:109AA0000CF05CFC242200211AA8CDED060A8DEDF5
:109AB000071A8DED050A6CF045FCF7F73DFD90EDBA
:109AC000810A8DED010AF7F737FD29EE281AD0ED4E
:109AD000820A9DED010A1AA80CF00CFE1AA923A80F
:109AE0000CF02AFD05A923A80CF038FC4FF0000962
:109AF0008DED050ACDED060A8DED071A95F8223099
:109B00005FFA89F4A3427FF678AF1FB127FA04F316
:109B1000DB071AD52B1993F92C32B3B1B8F1000F2A
:109B20000DD021462846FCF7C5FC88B934F0C2FFA9
:109B3000294A234603212EF0CDF900265DE7214670
:109B40002846FCF731FB0028EBD109F10109D5E7E4
:109B500008AA214628468DED088A8DED098A8DEDEB
:109B60000A8AFFF7A3FE20B934F0A4FF1B4A23465C
:109B7000E0E708A905A80EF009FA0BAA2146284635
:109B80008DED0B0ACDED0C0A8DED0D1AFCF7A0FA48
:109B90009AE807000EAB83E807001A4621462846DC
:109BA000FCF742FA23AA214628468DED238A8DED43
:109BB000248A8DED258AFCF749FAC6E700000034B7
:109BC000FCF7080895BFD63317F8080800007A4458
:109BD0000000000035FA8E3C2CF8080840F8080810
:109BE00094A40808012070470120704743689868D2
:109BF00070470000406803689B6C184710B5054B20
:109C000003600446806A10B103685B689847204689
:109C100010BD00BF28F90808406803685B6A184750
:109C200033B46C46406884E80C0003689D6A94E88D
:109C30000C00AC4602B030BC6047000010B50446D2
:109C4000FFF7DCFF2046FBF7C7FF204610BD0000F2
:109C5000406808F04FBB0000406808F0ADBB000052
:109C60004068012308F0A8BB4068002308F080BBCF
:109C700090F84420D20705D590F8421000F12C024C
:109C8000FFF780B870470000F8B504461E460F463F
:109C90001546FEF777FF084B23600023E36223633A
:109CA000636394F84430A76265F3410384F843602A
:109CB00084F844302046F8BD28F9080810B50D4B4B
:109CC00083630446806A036898221B6900219847D1
:109CD00070B1A06A036820221B690121984738B13E
:109CE000A06A0368BDE810401B69012202211847E1
:109CF000002010BDC5DC6A3F37B50446806A0368A2
:109D00006A469D6803210623A847D0B1BDF800200C
:109D1000BDF8041052BA95B249BAB5F5704F0BB2FE
:109D200011D013F5805F0ED0BDF802305BBA9DB242
:109D3000B5F5704F07D052425B42A287E187A4F885
:109D4000403003B030BD0020FBE70000806A0368AC
:109D500001221B690221184730B585B00446FFF780
:109D6000CBFF05462046FFF7F1FF6DB3B4F93C3059
:109D700094ED0E0A06EE903AB4F93E3007EE103A32
:109D8000B4F9403007EE903AF8EEE66AB8EEC77ADA
:109D9000F8EEE77A01A8CDED016A8DED027ACDEDFE
:109DA000037A0EF05DF994F842102046FFF768F848
:109DB00018B1022101A80EF0E9F994F842200E230F
:109DC00001A92046FFF7CCF805B030BDFFF7C4BFAE
:109DD00013B5806A036801AA9C680A210323A0477F
:109DE00038B10549032201A86CF052FAB0FA80F0AC
:109DF000400902B010BD00BF60F808082DE9F84323
:109E000000252DED028BDFF888819FED5D8A0446E9
:109E10002E462F46A06A036811221B6900210137D4
:109E2000984700287BD0D8F80090D9F8280003681C
:109E300032215B689847A06A036860221B69012190
:109E4000984700286BD0A06A036801221B69022191
:109E50009847002863D0D9F82800036832215B684E
:109E600098472046FFF748FF002858D00135022FB9
:109E7000EDB256DDB4F93C309FED425A9FED426A97
:109E800007EE903AF8EEE77AC5EE276AF0EEE66A5A
:109E9000F4EEC66AF1EE10FA41DDF4EEC86AF1EEB6
:109EA00010FA3CD5B4F93E30DFED385A07EE903A5F
:109EB000F8EEE77A85EEA77AB0EEC77AB4EEC67A06
:109EC000F1EE10FA2BDDB4EEC87AF1EE10FA26D5D9
:109ED000B4F9403005EE903AF8EEE55AC5EE257A31
:109EE000F0EEE77AF4EEC67AF1EE10FA17DDF4EE52
:109EF000C87AF1EE10FA12D594ED0B6A76EE266A66
:109F00000136C4ED0B6AD4ED0C6A36EE877A84ED27
:109F10000C7A94ED0D7A77EE277AC4ED0D7A192F2D
:109F200002D0052E7FF476AFA06A036810221B6969
:109F300000219847052E18D1D4ED0B6AF1EE047A72
:109F400086EEA77A0120D4ED0C6A84ED0B7A86EEBA
:109F5000A77AD4ED0D6A84ED0C7A86EEA77A84EDAB
:109F60000D7ABDEC028BBDE8F8834FF07E53052DD2
:109F7000E3622363636394BF00200120F1E700BF25
:109F8000CDCCAC3F00002E443333333F000022449D
:109F9000CC250020F0B50446806A036885B05B6973
:109FA0009847054648B9504B50491B689869036863
:109FB0001B689847284605B0F0BD03689B68984722
:109FC000A06A03680A21DB6A9847A06A03689B6954
:109FD000984760B9444B46491B68986903681B68F9
:109FE00098472B682846DB6898470025E2E720461B
:109FF000FFF7EEFE0028F4D02046FFF7FFFE30B951
:10A00000394B3C491B68986903681B68E8E72046A0
:10A01000FFF754FE0028E4D0A06A0368DB69984784
:10A0200030B9314B34491B68986903681B68D7E71E
:10A0300094F84430A06A43F0010384F84430036884
:10A040000321DB6A98472B682846DB68984723681A
:10A0500020469B689847A06A036807215B6A984777
:10A06000A06A03689B6A984704F1420201462046B1
:10A07000FEF7D6FE054600289CD0A06A94F8421050
:10A08000036801919B6A9847019902462046FEF7B2
:10A09000CBFE94F8432094F842102046FEF7FAFED7
:10A0A00094F844309B0705D594F8421001222046CD
:10A0B000FEF7CEFEA06A029403681E6A0F4B03935C
:10A0C00004AB13E90C0043F21541B047064BA06AFC
:10A0D0001B689E6933681F6803689B6A9847084934
:10A0E00002463046B84765E7CC25002064F80808EA
:10A0F0008AF80808B0F80808D5F80808CD9D0108C6
:10A1000003F9080810B5084B0360044600230868EB
:10A1100060600B60037A03F00703022B02D1C021B9
:10A1200008F016FA204610BD40F9080810B5044B97
:10A13000044640F8043BF9F7D7FD204610BD00BFA8
:10A1400040F9080810B50446FFF7F0FF2046FBF77A
:10A1500043FD204610BD0000F7B503680E461746C4
:10A160001BB90024204603B0F0BD00220260082085
:10A170000193FBF729FD054610B101A9FFF7C2FFC6
:10A1800001A8F9F7B1FD002DEBD04820FBF71CFD2D
:10A1900004460028E5D029463B463246FFF774FDC9
:10A1A0002046FFF7F7FE05460028DBD1236820464E
:10A1B0005B6898472C46D5E790F82D100022FEF7F3
:10A1C000E1BD0000F0B50446806A036889B05B6AAF
:10A1D000984703689B689847A06A03680A219B6CAC
:10A1E0009847A06A01230DF11702002108F0E4F856
:10A1F000002838D09DF81730082B34D14E4F052554
:10A2000000230122A06A322108F0B2F83B689B6A61
:10A210001A68526840B90A2118469047013D15F066
:10A22000FF05EDD145481CE018461421904706AEC5
:10A23000FF238DF81830A06A01233246322108F03E
:10A24000BBF80028EAD09DF8183013F00103E5D1DF
:10A25000A06A03930822322108F08AF8039B58B9B8
:10A26000374849F047FBA06A03685B6A9847036870
:10A27000DB68984700255CE0A06A03931A46342106
:10A2800008F076F80028EBD0039BA06A2422412135
:10A2900008F06EF80028E3D0039BA06A0822312161
:10A2A00008F066F80028DBD0A06A036803219B6CE5
:10A2B0009847A06A03685B6A98470368DB68984719
:10A2C000A06A102108F016F8A36A04F12D0299681B
:10A2D0002046FEF7A5FD054658B3A36A94F82D1055
:10A2E0009A682046FEF7A0FDA36A16481A7A597AA2
:10A2F00000919B681449D20849F0FCFA94F82C208C
:10A3000094F82D102046FEF7C5FD94F82E302BB1A1
:10A3100094F82D1001222046FEF79AFDA06A0368EA
:10A320009F6A0A4B0694079396E80C0042F210715C
:10A33000B847284609B0F0BDCC250020D0F9080860
:10A3400070F90808A7F908089FF90808D9A30108B7
:10A3500010B586B004460123806A0DF10302102176
:10A3600008F02AF898B39DF80330DB072FD5A06AD0
:10A37000062301AA112108F01FF840B3BDF90430EB
:10A380009FED146A94F82D2006EE903ABDF9063040
:10A3900007EE103ABDF808305B421BB207EE903A68
:10A3A000F8EEE66AB8EEC77AF8EEE77A66EE866A05
